:020000040800F2
:10000000F0380020950200087F600008DF570008E4
:10001000356000088F2300084D83000800000000B1
:10002000000000000000000000000000FD6B000860
:1000300037250008000000006F680008B76E000850
:10004000AF020008AF020008AF020008AF020008CC
:10005000AF020008AF020008AF020008AF020008BC
:10006000AF020008AF020008AF020008AF020008AC
:10007000AF020008AF020008DD230008ED230008EE
:10008000AF020008FD230008AF020008AF0200081D
:10009000AF020008AF020008AF020008AF0200087C
:1000A000AF020008856F0008AF020008AF02000829
:1000B000AF020008AF020008AF020008AF0200085C
:1000C000AF020008AF020008AF020008AF0200084C
:1000D000AF020008197A0008297A0008397A000866
:1000E000AF020008AF020008AF020008AF0200082C
:1000F000AF020008AF020008AF020008AF0200081C
:10010000AF020008AF020008AF020008AF0200080B
:1001100039740008AF0200089D6F0008AD6F000839
:100120000D240008AF020008AF020008AF0200086B
:10013000AF020008AF020008AF020008AF020008DB
:10014000AF020008AF020008AF020008AF020008CB
:10015000AF020008AF0200081D240008497A000819
:10016000AF020008AF020008AF020008AF020008AB
:10017000AF020008AF020008AF0200080000000054
:10018000AF020008AF02000800F002F800F072F8B9
:100190000AA090E8000C82448344AAF10107DA45E2
:1001A00001D100F067F8AFF2090EBAE80F0013F0C2
:1001B000010F18BFFB1A43F00103184788DD000048
:1001C000A8DD00000A444FF0000C10F8013B13F0CA
:1001D000070408BF10F8014B1D1108BF10F8015BA0
:1001E000641E05D010F8016B641E01F8016BF9D193
:1001F00013F0080F1EBF10F8014BAD1C0C1B09D1EA
:100200006D1E58BF01F801CBFAD505E014F8016B5B
:1002100001F8016B6D1EF9D59142D6D370470000ED
:100220000023002400250026103A28BF78C1FBD8FF
:10023000520728BF30C148BF0B607047642900F0E7
:100240000B81782900F04481002070471FB50DF024
:100250007AFD01F019F90400002000210CF07CFF68
:10026000401C6060002000210CF060FFE0601FBDBA
:1002700010B510BD00F03EFE1146FFF7E7FF0AF093
:10028000F7FC01F0B7F803B4FFF7F2FF03BC08F086
:10029000D0F900000948804709480047FEE7FEE71B
:1002A000FEE7FEE7FEE7FEE7FEE7FEE7FEE7FEE726
:1002B00004480549054A064B70470000716F000865
:1002C00089010008F0320020F0380020F0340020CE
:1002D000F03400207047704753EA020C00F0698048
:1002E0002DE9F04B4FF00006002B1FBFB3FA83F54A
:1002F00003FA05F424FA05F65E4012BF1643B2FA7B
:1003000082F502FA05F4C5F120051EBF22FA05FCAC
:1003100044EA0C04203556EA044C4FEA144418BF52
:10032000641C4FF000084FF00009904271EB030C81
:1003300039D3002919BFB1FA81F701FA07F6B0FAEB
:1003400080F700FA07F6C7F120071EBF20FA07FC66
:1003500046EA0C062037B6FBF4FCA7EB0507103F76
:1003600007F01F0BCBF120060CFA0BFB2CFA06F65C
:1003700044BFB3460026202FA4BF5E464FF0000BBB
:100380005BEA060C08BF4FF0010B19EB0B09ABFB46
:10039000027C48EB0608C01B06FB02CC0BFB03CC1F
:1003A00071EB0C01C1E70B46024641464846BDE8E9
:1003B000F08B13B54FF000004FF00001AFF3008059
:1003C000BDE81C40704700000FB4044910B503AAF3
:1003D000029800F021FB10BC5DF814FB9400002093
:1003E0000FB41CB5074B06AA7B44694600900598DC
:1003F00000F0F9FA0020694600F008FB1CBC5DF82B
:1004000014FB00002106000070B5044685690068F1
:10041000C10601D5302600E02026C00707D070BDF8
:10042000D4E9012130469047206A401C20626D1EAD
:10043000F6D570BD70B5044685690078C00707D150
:1004400070BDD4E9012120209047206A401C206221
:100450006D1EF6D570BD00002DE9F0410646002462
:1004600010687529314616A510D0AFF3008000281A
:1004700002DA404213A507E031688A0701D512A5C8
:1004800002E0490704D511A5012401E0AFF3008083
:1004900000210A2206F1240709E0B0FBF2FCB0FBC0
:1004A000F2F302FB1C00303078541846491C002837
:1004B000F3D123462A463046BDE8F04100F035BA74
:1004C000000000002D0000002B00000020000000B4
:1004D00070B504460D4621461068AFF300802188B0
:1004E000090502D50F4A7A4402E00E4A7A440E32D8
:1004F000002104F1240305E000F00F060009965DD9
:100500005E54491C0028F7D120780023000704D549
:10051000702D02D009B1022311322046BDE870408F
:1005200000F003BA8CD900002DE9F05F894604463B
:100530004FF0000ADFF824B1FB44C0F820A02046A9
:10054000E168884700287DD0252806D0D4E901211C
:100550009047206A401C2062F1E700255F46204654
:10056000E16888472028064607DB312E05D2B819F6
:1005700010F8200C08B10543F1E7A80701D525F0D4
:100580000405C4F81CA00027C4F818A02A2E09D01E
:10059000304608F047F838B304EB8708303EC8F817
:1005A000186019E059F8041B204604EB870291619A
:1005B000E1688847012F064618D1E069002820DA53
:1005C00025F020051DE0D8F8180000EB800006EBB0
:1005D00040003038C8F818002046E16888470646D1
:1005E00008F020F80028EED1012F0AD02E2E08D1D5
:1005F0002046E16888477F1C0646022F45F020050B
:10060000C4DBA069002803DA404245F00105A0617F
:10061000E80701D025F01005A6B1A6F14100192880
:1006200002D8203645F400654A463146204625600A
:100630004D46FFF703FE60B1012807D0ED1D25F000
:10064000070000E007E000F1080978E705F1040978
:1006500075E730467AE7206ABDE8F09F62D900006E
:100660000FB400B58DB010A9099000910B904FF018
:10067000FF300A9000200C90064878440690064807
:1006800078446A4607900F9909A800F0EBF90DB07D
:100690005DF814FB070400001F0400002DE9FF5F54
:1006A0001D464FF0FF3B91464FF000085F46D5E9ED
:1006B0000146A96901987F1C8847296A82468847B4
:1006C0000028F6D1BAF1FF3F0CD0002E24F4C0640C
:1006D00019DD600614D5BAF12B0F09D0BAF12D0F30
:1006E0000ED103E0584604B0BDE8F09F44F48064A6
:1006F000A96901987F1C8847761E8246002E02DD7C
:10070000BAF1300F03D0B9F1000F26D032E0A96959
:10071000761E01987F1C44F400748847002E8246A0
:1007200005DDBAF1780F06D0BAF1580F03D0B9F150
:10073000000F10D01EE0B9F1000F02D0B9F1100F78
:1007400018D1A969761E01987F1C24F4007488478B
:100750008246102002E0082000E00A20814609E0DD
:10076000A96908FB0908761E01987F1C44F40074EF
:1007700088478246002E05DD4946504600F05EF966
:100780000028EDDAE96901988847A00502D46FF0E6
:100790000100A8E7E00725D1600613D5600502D562
:1007A000C8F1000000E0404629680A1D2A60096877
:1007B000220501D5087015E0220701D5088011E057
:1007C00008600FE02868011D29600068210502D536
:1007D00080F8008006E0210702D5A0F8008001E043
:1007E000C0F8008038467EE7032A40F2308010F0DF
:1007F000030C00F0158011F8013BBCF1020F6244BC
:1008000098BF11F801CB00F8013B38BF11F8013B4C
:10081000A2F1040298BF00F801CB38BF00F8013BF9
:1008200011F0030300F02580083AC0F0088051F869
:10083000043B083A51F804CBA0E80810F5E7121D74
:100840005CBF51F8043B40F8043BAFF30080D20793
:1008500024BF11F8013B11F801CB48BF11F8012B5F
:1008600024BF00F8013B00F801CB48BF00F8012B82
:10087000704710B5203AC0F00B80B1E81850203A0C
:10088000A0E81850B1E81850A0E81850BFF4F5AF30
:100890005FEA027C24BFB1E81850A0E8185044BFBA
:1008A00018C918C0BDE810405FEA827C24BF51F827
:1008B000043B40F8043B08BF7047D20728BF31F81B
:1008C000023B48BF11F8012B28BF20F8023B48BF6C
:1008D00000F8012B70474FF0000200B51346944614
:1008E0009646203922BFA0E80C50A0E80C50B1F188
:1008F0002001BFF4F7AF090728BFA0E80C5048BF9C
:100900000CC05DF804EB890028BF40F8042B08BF39
:10091000704748BF20F8022B11F0804F18BF00F835
:10092000012B70477047704770472DE9F0470D461F
:1009300099469246044600F124080168880604D5C9
:10094000E06921F01001216000E00120A84201DDF2
:10095000471B00E00027A1697A1902EB0900081A79
:10096000A0612078C00602D42046FFF74DFD002686
:1009700008E0D4E901211AF806009047206A401CDB
:10098000761C20624E45F4DB2078C0060AD520464E
:10099000FFF73AFD06E0D4E9012130209047206AB4
:1009A000401C2062381EA7F10107F4DC07E0D4E9FF
:1009B000012118F805009047206A401C2062281E7B
:1009C000A5F10105F3DC2046FFF734FD2078000691
:1009D00002D50220BDE8F0870120FBE701694A1C2F
:1009E00002610878704700B58FB0CDE90131002170
:1009F000059105497944CDE9031011466846FFF792
:100A000093FD0FB000BD0000E5FFFFFF0A6802F88C
:100A1000010B0A6070470000074B70B50D467B4420
:100A2000FFF7E1FF0446284600F060FA10B14FF0EE
:100A3000FF3070BD204670BD079900003A2800D2F3
:100A4000303820F02002412A01D3A2F13700884239
:100A500001D34FF0FF3070470268114413780160F2
:100A600018467047D1600549794451610449794479
:100A7000116200211161114600F07EB8EDFFFFFF09
:100A8000F3000000426842B1016811F8013B23B154
:100A9000521EC0E90012184670470121C160881E2D
:100AA000704742685AB1C368016843B983688B4292
:100AB00005D0491E521CC0E90012002070474FF0BB
:100AC000FF3070470FB4002300B589B00CA9009126
:100AD0000B99CB60204B7B440693204B7B440793C0
:100AE00004236FF00042CDE901321D4A7A446B467F
:100AF0000892024600200DF090F909B05DF814FB51
:100B000070B506464FF0FF3015460C46324686B0AB
:100B10000091CDE9010169460020049004A8FFF787
:100B2000D1FF03460498211825B108B10A4600E018
:100B300022462A6000280DD0002B02DD0098884252
:100B400008D03246081B69460094CDE9010404A888
:100B5000FFF7B8FF06B070BDABFFFFFFC3FFFFFF9D
:100B60007500000010B5044600F0EAF90068005D69
:100B700000F0010010BD00002DE9F34F4FF0000A16
:100B80000C4656468DB001200C9001F10C000B90E4
:100B900062690B980121904705002DD0252D2CD09E
:100BA000216A8847C0B162690B9801219047216A88
:100BB00088470028F7D16269411E0B98904700E0F2
:100BC000761CA1690D988847216A88470028F7D1CB
:100BD000E1690D988847DBE7A1690D988847A8422D
:100BE000074601D1761CD3E7E1690D9888477F1C41
:100BF00002D1BAF1000F6FD06BE162690B98002748
:100C00003D46394690472A2804D162690B98012154
:100C100090470125DFF8D08262690B980121904747
:100C2000A0F130010A290AD24745E5DC07EB87012C
:100C300000EB4107303FDFD445F01005ECE7E90653
:100C400001D46FF000476C280AD04C2814D06828D3
:100C500015D06A280DD074281CD07A281AD01DE02F
:100C600062690B98012190476C2802D045F0040579
:100C700014E045F002050DE045F020050AE0626948
:100C80000B9801219047682802D045F0080505E03F
:100C900045F4006562690B9801219047C4E901574A
:100CA00065283DD019DC58287AD00CDC452837D08F
:100CB00004DC252826D041289ED131E046282FD0BB
:100CC000472899D12CE05B2877D0612828D0632869
:100CD0007CD0642823D15AE0F6E06F2848D008DCA5
:100CE00066281DD067281BD0692821D06E2816D110
:100CF00027E0702845D0732868D0752847D0782819
:100D00000DD14DE0A1690D988847252805463FF48F
:100D100069AFE1690D9888476D1C3FF46AAFD8E070
:100D20000D9923466A466FF001000DF076F8C5E094
:100D300045F0400023464FF000026060A80736D41B
:100D40003EE0E8077FF447AF2068011D216000689E
:100D5000290501D506701BE7290701D5068017E78D
:100D6000A90703D5F117C0E9006111E706600FE795
:100D700045F0400023464FF008026060A80716D4F3
:100D80001EE040F60E0125EA0100606016E045F025
:100D9000400023464FF00A026060A80707D40FE026
:100DA00045F040006060A80708D5234610220D9941
:100DB0006FF00100AFF3008080E007E010222346CF
:100DC0000D996FF00100FFF769FC77E04FF0000923
:100DD00063284F46C8464B46CB4602D05B2806D018
:100DE00038E0E80601D40120A060012732E0626902
:100DF000D4F80CB00B98012190475E2807D14FF032
:100E0000010949466269D4F80CB00B9890472169F2
:100E100039B900210A4603AB43F82120491C0829AF
:100E2000FADBD8B3216949B308F1010862690B986C
:100E3000012190475D28F4D1B9F1000F09D00020BD
:100E400003A951F82020D24341F82020401C082853
:100E5000F7DB03AB2069002820794FEA40701ED0F1
:100E60005B462246CDF80080CDE901970D99002818
:100E70006FF0010020DAAFF300801FE0C11703AA72
:100E800000EBD1614B1121F01F0102EB8302411AEB
:100E900013680120884003431360C7E719E00D99E8
:100EA000224600286FF00100009702DAAFF30080BD
:100EB00004E0AFF3008001E0AFF3008000280ADA1D
:100EC000401C06D10C9820B14FF0FF300FB0BDE8A8
:100ED000F08F5046FAE7E90701D10AF1010A06440A
:100EE00000200C9054E60000CCCCCC0C007B00F031
:100EF00080007047754600F0C3FAAE4605006946AB
:100F0000534620F00700854618B020B5FFF7D0F90A
:100F1000BDE820404FF000064FF000074FF00008FA
:100F20004FF0000B21F00701AC46ACE8C009ACE87B
:100F3000C009ACE8C009ACE8C0098D4670470000A4
:100F400010B500F0A1FA001D10BD00BF0DC20000D9
:100F50002DE9FF4F064689B00878FF2806D0491CC6
:100F60002D2805D000244FF0000908E000200CE0F7
:100F70000124F8E709EB8903491C00EB43090878D1
:100F8000FF28F7D114B1C9F100008146107800257F
:100F90002C46AA4629462D2801D02B2804D1521CC4
:100FA0002D2813D0002082468B461078FF280FD0C2
:100FB0004FF0000C0A21521CA5FB017804FB0181B3
:100FC00005FB0C11C5194BEB0104EEE70120EAE724
:100FD000002108464FF00000BAF1000F02D000EBEC
:100FE00080004008C0F38158B8F1010F01DD4FF0D7
:100FF000FF380C9809EB000755EA040009D04FF0C0
:10100000020917F5FA7F0BDA4FEACA70C6E900B099
:1010100012E04FEACA70C6E900B00DB0BDE8F08F2B
:10102000B7F5FA7F0DDDF0487844D0E90010C6E945
:10103000001040EACA70706000F02AFAC0F8009010
:10104000EBE7391E02DAC8F1000200E0424600DA9E
:10105000794206A800F020FA06AB93E8070003AB3C
:1010600083E8070044F23E005BEA04010090584622
:1010700004D144F21E012C465D460091210C090466
:10108000014306D10099240444EA15442D04103983
:10109000009104F07F41014306D10099240244EA03
:1010A00015642D020839009104F07041014306D106
:1010B0000099240144EA15742D01091F009104F0E0
:1010C0004041014306D10099A40044EA9574AD0063
:1010D000891E009104F00041084304D100986D1965
:1010E0006441401E009042466846002FCDE901450C
:1010F00003A902DD00F0E9FE01E000F0BEFEBAF156
:10110000000F04460D4601D084F0004440F2FF7702
:1011100024F00040284303D0C4F30A50B84212D14F
:1011200000F0B6F9C0F80090C4F30A50B8420AD1F2
:10113000AE487844D0E90010C6E9001004F0004140
:101140000843706069E7C6E9005466E72DE9FF4F80
:101150001F464FF0000A4FF0FF38454691B0D7E9DF
:101160000146CDF83CA000F08FF9C0680168405CF2
:101170001090B96912986D1C8847396A8146884772
:101180000028F6D1B9F1FF3F0AD0002E24F4D06434
:1011900011DDB9F12B0F08D0B9F12D0F0BD102E001
:1011A000404615B03AE744F48064B96912986D1C62
:1011B0008847761E8146600504A901D52D2000E0F0
:1011C0002B20002E01F1010B0DF130088DF81000DD
:1011D0003FDDB9F1690F08D0B9F1490F05D0B9F178
:1011E0006E0F02D0B9F14E0F1CD13B4601A80095FD
:1011F00080E85002DDE912126FF002000CF011FEDF
:10120000C11CCED10EE0B96912986D1C8847814689
:101210001398761E44F4007405600F98401C002E4D
:101220000F9016DDB9F1300FEDD0B9F1780F02D083
:10123000B9F1580F0DD10F9801280AD13B46CDE9DD
:101240000054DDE91212001F02960CF0E8FDC11CEB
:10125000A7D1109989453ED144F0800406E0139946
:10126000681CAAF1010A44F400740860B9696D1C95
:101270001298761E884730288146F0D02BE01099CE
:10128000894505D1200603D4761E44F0800418E079
:10129000484607F0C7F908B3761E0DF123018B45C8
:1012A00044F4007408D2A9F130000BF8010B2006B9
:1012B00007D5AAF1010003E0200602D40AF10100DB
:1012C0008246A00502D51399681C0860B969129876
:1012D0006D1C88478146002ED1DC53E0002E51DD85
:1012E000B9F1650F02D0B9F1450F4BD1A00549D531
:1012F000B9696D1C1298761E24F440748847002E3C
:1013000081460CDD2B2804D0B9F12D0F07D144F410
:101310008074B96912986D1C8847761E8146E00575
:1013200001D52D2100E02B2108F8011BCDF800800C
:1013300021E0761E0DF13901884544F400740CD289
:10134000A9F1300010F0FF0088F8000002D10099E8
:10135000884509D908F1010806E0E00501D52448CF
:1013600001E042F20F708246B96912986D1C8847FD
:10137000814613980560002E04DD484607F052F9B7
:101380000028D6D1F96912988847FF2053468BF878
:10139000000088F8000000200A900B9004AA0CA915
:1013A0000AA8FFF7D5FDA00502D46FF00100F8E60A
:1013B00014F0240F0AD0E00714D13868DDE90A12CE
:1013C000031D3B600068C0E900120BE00AA96846F3
:1013D00007F0C2F8E00705D13868009A011D3960AE
:1013E000006802602846DCE638CF00002ECE000000
:1013F000F1D8FFFF0446AFF300802046FEF743FF1D
:101400004FF0013C50F8042B51F8043B9A4221D193
:10141000A2EB0C03934313EACC1317D150F8042B1F
:1014200051F8043B9A4215D1A2EB0C03934313EA03
:10143000CC130BD150F8042B51F8043B9A4209D13C
:10144000A2EB0C03934313EACC13DBD04FF0000064
:10145000704700BFD01A01BAB1FA81F101F018014A
:1014600022FA01F0CB40C1F12001DBB2C0B2C01AB8
:101470002CFA01F3D11A914311EAC311E6D1704756
:10148000004870478C32002000487047AC32002082
:10149000004870478C3200202DE9F04781461646FF
:1014A0008AB0334878440DC88DE80D003048784440
:1014B000801C03AC0DC884E80D0041F69B30084445
:1014C000372190FBF1F290FBF1F5A5F1800501FBCE
:1014D00012041B3C02D56442012000E00020DFF82A
:1014E00090A080460027FA44AAF1BE0A0DE0E0076A
:1014F00009D03246684607EB47010AEB810100F04C
:10150000D0FC8DE8070064107F1C002CEFD1184F31
:101510007F44AC3F18E0E80714D007EB04100DF14E
:10152000180A90E80E008AE80E00C068F04201D167
:1015300098190890324606A903A800F0B2FC03AB44
:1015400083E807006D10641C002DE4D13246694623
:10155000B8F1000F03A802D000F07BFC01E000F01E
:10156000A0FCC9E90001C9F808200AB0BDE8F0876D
:1015700084CA000010B5FFF78BFF006810BD10B5DE
:101580000446FFF785FF046010BD00002DE9FF4F02
:101590001F464FF03C0987B04FF00042DDE91410C0
:1015A00001F10108DDF858A002EA40500390002044
:1015B00004908346054604460590B969461E08987E
:1015C0008847AAF1010A0290BAF1000F37DD0298AC
:1015D0002E2815D01021FFF731FA00282ADB4FF012
:1015E000010B0499014316D0B9F1000F0BDB4A46F9
:1015F000C11700F0F1F905430C43A9F1040905E016
:101600000120059007E008B145F001050120049094
:10161000059800B9361DB969089808F1010888478E
:10162000BBF1000FAAF1010A0290CDD00999C1F8CF
:101630000080C9E70298702808D0502806D0F969C0
:1016400008988847BBF1000F14D04FE000200290AB
:101650000120BBF1000F049009D0B969089808F186
:1016600001088847AAF10109B9F1000F07DCF969FF
:10167000089888476FF001000BB0BDE8F08F2B2869
:1016800004D02D280CD14FF0FF300490B969089890
:1016900008F101088847A9F10109B9F1000FE6DD59
:1016A000411CE4D00A21FFF7C9F90028DFDB0299C9
:1016B00008F1010801EB810100EB41000290B969DA
:1016C000089888470A21FFF7B9F9099AA9F1010991
:1016D000B9F1000FC2F8008001DD0028E7DAF969EE
:1016E000089888470499029800FB016655EA0400AF
:1016F00004D004F04041090002D006E0039898E0CD
:10170000A40044EA9574AD00B61E04F00041080040
:1017100002D16D196441761E159810F0240F03D084
:101720004FF00B095C4803E04FF028096FF07D0093
:101730008246564507DAAAEB06018944B9F1410F02
:1017400001DD4FF0410901200021A9F1010200F063
:1017500043F9024628400B462140084301D00121AD
:1017600000E00021501E029143F1FF31284021404A
:10177000084301D0012000E000200299834651EA8D
:101780000B014FD0002108464FF00000039900F4F0
:10179000400039B100EB80004FF4400100EBD07005
:1017A00001EA60008015012802DD4FF0FF3000E003
:1017B00013D0401C36D0029860B3BBF1000F0CD19F
:1017C0004A460120002100F007F928402140084343
:1017D00001D0012000E00020E0B101204A460021B4
:1017E00000F0FAF8034640190A4661412D1A8C416F
:1017F00011D3B9F1400F09DD159810F0240F02D074
:10180000AAF1340603E0AAF1170600E0761C0025D1
:101810004FF0004406E05B1E42F1FF3220EA030570
:1018200021EA0204CAF10100B04206DA1B4903981A
:1018300008430190002000900EE0039AC4F3D321E6
:10184000E80A0A43164940EA44500A433146CDE9C2
:101850000002684606F0DCFE159810F0240F0BD04D
:101860001598C00715D13868DDE90012031D3B60EB
:101870000068C0E900120CE002A8694606F06CFEA0
:101880001598C00705D13868029A011D39600068B3
:1018900002604046F0E6000002FCFFFF0000F07F1F
:1018A0000000F03F2DE9FF4F92461D4685B04FF0F6
:1018B0000041DDE9124BDDE914727F1E01EA4B5055
:1018C000414940F0FF4940EA0108002122F0200090
:1018D0004928049102D04E2828D04CE03BA0012694
:1018E00007C88DE80700A9690698641C88477F1E11
:1018F000014606D41DF8060018B121F020018142EE
:101900000BD0E96906988847032E34D0082E32D0D0
:101910006FF0010009B0BDE8F08F761C032E01D0F6
:10192000082EE0D1601CCAF80000DCE7A96906981F
:10193000641C88477F1E2AD420F02000412826D12D
:10194000A9690698641C88477F1E20D420F02000D7
:101950004E281CD1A9690698641C88477F1E48F44C
:10196000002849F48009CAF8004001D4282806D08C
:10197000E969069888475FEACB7012D022E0A9692E
:101980000698641C88477F1E01D4002803DAE969A1
:1019900006988847BCE72928F1D1641CCAF80040A2
:1019A000E9E71BF0240F07D028680499031D2B607A
:1019B0000068C0E9001805E02868021D2A60006878
:1019C000C0F800902046A5E70000F07F494E464948
:1019D0004E49545900000000B2F120030AD5C2F16B
:1019E000200301FA02F120FA03F300FA02F041EABF
:1019F0000301704700FA03F14FF00000704720F038
:101A00007F4C80EA030023F07F47ACEB070303F52C
:101A10007C5300F0004003F1FF032DE980494FEAB9
:101A2000154B09B44FEA144325EA0B4E24EA034848
:101A30000FF2042606EB132749083E785FEA3202CC
:101A400003FB0667C7F5000707FB06F64FEA5437A6
:101A50004FEAD64606F1020607FB066CCCF1005CA5
:101A60004FEA1C472CEA074C07FB06F40CFB06F573
:101A700004EB15464FEA961634BF00204FF00040A5
:101A80004FEAD13706FB07FC4FEA1C4C0CFB0BF767
:101A9000D21B03FB0CF761EB07010CFB0EF7B0EB5D
:101AA000074072EB17420CFB08F734BFA2EB07426A
:101AB000B2EB074261EB17414FEA0C444FEA910742
:101AC00006FB07FC4FEA1C4C0CFB0BF7B0EBC740C6
:101AD00072EB573203FB0CF734BFA2EBC742B2EBF9
:101AE000C74261EB57310CFB0EF7B0EBC70072EB4E
:101AF00057720CFB08F734BFA2EBC702B2EBC70268
:101B000061EB5771039F4FEA816141EA921104EB47
:101B1000CC044FEAD1374FEA826206FB07FC42EA67
:101B200090124FEA80604FEA1C4C0CFB0BF7D21B63
:101B300003FB0CF761EB07010CFB0EF7B0EB074062
:101B400072EB17420CFB08F734BFA2EB0742B2EB73
:101B5000074261EB17414FEA8C554FEA910704EBBE
:101B60009C2406FB07FC4FEA1C4C0CFB0BF7B0EB6C
:101B7000C74072EB573203FB0CF734BFA2EBC742EE
:101B8000B2EBC74261EB57310CFB0EF7B0EBC7006D
:101B900072EB57720CFB08F734BFA2EBC702B2EB33
:101BA000C70261EB577115EB4C254FEA816141EAA1
:101BB00092114FEA82624FEAD13742EA901206FB55
:101BC00007FC44F100044FEA80604FEA1C4C0CFB18
:101BD0000BF7D21B03FB0CF761EB07010CFB0EF7B5
:101BE000B0EB074072EB17420CFB08F734BFA2EBD7
:101BF0000742B2EB074261EB174115EB1C154FEAA8
:101C0000813141EA92414FEA823242EA90424FEA00
:101C100080304FEA0C7644F1000448EA03434EEA70
:101C20000B484FF0000EB2EB080C71EB030724BF1A
:101C3000624639464EEB0E0E4FF0000B0018524133
:101C400049414BEB0B0BB2EB080C71EB03077BF13B
:101C5000000B24BF624639464EEB0E0E4FF0000BD0
:101C60000018524149414BEB0B0BB2EB080C71EBE6
:101C700003077BF1000B24BF624639464EEB0E0E84
:101C800051EA020718BF46F0010616EB0E7655F131
:101C9000000254F1000103D5BDE88901BDE80088C8
:101CA000BDE88901BDE80048B619524141EB010188
:101CB000A3F10103704780807F7E7D7C7B7A7978F9
:101CC000777676757473727171706F6E6E6D6C6C01
:101CD0006B6A6A69686867666665646463636261A3
:101CE0006160605F5F5E5E5D5D5C5C5B5B5A5A5924
:101CF0005958585757565655555554545353525290
:101D00005251515050504F4F4F4E4E4D4D4D4C4CE7
:101D10004C4B4B4B4A4A4A49494948484847474730
:101D2000474646464545454444444443434343426D
:101D3000424242414141000046EA0646A3F5705343
:101D40004FEA164646EA42564FEAD22242EA41524A
:101D500010B54FEAD121A3F1010300F017F820F0EC
:101D6000004000F1010C00F0004701EB005011466B
:101D7000BCF5006F40EA070000D210BD02484FF0EA
:101D8000000140EA070010BD0000F07F002B26D4C0
:101D9000770021D01CB54FEA370703B44FF010008D
:101DA0004FF010014FF000000FBCBDE810400BF1E8
:101DB000010BBBF1010F08BF5FEA170722BF12F149
:101DC000010211F101014FF0004143F1000300F065
:101DD000004043EA00007047F9D35708DAE746EAC3
:101DE000064613F1400F4FEA16461FDD13F1200F90
:101DF000DFBF16430A46002120335B42C8D0C3F13F
:101E0000200746EA064602FA07F74FEA164646EA70
:101E10000706C3F1200722FA03F201FA07F721FAB5
:101E200003F14FF0000342EA0702B1E746EA020677
:101E300046EA06464FEA164646EA0106BCBF46EAAF
:101E40000646360C4FF000034FF000024FF0000141
:101E50009EE72DE9C048934630B491E8380007C8A2
:101E600031EA400C48BF34EA430C03D5FFF7C7FD05
:101E7000FFF78CFFF0BCBDE800882DE9C048934611
:101E800030B491E8380007C831EA400C48BF34EA62
:101E9000430C03D5FFF7B3FDFFF74EFFF0BCBDE8E1
:101EA00000882DE9C048934630B491E8380007C84F
:101EB00010F0804F08BF13F0804F03D100F019F8E5
:101EC000FFF764FFF0BCBDE800882DE9C0489346E9
:101ED00030B491E8380007C810F0804F08BF13F005
:101EE000804F03D100F005F8FFF726FFF0BCBDE8F6
:101EF000008820F07F4780EA030023F07F4C07EB47
:101F00000C03A3F57C5300F00040A3F1FE0392F014
:101F1000000F00F0B38095F0000F00F077802DE9FE
:101F200001494FEA11404FEA144621EA004800FBFC
:101F300006FC24EA064708FB06F607FB08F800FB48
:101F400007F718EB06484CEB164C4FEA124B18EB10
:101F500007484FEA15464CEB174022EA0B4E0BFBA5
:101F600006FC25EA06470EFB06F607FB0EFE0BFBFA
:101F700007F71EEB064E4CEB164C4FF000061EEB1F
:101F8000074E4CEB174B18EB0B0840F1000018EB19
:101F90000E0B58EB000840F100008F1A4FF00001C3
:101FA0003CBFC943661B14BFB5EB040C00213CBF0A
:101FB000C943F61B4FEA17444EEA8E0E27EA044542
:101FC0004FEA1C4704FB07622CEA074C05FB07F7A6
:101FD0000CFB05F604FB0CFC16EB074642EB174224
:101FE00016EB0C4642EB1C421BEB060658EB0202BA
:101FF000414146EA9E0601D5BDE80189B619524124
:1020000041EB0101A3F10103BDE801894FEA144549
:102010004FEA114724EA054621EA074C05FB07F47D
:1020200006FB07F70CFB06F105FB0CFC11EB074167
:1020300044EB17444FEA124711EB0C4144EB1C44AC
:1020400022EA074C05FB07F206FB07F70CFB06F636
:1020500005FB0CFC16EB074642EB174216EB0C4651
:1020600042EB1C456A1854F1000148BF7047B6198D
:10207000524141EB0101A3F10103704795F0000FBC
:1020800037D04FEA11424FEA144721EA024624EAC8
:10209000074C02FB07F106FB07F70CFB06F402FBFB
:1020A0000CFC14EB074441EB17414FEA154714EBC6
:1020B0000C4441EB1C4125EA074C02FB07F506FBEB
:1020C00007F70CFB06F602FB0CFC16EB074645EB8C
:1020D000174516EB0C4645EB1C42121951F1000155
:1020E00048BF7047B619524141EB0101A3F101030A
:1020F00070474FEA14454FEA114724EA054621EAA2
:10210000074C05FB07F106FB07F70CFB06F24FF047
:10211000000605FB0CFC12EB074241EB174112EBEA
:102120000C4251EB1C4148BF7047921841EB010132
:10213000A3F10103704770B50546AC6B206C00F04D
:10214000500050BB206C40F4007020642068806810
:1021500000F04050E8B9207ED8B92068C06A00F489
:10216000700020B12068806800F4806088B9206821
:10217000406820F0200021684860206C20F48070C6
:102180002064206C00F4805018B9206C40F00100ED
:102190002064204600F016FB0BE0206C00F01000DD
:1021A00018B1204600F010FB03E0A06BC16C28467C
:1021B000884770BD70B50546AC6B40202064606CEC
:1021C00040F004006064204600F0FEFA70BD70B577
:1021D0000446A56B284600F0F6FA70BD55494A68DA
:1021E00022F440324A604A6843681A434A600268EF
:1021F000526822F4807203685A6002685368026968
:1022000043EA022203685A600268526822F0407270
:1022100003685A600268526883681A4303685A6008
:102220000268926822F4006203689A600268926809
:10223000C3681A4303689A603F4B826A9A4218D077
:102240000268926822F0706203689A60026892687D
:10225000836A1A4303689A600268926822F04052C7
:1022600003689A6002689268C36A1A4303689A60B6
:102270000BE00268926822F0706203689A6002685C
:10228000926822F0405203689A600268926822F0D5
:10229000020203689A6002689368027E43EA42027F
:1022A00003689A602022125CA2B10268526842F46C
:1022B000006203685A600268526822F46042036850
:1022C0005A6002685368426A521E43EA4232036807
:1022D0005A6005E00268526822F4006203685A609E
:1022E0000268D26A22F470020368DA620268D36A72
:1022F000828B521E43EA02520368DA6202689268D5
:1023000022F4007203689A600268936890F83020A3
:1023100043EA422203689A600268926822F480626B
:1023200003689A6002689368426943EA82220368FC
:102330009A607047002301400100000F70B5044609
:102340000D461646EE2004F05BFCB12004F058FC6C
:10235000232004F055FC200A04F052FCE0B204F003
:102360004FFC280A04F04CFCE8B204F049FCF0B23F
:1023700004F046FCFF2004F043FCFC2004F040FC89
:10238000FF2004F03DFCFF2004F03AFC70BD00BFCC
:10239000FEE7000010B50E480078012804D002289E
:1023A00008D0032812D10BE000221021094800F0C8
:1023B00003FF0BE000222021064800F0FDFE05E0AF
:1023C00000220121044800F0F7FE00BF00BF10BD4D
:1023D000A8000020000802400004024010B5024896
:1023E00000F0EAFB10BD0000F008002010B5024824
:1023F00000F0E2FB10BD0000D007002010B502483D
:1024000000F0DAFB10BD00009008002010B5024873
:1024100000F0D2FB10BD00009C02002010B5024865
:1024200000F0CAFB10BD000030080020014608780B
:1024300010381823B0FBF3F20848805CC865032A03
:1024400005D908686FF30900001D886503E0086876
:102450006FF309008865886D7047000056DE00083C
:10246000014600208A6A8B69CBB932B1012A0DD0AE
:10247000022A03D0032A10D10EE000BFCB6A03F07A
:102480008073B3F1807F00D1012007E0CB6AB3F104
:10249000C07F00D1012001E000E000BF34E08B6983
:1024A000B3F5005F1AD132B1012A07D0022A03D056
:1024B000032A11D10AE000BF01200EE0CB6A03F02D
:1024C0008073B3F1807F00D1012006E0CB6AB3F1C5
:1024D000C07F00D1012000E000BF15E032B1012A29
:1024E00005D0022A04D0032A0CD103E000BF00BFAC
:1024F000012008E0CB6A03F08073B3F1807F00D144
:10250000012000E000BF00BF704730B504682468B8
:1025100024F4802405682C60046863608468402C7F
:1025200004D10468A2600468E16003E00468A1606B
:102530000468E26030BD704772B600BFFEE700007D
:1025400001460846024B33F8100002B290B27047C1
:10255000E600002001460846024B33F8100002B2A4
:1025600090B27047140B002030B5A0F11002D417C0
:1025700002EB5474E410094D2B5DD41702EB547434
:10258000E410A2EBC4050124AC401C4014B10122AC
:102590000A7001E000220A7030BD0000080B002024
:1025A00030B50246D41702EB5474E410094D2B5D8C
:1025B0000246D41702EB5474E410A2EBC4050124C4
:1025C000AC401C4014B101220A7001E000220A70E4
:1025D00030BD0000DA00002010B51648002101606F
:1025E00001710821302009F0BAFF022000F0C4FC7C
:1025F000092009F0A3FF0F49C8700A2009F09EFFC7
:102600000C4908710921302009F0A9FF032000F0CE
:10261000B3FC062009F092FF06490870072009F074
:102620008DFF04494870082009F088FF014988702F
:10263000084610BDA900002038B5024600200090D1
:1026400000BF92F83C00012801D1022038BD0120D2
:1026500082F83C0000BF0868092816D91068C068D5
:102660000C780A3C04EB44050724AC40A0431468F2
:10267000E0600C780A3C04EB44048868A0401468CD
:10268000E46820431468E06013E0106800690C7887
:1026900004EB44050724AC40A043146820610C7887
:1026A00004EB44048868A04014682469204314683B
:1026B00020614868072817D21068406B0C79641EA7
:1026C00004EB84051F24AC40A043146860630888B1
:1026D00080B20C79641E04EB8404A0401468646B1F
:1026E00020431468606331E048680D2817D21068F1
:1026F000006B0C79E41F04EB84051F24AC40A0435D
:1027000014682063088880B20C79E41F04EB840409
:10271000A0401468246B20431468206316E01068FE
:10272000C06A0C790D3C04EB84051F24AC40A04327
:102730001468E062088880B20C790D3C04EB8404D4
:10274000A0401468E46A20431468E062194B1A4CF4
:102750001068A04206D10868122803D1586840F4D6
:1027600080005860144C1068A0421CD108681028E2
:1027700002D00868112816D1586840F4000058604B
:10278000086810280FD10D4800680D4CB0FBF4F01C
:1027900000EB80004000009002E00098401E009096
:1027A00000980028F9D100BF002082F83C0000BF4B
:1027B00000BF4BE70023014000200140A40000209F
:1027C00040420F00704770477047000070B50446E4
:1027D00000250CB9012070BD1549A06A884200D0BF
:1027E00000BF206C30B9204600F024F8002060645F
:1027F00084F83C00206C00F0100088B9206C20F4B4
:10280000885040F0020020642046FFF7E7FC0020DB
:102810006064206C20F0020040F00100206400E0C1
:10282000012500BF002084F83C0000BF2846D2E705
:102830000100000F10B586B00446142101A8FEF770
:102840004AF835492068884263D100BF00200090D3
:102850003248006840F480703049086008460068DB
:1028600000F48070009000BF00BF00BF0020009007
:102870002A481438006840F00400284914390860D8
:102880000846006800F00400009000BF00BF00BFD1
:10289000002000900846006840F0010008600846EB
:1028A000006800F00100009000BF00BF0C20019004
:1028B000032002900020039001A9194800F070FB4A
:1028C00014200190032002900020039001A91548D4
:1028D00000F066FB1448154908600020486000219C
:1028E00012488160C1604FF480610161490041611B
:1028F000890081614911C16100210162416200F0DA
:102900007BFA08B1FFF718FE00BF0848A063846394
:1029100000BF06B010BD0000002001404438024056
:102920000008024000000240106402409C020020A7
:10293000F8B504460D4616460020009000BF94F8F6
:102940003C00012801D10220F8BD012084F83C00A0
:1029500000BF2068806800F00100A0B9206880688E
:1029600040F0010021688860554800685549B0FB77
:10297000F1F000EB4000009002E00098401E009053
:1029800000980028F9D12068806800F48070B0F5C4
:10299000807F05D12068806820F48070216888607D
:1029A0002068806800F0010000287ED0206C40F292
:1029B0000161884340F4807020642068406800F41E
:1029C000806028B1206C20F4005040F480502064D6
:1029D000206C00F48050B0F5805F04D1606C20F072
:1029E0000600606401E00020606400BF002084F8FD
:1029F0003C0000BF344F3548A16BC8633448A16B1D
:102A000008643448A16BC8646FF022002168086034
:102A10002068406840F080602168486020688068D5
:102A200040F4807021688860226802F14C013346CE
:102A30002A46A06B00F056FA786800F01F0018BB19
:102A400025492068884213D024492068884204D14F
:102A5000381D006800F01F0050B1214920688842ED
:102A60002BD11948001D006800F01F00102824D247
:102A70002068806800F04050F8B92068806840F015
:102A800080402168886018E013492068884214D18A
:102A90002068806800F0405078B92068806840F075
:102AA00080402168886008E0FFE7206C40F010005B
:102AB0002064606C40F001006064002044E7000086
:102AC000A400002040420F000023014037210008ED
:102AD000CF210008B521000800200140002101405D
:102AE0000022014070B50446A56D00F06BFB064660
:102AF00094F83500022808D08020606500BF0020CF
:102B000084F8340000BF012070BD2068006820F008
:102B10001600216808602068406920F08000216864
:102B20004861206C08B9A06C28B12068006820F0CA
:102B30000800216808602068006820F00100216812
:102B4000086010E000F03EFB801B05280BD9202018
:102B50006065032084F8350000BF002084F834004D
:102B600000BF0320D0E72068006800F001000028C3
:102B7000E8D194F85C103F208840A860012084F8D8
:102B8000350000BF002084F8340000BF00BFBBE761
:102B9000014691F83500022803D0802048650120C5
:102BA0007047052081F835000868006820F00100B2
:102BB0000A6810600020F3E7F8B504460020009092
:102BC0008C4800684FF41651B0FBF1F7A56D2E68E4
:102BD00094F85C1008208840304098B12068006864
:102BE00000F0040070B12068006820F00400216843
:102BF000086094F85C1008208840A860606D40F080
:102C00000100606594F85C1001208840304068B194
:102C10002068406900F0800040B194F85C10012009
:102C20008840A860606D40F00200606594F85C1018
:102C300004208840304068B12068006800F002003D
:102C400040B194F85C1004208840A860606D40F0AA
:102C50000400606594F85C1010208840304078B320
:102C60002068006800F0080050B394F85C10102051
:102C70008840A8602068006800F4802080B1206847
:102C8000006800F4002028B9206CC8B12046216CEF
:102C9000884715E0A06C98B12046A16C88470FE0EA
:102CA0002068006800F4807028B92068006820F06F
:102CB000080021680860206C10B12046216C88470C
:102CC00094F85C10202088403040002865D02068AF
:102CD000006800F0100000285FD094F85C102020FD
:102CE0008840A86094F83500052828D1206800683D
:102CF00020F01600216808602068406920F08000FC
:102D000021684861206C08B9A06C28B1206800686F
:102D100020F008002168086094F85C103F2088408B
:102D2000A860012084F8350000BF002084F834003A
:102D300000BF206D10B12046216D8847F8BD206886
:102D4000006800F4802080B12068006800F4002052
:102D500028B9606C10B12046616C88471DE0E06BBB
:102D6000D8B12046E16B884717E02068006800F47E
:102D7000807068B92068006820F010002168086041
:102D8000012084F8350000BF002084F8340000BF23
:102D9000E06B10B12046E16B8847606D38B3606D21
:102DA00000F00100F0B1052084F8350020680068CB
:102DB00020F001002168086000BF0098401C0090CE
:102DC000B84200D905E02068006800F00100002842
:102DD000F3D100BF012084F8350000BF002084F843
:102DE000340000BFE06C10B12046E16C884700BFA2
:102DF000A4E70000A40000202DE9F04104460025CE
:102E000000F0E0F9074614B90120BDE8F081606ADE
:102E100000B100BF022084F8350000BF002084F814
:102E2000340000BF2068006820F0010021680860BD
:102E30000AE000F0C7F9C01B052805D9202060650D
:102E4000032084F83500E0E72068006800F0010006
:102E50000028EED12068056821480540D4E9010129
:102E60000843E16808432169084361690843A1698F
:102E70000843E1690843216A08430543606A04285E
:102E800003D1D4E90B01084305432068056020689D
:102E9000456925F00705606A0543606A04280DD17D
:102EA000A06A0543E06A48B12046FFF7D9FA28B185
:102EB00040206065012084F83500A6E72068456160
:102EC0002046FFF7B3FA064694F85C103F2088408E
:102ED000B06000206065012084F83500002094E790
:102EE0003F8010F02DE9F04704460D4616461F4678
:102EF0004FF00008D4F8589000BF94F8340001282F
:102F000002D10220BDE8F087012084F8340000BF20
:102F100094F83500012825D1022084F835000020DE
:102F200060653B46324629462046FFF7EEFA94F8A4
:102F30005C103F208840C9F808002068006840F015
:102F4000160021680860206C28B12068006840F0F5
:102F50000800216808602068006840F001002168CE
:102F6000086006E000BF002084F8340000BF4FF086
:102F700002084046C6E7000070B5044600F022F99A
:102F800006462546681C10B104480078054400BF79
:102F900000F018F9801BA842FAD370BDA0000020F1
:102FA000F8B502460B460025002400200021D6E09B
:102FB000012606FA01F51E6806EA0504AC4274D142
:102FC0001E7906F00306012E04D01E7906F00306D2
:102FD000022E13D190684F000326BE40B0434F002D
:102FE000DE68BE4030439060506801268E40B0439A
:102FF0001E79C6F300168E40304350601E7906F0ED
:103000000306032E09D0D0684F000326BE40B0430C
:103010004F009E68BE403043D0601E7906F0030624
:10302000022E13D1CF0802F1200656F827004E07D2
:10303000F70E0F26BE40B0434F07FF0E1E69BE407D
:103040003043CF0802F1200646F8270010684F00F1
:103050000326BE40B0431E7906F003064F00BE4073
:10306000304310605E6806F44036002E76D000BF14
:10307000002600963C4E366846F480463A4F3E6045
:103080003E46366806F48046009600BF00BF374EC5
:103090008F0856F827008E07370F0F26BE40B04323
:1030A000334EB24202D1002624E057E0314EB24204
:1030B00001D101261EE0304EB24201D1022619E0B4
:1030C0002E4EB24201D1032614E02D4EB24201D160
:1030D00004260FE02B4EB24201D105260AE02A4E0B
:1030E000B24201D1062605E0284EB24201D10726A0
:1030F00000E008268F073F0FBE4030431B4E8F086D
:1031000046F82700224E3068A0435E6806F4801619
:1031100006B120431E4E3060361D3068A0435E6805
:1031200006F4001606B12043194E361D3060184EC5
:10313000361F3068A0435E6806F4003606B12043AF
:10314000134E361F3060361F3068A0435E6806F4A9
:10315000803606B120430E4E083E3060491C1029CF
:10316000FFF426AFF8BD00004438024008380140A3
:10317000000002400004024000080240000C02402F
:10318000001002400014024000180240001C0240DF
:10319000083C0140024613690B400BB1012000E0DE
:1031A0000020704710B5426921EA020302EA0104D7
:1031B00043EA0443836110BD0AB1816101E00B045D
:1031C0008361704701480068704700009800002044
:1031D00070B504460CB9012070BD94F83D0028B9C3
:1031E000002084F83C00204600F0DAF8242084F81F
:1031F0003D002068006820F0010021680860206818
:10320000006840F40040216808602068006820F4ED
:1032100000402168086000F037FB05465C496068A3
:10322000884206D85B48854201D2012007E0002091
:1032300005E05948854201D2012000E00020012824
:1032400000D1C9E75548B5FBF0F62068406820F08A
:103250003F003043216848604D496068884201D88A
:10326000701C07E04FF4967070434FF47A71B0FB16
:10327000F1F0401C2168096A21F03F0108432168F0
:10328000086243496068884214D8681E6168490032
:10329000B0FBF1F0401CC0F30B00042801D2042065
:1032A0003DE0681E61684900B0FBF1F0401CC0F3CE
:1032B0000B0034E0A06838B9681E616801EB410179
:1032C000B0FBF1F0401C0AE0681E616801EBC1022E
:1032D00002EB0111B0FBF1F0401C40F48040C0F360
:1032E0000B0008B901201AE0A06848B9681E61689F
:1032F00001EB4101B0FBF1F0401CC0F30B000CE00E
:10330000681E616801EBC10202EB0111B0FBF1F034
:10331000401CC0F30B0040F4804040F400402168A2
:10332000C9694CF6FF72914308432168C861D4E92A
:10333000070108432168096821F0C001084321689A
:103340000860D4E9031008432168896848F2FF3215
:103350009143084321688860D4E905010843216846
:10336000C96821F0FF0108432168C860206800682F
:1033700040F001002168086000202064202084F8CB
:103380003D000020206384F83E0000BF24E70000D9
:10339000A086010080841E0000093D0040420F000D
:1033A00010B586B00446142101A8FDF794FA5E49D1
:1033B000206888422FD100BF002000905B48006841
:1033C00040F00200594908600846006800F0020019
:1033D000009000BF00BFC02001901220029000208A
:1033E0000390032004900420059001A95048FFF7A2
:1033F000D7FD00BF002000904C481030006840F41A
:1034000000104A49103108600846006800F40010B6
:10341000009000BF86E047492068884230D100BF55
:10342000002000904148006840F002003F490860D9
:103430000846006800F00200009000BF00BF4FF493
:10344000406001901220029000200390032004901D
:103450000420059001A93648FFF7A2FD00BF002017
:10346000009032481030006840F480002F4910313D
:1034700008600846006800F48000009000BF51E03A
:103480002D49206888424DD100BF00200090274878
:10349000006840F00400254908600846006800F014
:1034A0000400009000BF00BF00BF0020009008464D
:1034B000006840F0010008600846006800F0010064
:1034C000009000BF00BF481501901220029000201C
:1034D0000390032004900420059001A91748FFF7EA
:1034E0005FFD4FF480700190122002900020039045
:1034F000032004900420059001A91148FFF750FD16
:1035000000BF0020009009481030006840F400001F
:103510000649103108600846006800F40000009079
:1035200000BF00BF06B010BD00540040303802405C
:103530000004024000580040005C004000080240C7
:103540000000024003480068034909780844014923
:103550000860704798000020A000002010B50D48BA
:10356000006840F400700B4908600846006840F4A9
:10357000806008600846006840F48070086003209E
:1035800000F0A6F80F2000F007F800F02BF800205C
:1035900010BD0000003C024070B504460E480078A3
:1035A0004FF47A71B1FBF0F00C490968B1FBF0F50A
:1035B000284600F037FE08B1012070BD102C07D25C
:1035C00000222146501E00F045F80548046001E045
:1035D0000120F2E70020F0E7A0000020A400002076
:1035E0009C00002008B500BF002000900E48006835
:1035F00040F480400C4908600846006800F48040B0
:10360000009000BF00BF00BF00200090081F0068AE
:1036100040F08050091F08600846006800F08050A4
:10362000009000BF00BF08BD443802400146084674
:1036300000280DDB00BF00BF00F01F0301229A40ED
:1036400043099B0003F1E023C3F8002100BF00BF42
:1036500000BF70472DE9F05F80460D4616460027F3
:1036600004F0BAFE074639462A46334601F0070001
:10367000C0F1070ABAF1040F02D94FF0040A01E0C1
:10368000C0F1070AD14600F1040ABAF1070F02D2CD
:103690004FF0000A01E0A0F1030AD4464FF0010AFE
:1036A0000AFA09FAAAF1010A0AEA020A0AFA0CFA63
:1036B0004FF0010B0BFA0CFBABF1010B0BEA030B08
:1036C0004AEA0B042146404604F08EFEBDE8F09F16
:1036D00000BF00F00702064B19684FF6FF031940C0
:1036E000044B0B4343EA0221014B196000BF7047B2
:1036F0000CED00E00000FA0570B504460D460CB96B
:10370000012070BD5848006800F00700A84209D2A7
:1037100055490D700846006800F00700A84201D026
:103720000120EEE7207800F0020002281DD1207869
:1037300000F00400042805D14C48006840F4E05033
:103740004A490860207800F00800082805D1474859
:10375000006840F46040454908604448006820F033
:10376000F000A168084341490860207800F001009A
:10377000A8B36068012807D13C4808380068C0F346
:103780004040B8B90120BCE76068022802D06068F8
:10379000032807D1354808380068C0F3406048B9AD
:1037A0000120AEE7314808380068C0F3400008B98E
:1037B0000120A6E72D48006820F003006168084357
:1037C0002A490860FFF7FEFC064609E0FFF7FAFC0D
:1037D000801B41F28831884202D9032091E707E03B
:1037E0002248006800F00C006168B0EB810FEDD159
:1037F0001D48006800F00700A84209D91A490D7059
:103800000846006800F00700A84201D0012078E7D0
:10381000207800F00400042807D11448006820F440
:10382000E050E168084311490860207800F0080082
:10383000082808D10D48006820F46040216940EA5A
:10384000C1000A49086000F03FF808490968C1F35F
:103850000311074A515CC8400649086006480068E1
:10386000FFF79AFE00204CE7003C02400838024077
:103870005EDE0008A40000209C00002001480068D3
:1038800070470000A400002000B5FFF7F7FF0449CF
:103890000968C1F38221034A515CC84000BD0000A1
:1038A000083802406EDE000800B5FFF7E7FF044964
:1038B0000968C1F34231034A515CC84000BD0000B1
:1038C000083802406EDE00082DE9F047002400258C
:1038D0000026A1462548006800F00C0020B104280D
:1038E00005D008283AD105E0DFF8849039E0DFF808
:1038F000849036E01D48001F006800F03F041B481C
:10390000001F006800F4800078B11A481749091FA9
:103910000968C1F38811A0FB01700146224600230B
:103920003846FCF7D9FC05460EE011480F49091F3F
:103930000968C1F38811A0FB0170014622460023EB
:103940003846FCF7C9FC05460848001F0068C0F36C
:103950000140401C4600B5FBF6F902E0DFF810908C
:1039600000BF00BF4846BDE8F087000008380240AD
:103970000024F40000C0A800F8B504460CB90120EA
:10398000F8BD207800F00100002874D0F9480068E4
:1039900000F00C0004280DD0F648006800F00C0080
:1039A000082813D1F348001F006800F48000B0F528
:1039B000800F0BD1EF4808380068C0F34040002862
:1039C00059D06068002856D10120D9E700BF60684F
:1039D000B0F5803F08D1E7480838006840F48030EF
:1039E000E449083908601EE06068B0F5A02F0DD1E9
:1039F000E0480838006840F48020DE490839086053
:103A00000846006840F4803008600CE0D948083867
:103A1000006820F48030D7490839086008460068FB
:103A200020F48020086000BF606890B1FFF7CAFBF7
:103A3000054606E0FFF7C6FB401B642801D90320BA
:103A40009EE7CC4808380068C0F340400028F1D019
:103A500011E0FFF7B7FB054606E0FFF7B3FB401B9D
:103A6000642801D903208BE7C24808380068C0F3F6
:103A700040400028F1D1207800F0020002285FD1F8
:103A8000BC48006800F00C0058B1BA48006800F06B
:103A90000C0008281CD1B748001F006800F4800003
:103AA000B0B9B44808380068C0F3400020B1E068FD
:103AB000012801D0012063E7AE480838006820F0F3
:103AC000F800216940EAC100AA490839086037E0D6
:103AD000E06800B30120A8490860FFF773FB0546C2
:103AE00006E0FFF76FFB401B022801D9032047E7E0
:103AF000A04808380068C0F340000028F1D09D4875
:103B00000838006820F0F800216940EAC1009949AE
:103B10000839086014E0002097490860FFF752FB5D
:103B2000054606E0FFF74EFB401B022801D90320A3
:103B300026E7904808380068C0F340000028F1D11B
:103B4000207800F0080008282CD16069A8B1012075
:103B50008A490860FFF736FB054606E0FFF732FBAF
:103B6000401B022801D903200AE782486C30006814
:103B7000C0F340000028F1D014E000207F49086025
:103B8000FFF720FB054606E0FFF71CFB401B022861
:103B900001D90320F4E677486C300068C0F3400098
:103BA0000028F1D1207800F00400042870D100270B
:103BB00070483830006800F0805090B900BF002095
:103BC00000906C483830006840F0805069493831C6
:103BD00008600846006800F08050009000BF00BFF9
:103BE00001276748006800F48070B0B96448006835
:103BF00040F4807062490860FFF7E4FA054606E089
:103C0000FFF7E0FA401B022801D90320B8E65C4820
:103C1000006800F480700028F2D000BFA06801287E
:103C200008D154486830006840F0010051496831BB
:103C300008601DE0A06805280DD14E486830006876
:103C400040F004004B49683108600846006840F0C5
:103C5000010008600CE047486830006820F001006F
:103C60004449683108600846006820F00400086094
:103C700000BFA068A8B1FFF7A5FA054609E0FFF765
:103C8000A1FA401B41F28831884202D9032077E62D
:103C900026E0384868300068C0F340000028EED0C5
:103CA00013E0FFF78FFA054608E0FFF78BFA401B99
:103CB00041F28831884201D9032061E62D486830FD
:103CC0000068C0F340000028EFD1012F07D1294838
:103CD0003830006820F0805026493831086000BF35
:103CE000A069002845D02348006800F00C0008288F
:103CF0005DD0A069022845D100201F490866FFF762
:103D000061FA054606E0FFF75DFA401B022801D97B
:103D1000032035E6174808380068C0F340600028E3
:103D2000F1D1D4E907010843616A40EA8111012217
:103D3000A06AC2EB500041EA00412C20005D41EA3C
:103D400000600C49091F086001200B490866FFF755
:103D500039FA054606E0FFF735FA401B022801D97B
:103D600003200DE6034808380068C0F340600028CF
:103D7000F1D049E00838024000004742800E474237
:103D800000700040002021490866FFF71BFA054635
:103D900006E0FFF717FA401B022801D90320EFE5E0
:103DA0001B480068C0F340600028F2D12CE0A069F5
:103DB000012800D1E4E51648001D0668A069012825
:103DC00020D006F48001E06981421BD106F03F015A
:103DD000206A814216D147F6C0703040616AB0EB6C
:103DE000811F0FD106F440310122A06AC2EB5000BE
:103DF000B1EB004F06D106F070612C20005DB1EBF5
:103E0000006F01D00120BBE50020B9E5000047426A
:103E10000038024010B504460CB9012010BD606A9C
:103E200038B96068B0F5827F00D105E00021E1611A
:103E300002E00021216161610021A16294F851003A
:103E400028B9002084F85000204600F047F80220EE
:103E500084F851002068006820F040002168086064
:103E6000A08800F48270218901F404410843A189EB
:103E700001F400610843217C01F002010843217D27
:103E800001F001010843218B01F400710843217FF7
:103E900001F0380108432021095D01F08001084349
:103EA000218D01F400510843216808600421A069B4
:103EB00001EA104094F8241001F010010843216831
:103EC00048602068C06920F400602168C861002053
:103ED0006065012084F8510000209FE710B586B08E
:103EE0000446142101A8FCF7F6FC374920688842F3
:103EF00030D100BF002000903448006840F480506A
:103F0000324908600846006800F48050009000BF05
:103F100000BF00BF002000902C481438006840F01B
:103F200001002A49143908600846006800F00100C1
:103F3000009000BF00BFE02001900220029000200E
:103F40000390032004900520059001A92048FFF765
:103F500027F836E01F492068884232D100BF002090
:103F600000901A48001F006840F400401749091FDC
:103F700008600846006800F40040009000BF00BFE1
:103F800000BF0020009011481438006840F0040081
:103F90000E49143908600846006800F004000090DB
:103FA00000BF00BF4FF4E0500190022002900020BB
:103FB0000390032004900620059001A90648FEF70F
:103FC000EFFF06B010BD0000003001404438024051
:103FD00000000240003C0040000802402DE9FE4F76
:103FE00004460F4690461D460C9E01200190FFF7A7
:103FF000E9F8814694F851B060680290AA46BBF196
:10400000010F0BD00298B0F5827F04D1A06810B9DF
:10401000BBF1040F02D00220BDE8FE8F1FB1B8F142
:10402000000F00D00DB90120F6E700BF94F8500052
:10403000012801D10220EFE7012084F8500000BFE1
:1040400094F85100042802D0052084F85100002083
:104050006065C4F83880E587A5872763E586A5866F
:10406000206460642068006800F04000402805D0AB
:104070002068006840F0400021680860E068B0F502
:10408000006F52D1606810B1BAF1010F09D1206BF5
:1040900000882168C860206B801C2063E08E401E71
:1040A000E0863BE02068806800F00200022810D122
:1040B000E08E70B1019801280BD1206B0088216837
:1040C000C860206B801C2063E08E401EE0860020CC
:1040D00001902068806800F0010068B1E08F58B15D
:1040E0002068C068A16B0880A06B801CA063E08F73
:1040F000401EE08701200190FFF764F8A0EB090063
:10410000B0420BD3701C48B1012084F8510000BFAD
:10411000002084F8500000BF03207DE7E08E0028D7
:10412000C0D1E08F0028BDD152E0606810B1BAF173
:10413000010F09D1206B007821680873206B401CA7
:104140002063E08E401EE0863CE02068806800F03E
:104150000200022810D1E08E70B1019801280BD125
:10416000206B007821680873206B401C2063E08E70
:10417000401EE086002001902068806800F0010069
:1041800068B1E08F58B12068C068A16B0870A06B5F
:10419000401CA063E08F401EE08701200190FFF7E4
:1041A00011F8A0EB0900B04201D3701C00B94EB960
:1041B000012084F8510000BF002084F8500000BFA7
:1041C000032029E7E08E0028BFD1E08F0028BCD172
:1041D0004A463146204602F007FC40B12020606587
:1041E00000BF002084F8500000BF012014E7A06841
:1041F00050B900BF002000902068C068009020687F
:104200008068009000BF00BF012084F8510000BF0B
:10421000002084F8500000BF606D08B10120FBE66B
:104220000020F9E670B504462546681EB0F1807F8F
:1042300001D301200FE0681E4FF0E02148610F21FB
:104240004FF0FF3004F0D0F800204FF0E0218861FB
:1042500007200861002070BD7047704730B50246E6
:104260000B4600BF92F83C00012801D1022030BD6E
:10427000012082F83C0000BF022082F83D00106857
:1042800044681068816824F070041868044310685A
:104290004460184D1068A8421BD01068B0F1804FE0
:1042A00017D0154D1068A84213D0144D1068A842BD
:1042B0000FD0134D1068A8420BD0124D1068A842C1
:1042C00007D0114D1068A84203D0104D1068A842C5
:1042D00005D121F0800158680143106881600120F8
:1042E00082F83D0000BF002082F83C0000BF00BF04
:1042F000BDE700000000014000040040000800404D
:10430000000C004000040140004001400018004043
:1043100010B504460CB9012010BD94F83D0028B931
:10432000002084F83C00204600F026F8022084F8A3
:104330003D00211D206802F041FE012084F8460066
:1043400000BF84F83E0001213F2001554020015567
:104350004120015500BF00BF012084F842004320E6
:104360000155442001554520015500BF012084F826
:104370003D000020D0E7000038B504462068B0F1C9
:10438000804F0FD100BF002000903D48006840F0F2
:1043900001003B4908600846006800F001000090F9
:1043A00000BF6BE03749206888420FD100BF002072
:1043B00000903348006840F0020031490860084628
:1043C000006800F00200009000BF57E02E4920680E
:1043D000884218D100BF002000902948006840F0B2
:1043E0001000274908600846006800F0100000909F
:1043F00000BF00BF002211463620FFF72BF9362000
:10440000FFF714F93AE021492068884218D100BF2B
:10441000002000901A48006840F020001849086009
:104420000846006800F02000009000BF00BF002296
:1044300011463720FFF70EF93720FFF7F7F81DE098
:1044400013492068884219D100BF002000900C4811
:10445000001D006840F400300949091D0860084645
:10446000006800F40030009000BF00BF0022114639
:104470001920FFF7EFF81920FFF7D8F838BD000032
:10448000403802400004004000100040001400408A
:1044900000440140014691F83D00012801D001206F
:1044A0007047022081F83D000868C06840F00100B4
:1044B0000B68D8601A4B086898421BD00868B0F1A6
:1044C000804F17D0174B0868984213D0164B0868D6
:1044D00098420FD0154B086898420BD0144B0868CF
:1044E000984207D0134B0868984203D0124B0868D3
:1044F00098420CD10868806800F00702062A0CD0A8
:104500000868006840F001000B68186005E0086862
:10451000006840F001000B6818600020C0E7000050
:10452000000001400004004000080040000C004072
:1045300000040140004001400018004001460868A6
:10454000C06820F001000A68D06000BF0868006AF7
:1045500041F21112104050B90868006A92101040E0
:1045600028B90868006820F001000A68106000BFE0
:10457000012081F83D00002070472DE9F0410446FC
:104580000D46002700BF94F83C00012802D102200C
:10459000BDE8F081012084F83C0000BF022084F8CF
:1045A0003D002068866826F0770626F47F4620685E
:1045B00086602868502833D00CDC202850D004DCDA
:1045C00000284BD0102851D149E0302849D040284C
:1045D0004CD139E060282DD0702807D0B0F5805F2D
:1045E00003D0B0F5005F41D10DE041E0D5E9021301
:1045F0006A68206802F067FD2068866846F07706E2
:104600002068866034E0D5E902136A68206802F009
:104610005AFD2068806840F480402168886027E067
:10462000EA686968206802F03FFE5021206802F0C5
:1046300055FD1DE0EA686968206802F091FE60217E
:10464000206802F04BFD13E0EA686968206802F018
:104650002BFE4021206802F041FD09E000BF00BFB1
:1046600000BF2968206802F039FD01E0012700BF82
:1046700000BF012084F83D0000BF002084F83C000A
:1046800000BF384684E72DE9F04104460D4614B9D1
:104690000120BDE8F08194F83D0028B9002084F89D
:1046A0003C00204600F053F8022084F83D002068CA
:1046B000806844F20701884321688860211D2068D2
:1046C00002F07CFC2068D0F80880206886692068A9
:1046D000076A286840EA080840F203308643A9695F
:1046E000A86840EA0120064340F60C4086434FF29A
:1046F000F0008643E969E86840EA0120064328693A
:104700000001296A40EA0130064327F0220727F01A
:1047100088076969686840EA011007432068C0F8A3
:1047200008802068866120680762012084F84600BE
:1047300084F83E0001213F200155012084F8420009
:1047400043200155012084F83D000020A1E7704777
:104750002DE9F04304460D4694F83E603F20075D86
:1047600094F84280432010F804906DB9012E02D1D4
:10477000B8F1010F02D00120BDE8F083022084F8D7
:104780003E0084F8420025E0042D0CD1012F02D117
:10479000B9F1010F01D00120EEE702213F200155C0
:1047A0004320015516E0012E07D1012F05D1B8F1A4
:1047B000010F02D1B9F1010F01D00120DCE7022085
:1047C00084F83E0002213F200155022084F8420077
:1047D0004320015515B1042D0CD105E00122002123
:1047E000206802F05FFC10E001220421206802F042
:1047F00059FC0AE001220021206802F053FC01224A
:104800000421206802F04EFC00BF00BF2068006851
:1048100040F00100216808600020ADE770472DE9F5
:10482000F04104460D461646002700BF94F83C00B0
:10483000012802D10220BDE8F081012084F83C006B
:1048400000BF96B9EB68D5E90012206802F040FD80
:104850002068806920F00C002168886120688069E8
:10486000A96808432168886141E0042E13D1EB68F0
:10487000D5E90012206802F087FD2068806920F4E5
:1048800040602168886120688069A96840EA012049
:10489000216888612BE0082E12D1EB68D5E900125F
:1048A000206802F08EFD2068C06920F00C002168AD
:1048B000C8612068C069A96808432168C86116E01A
:1048C0000C2E13D1EB68D5E90012206802F095FD9B
:1048D0002068C06920F440602168C8612068C06910
:1048E000A96840EA01202168C86100E0012700BFF3
:1048F000002084F83C0000BF38469CE710B5044611
:104900000CB9012010BD94F83D0028B9002084F8AE
:104910003C00204600F026F8022084F83D00211DCE
:10492000206802F04BFB012084F8460000BF84F8A9
:104930003E0001213F2001554020015541200155F5
:1049400000BF00BF012084F84200432001554420ED
:1049500001554520015500BF012084F83D0000208D
:10496000D0E7000010B586B00446142101A8FBF77B
:10497000B2FF1F492068884237D100BF0020009055
:104980001C48006840F001001A49086008460068A9
:1049900000F00100009000BF00BF00BF00200090A9
:1049A00014481438006840F01000124914390860A7
:1049B0000846006800F01000009000BF00BF4FF4F0
:1049C00028500190022002900020039004900120C2
:1049D000059001A90848FEF7E3FA002211461920C4
:1049E000FEF738FE1920FEF721FE06B010BD0000CC
:1049F00000000140443802400010024070B50446F7
:104A00002068C5682068066906F00200022819D1EE
:104A100005F00200022815D1401F2168086101201D
:104A200020772068806900F0030018B12046FFF766
:104A3000F5FE05E0204600F0E9F8204600F09DF97B
:104A40000020207706F00400042819D105F00400A6
:104A5000042815D1C043216808610220207720680E
:104A6000806900F4407018B12046FFF7D7FE05E0DA
:104A7000204600F0CBF8204600F07FF90020207798
:104A800006F00800082819D105F00800082815D1FB
:104A9000C04321680861042020772068C06900F0C5
:104AA000030018B12046FFF7B9FE05E0204600F0EC
:104AB000ADF8204600F061F90020207706F01000E4
:104AC000102819D105F01000102815D1C043216815
:104AD0000861082020772068C06900F4407018B190
:104AE0002046FFF79BFE05E0204600F08FF82046A9
:104AF00000F043F90020207706F0010048B105F0EE
:104B0000010030B16FF0010021680861204600F01B
:104B1000BBF906F08000802809D105F080008028CC
:104B200005D1C043216808612046FFF795FB06F0D8
:104B30004000402809D105F04000402805D1C0437D
:104B400021680861204600F0C7F906F020002028FF
:104B500009D105F02000202805D1C0432168086153
:104B60002046FFF77AFB70BD10B586B004461421CD
:104B700001A8FBF7B0FE2068B0F1804F1DD100BF47
:104B8000002000901E48006840F002001C490860A8
:104B90000846006800F00200009000BF00BF082037
:104BA00001900220029000200390049001200590C3
:104BB00001A91448FEF7F4F920E01349206888425F
:104BC0001CD100BF002000900D48006840F002009A
:104BD0000B4908600846006800F00200009000BF22
:104BE00000BF20200190022002900020039004903A
:104BF0000220059001A90348FEF7D2F906B010BDC6
:104C000030380240000402400004004070472DE9A3
:104C1000F04104460D461646002700BF94F83C00BC
:104C2000012802D10220BDE8F081012084F83C0077
:104C300000BF36B1042E1BD0082E31D00C2E5ED111
:104C400045E02946206802F053FA2068806940F068
:104C50000800216888612068806920F004002168CC
:104C6000886120688069296908432168886148E073
:104C70002946206802F074FA2068806940F40060D8
:104C8000216888612068806920F4806021688861DB
:104C900020688069296940EA01202168886130E044
:104CA0002946206802F09AFA2068C06940F008009E
:104CB0002168C8612068C06920F004002168C861CB
:104CC0002068C069296908432168C86119E029463C
:104CD000206802F0BFFA2068C06940F400602168D3
:104CE000C8612068C06920F480602168C8612068BC
:104CF000C069296940EA01202168C86101E00127F3
:104D000000BF00BF00BF002084F83C0000BF384651
:104D100089E710B504460CB9012010BD94F83D0098
:104D200028B9002084F83C00204600F025F8022035
:104D300084F83D00211D206802F040F9012084F82C
:104D4000460000BF84F83E0001213F20015540206D
:104D500001554120015500BF00BF012084F84200E9
:104D600043200155442001554520015500BF012035
:104D700084F83D000020D0E77047704770B50446C6
:104D80000D4615B994F83E000BE0042D02D13F20EA
:104D9000005D06E0082D02D14020005D01E04120C9
:104DA000005D012801D0012070BD1DB9022084F8EA
:104DB0003E000EE0042D03D102213F20015508E002
:104DC000082D03D102214020015502E0022141209B
:104DD000015501222946206802F064F92349206820
:104DE000884203D022492068884201D1012000E096
:104DF000002028B12068406C40F4004021684864DD
:104E00001A49206888421BD02068B0F1804F17D023
:104E100018492068884213D01749206888420FD06B
:104E20001649206888420BD011492068884207D073
:104E300013492068884203D01249206888420CD167
:104E40002068806800F00706062E0CD020680068F5
:104E500040F001002168086005E02068006840F02B
:104E600001002168086000209EE70000000001406A
:104E7000000401400004004000080040000C004015
:104E8000004001400018004010B504460E4884421E
:104E900001D107F089FA0D4884420FD16FF001006B
:104EA0000A49096808610948FFF748FB08488088F3
:104EB0000749C8800020888006F012FB054884421C
:104EC00001D105F037FB10BD90050020D80500206A
:104ED000500A0020200600207047704770470000ED
:104EE0002DE9F84F0446206805682068C6682068E8
:104EF00047694FF00009CA4605F00F09B9F1000FE4
:104F00000AD105F0200038B106F0200020B120467B
:104F100002F058FBBDE8F88FB9F1000F7CD007F024
:104F2000010018B906F49070002875D005F0010052
:104F300030B106F4807018B1606C40F0010060641C
:104F400005F0040030B107F0010018B1606C40F0CA
:104F50000200606405F0020030B107F0010018B1F2
:104F6000606C40F00400606405F0080048B106F091
:104F7000200010B907F0010018B1606C40F0080083
:104F80006064606C002846D005F0200028B106F06F
:104F9000200010B1204602F015FB20684069C0F3E4
:104FA000801A606C00F0080010B9BAF1000F2DD023
:104FB000204602F0AEFA2068406900F04000402828
:104FC00020D100BF00BF2168143151E8001F21F03B
:104FD00040002168143141E80002002AF3D100BFEB
:104FE000E06B50B17748E16B0865E06BFDF7D0FDF1
:104FF00088B1E06B016D88470DE02046FFF76EFF3A
:1050000009E009E02046FFF769FF04E02046FFF7CA
:1050100065FF002060647DE7206B012878D105F0F2
:105020001000002874D006F010000028FAD000BF4D
:105030000020009020680068009020684068009080
:1050400000BF00BF2068406900F04000402860D1E8
:10505000E06B006840681FFA80F8B8F1000F56D086
:10506000A08D404553DDA4F82E80E06BC069B0F5FB
:10507000807F43D000BF00BF21680C3151E8001F82
:1050800021F4807021680C3141E80002002AF3D13C
:1050900000BF00BF00BF2168143151E8001F21F09C
:1050A00001002168143141E80002002AF3D100BF59
:1050B00000BF00BF2168143151E8001F21F04000FB
:1050C0002168143141E80002002AF3D100BF2020FA
:1050D00084F842000020206300BF00BF21680C312B
:1050E00051E8001F21F0100021680C3141E8000256
:1050F000002AF3D100BFE06BFDF7F4FC02206063EF
:10510000A08DE28D801A81B22046FFF7E6FE01E70E
:1051100042E0A08DE18D401A1FFA80F8E08DD0B3F7
:10512000B8F1000F37D000BF00BF21680C3151E843
:10513000001F21F4907021680C3141E80002002A20
:10514000F3D100BF00BF00BF2168143151E8001F38
:1051500021F001002168143141E80002002AF3D156
:1051600000BF202084F842000020206300BF00BF61
:1051700021680C3151E8001F21F0100021680C312A
:1051800041E80002002AF3D100BF022060634146DB
:105190002046FFF7A2FEBDE605F0800030B106F024
:1051A000800018B1204602F0C1FBB3E605F04000D4
:1051B00030B106F0400018B1204602F0E0F9A9E64F
:1051C00000BFA7E64974000810B504460CB90120D9
:1051D00010BDA06900B100E000BF94F8410028B9FB
:1051E000002084F84000204600F02AF8242084F8AB
:1051F00041002068C06820F400502168C860204643
:1052000002F05EFA2068006920F49040216808618D
:105210002068406920F02A00216848612068C06841
:1052200040F400502168C86000206064202084F8A9
:10523000410084F842000020606300BFC8E700001E
:1052400010B586B00446142101A8FBF744FBD949E8
:105250002068884256D100BF00200090D6480068E0
:1052600040F40020D44908600846006800F400209B
:10527000009000BF00BF00BF00200090CE48103853
:10528000006840F00100CC49103908600846006809
:1052900000F00100009000BF00BF03200190022039
:1052A000029000200390032004900820059001A99B
:1052B000C248FDF775FEC248C24908604FF0006061
:1052C00048604021BF4881600021C1604FF4806187
:1052D0000161002141618161C16101624162FDF7AB
:1052E0008BFD08B1FDF728F900BFB648A0638463C1
:1052F00000BF002211463420FEF7ACF93420FEF73F
:1053000095F954E1B0492068884259D100BF002086
:105310000090A948001D006840F01000A649091D32
:1053200008600846006800F01000009000BF00BF51
:1053300000BF00200090A0481038006840F0010035
:105340009D49103908600846006800F0010000908F
:1053500000BF00BF4FF4C060019002200290002007
:105360000390032004900720059001A99348FDF7BE
:1053700017FE9648964908604FF00060486040214B
:10538000934881600021C1604FF480610161002178
:1053900041618161C16101624162FDF72DFD08B18A
:1053A000FDF7CAF800BF8A48A063846300BF0022EB
:1053B00011462520FEF74EF92520FEF737F9F6E0D5
:1053C00084492068884257D100BF002000907A4865
:1053D000006840F40030784908600846006800F42E
:1053E0000030009000BF00BF00BF00200090724856
:1053F0001038006840F008006F491039086008460E
:10540000006800F00800009000BF00BF602001901D
:1054100002200290002003900320049007200590B2
:1054200001A96D48FDF7BCFD654830306B49086047
:105430004FF0006048604021684881600021C160F1
:105440004FF480610161002141618161C1610162AC
:105450004162FDF7D1FC08B1FDF76EF800BF5F486F
:10546000A063846300BF002211462620FEF7F2F8F5
:105470002620FEF7DBF89AE059492068884258D187
:1054800000BF002000904C48006840F480204A494A
:1054900008600846006800F48020009000BF00BF4C
:1054A00000BF0020009044481038006840F0080019
:1054B0004149103908600846006800F00800009073
:1054C00000BF00BF4FF44070019002200290002006
:1054D0000390032004900720059001A93E48FDF7A2
:1054E0005FFD374818383F4908604FF0006048605A
:1054F00040213C4881600021C1604FF4806101611E
:10550000002141618161C16101624162FDF774FC6A
:1055100008B1FDF711F800BF3248A063846300BFF3
:10552000002211462720FEF795F82720FEF77EF887
:105530003DE02D492068884239D100BF002000900D
:105540001D48001D006840F020001B49091D08602F
:105550000846006800F02000009000BF00BF00BFB8
:105560000020009014481038006840F004001249F0
:10557000103908600846006800F00400009000BF81
:1055800000BFC02001900220029000200390032061
:1055900004900820059001A91448FDF701FD0022A0
:1055A00011464720FEF756F84720FEF73FF806B0B1
:1055B00010BD0000004C0040403802400000024096
:1055C00070600240D007002000100140B864024023
:1055D0003008002000440040000C024090080020E9
:1055E00000480040F008002000140140000802407C
:1055F00070B504460D46164694F8420020280BD19B
:1056000005B10EB9012070BD002020633246294645
:10561000204602F06BF9F6E70220F4E710B50446E5
:105620000E492068884201D105F0C0FF0C4920686E
:10563000884206D1012210210A48FDF7BDFD06F07F
:10564000EFFE09492068884201D106F017FF07499B
:105650002068884201D106F055FF10BD00100140BE
:1056600000440040000C0240004C00400014014087
:105670002DE9F84F04460E46174699464FF0000AAA
:1056800094F84100202850D106B117B90120BDE897
:10569000F88F00206064212084F84100FDF792FD1E
:1056A0008246A784E784A068B0F5805F04D12069B2
:1056B00010B90025B04602E035464FF000081EE064
:1056C0005346002280212046CDF8009002F05EF97A
:1056D00020B1202084F841000320D8E745B9B8F86C
:1056E0000000C0F308002168486008F1020803E0E8
:1056F0002878216848606D1CE08C401EE084E08CB6
:105700000028DDD15346002240212046CDF80090EC
:1057100002F03CF920B1202084F841000320B6E7D4
:10572000202084F841000020B1E70220AFE700000C
:10573000F7B50446154694F84100202836D1019863
:1057400000B10DB90120FEBD01982062A584E58459
:1057500000206064212084F841001548A16BC863D3
:105760001448A16B08641448A16BC8640020A16BA5
:10577000086501AE23681A1D31682B46A06BFDF742
:10578000B1FB6FF040002168086000BF00BF2168D6
:10579000143151E8001F41F080002168143141E8C4
:1057A0000002002AF3D100BF0020CCE70220CAE7A4
:1057B000AD740008057500085D74000810B5044656
:1057C00004492068884204D1012210210248FDF7D3
:1057D000F3FC10BD00440040000C0240704700BFC5
:1057E000FEE700001FB5002000900190029003909A
:1057F0002848294908604FF4803048600021264835
:105800008160012101610021017680F820104FF0B4
:105810008051C1624FF0407181620021C16004215A
:10582000C161012180F830104161FCF7CFFF08B160
:10583000FCF782FE022000900120019000200290DF
:1058400069461548FCF7F8FE08B1FCF775FE042020
:1058500000900220019069460F48FCF7EDFE08B168
:10586000FCF76AFE0C2000900320019069460A486C
:10587000FCF7E2FE08B1FCF75FFE0D20009004206B
:10588000019069460448FCF7D7FE08B1FCF754FEC6
:105890001FBD0000002001405402002008B500BFD9
:1058A000002000902248006840F4800020490860F1
:1058B0000846006800F48000009000BF00BF00BFF1
:1058C000002000900846006840F400100860084678
:1058D000006800F40010009000BF00BF00221146D5
:1058E0000E20FDF7B7FE0E20FDF7A0FE00221146A8
:1058F0000F20FDF7AFFE0F20FDF798FE00221146A6
:105900001120FDF7A7FE1120FDF790FE00221146A1
:105910003820FDF79FFE3820FDF788FE0022114653
:105920004620FDF797FE4620FDF780FE08BD0000EB
:105930003038024000B587B0142102A8FAF7CBFF37
:1059400000BF002001907048006840F010006E49D0
:1059500008600846006800F01000019000BF00BF1A
:1059600000BF002001900846006840F00400086075
:105970000846006800F00400019000BF00BF00BFAF
:10598000002001900846006840F08000086008464A
:10599000006800F08000019000BF00BF00BF002041
:1059A00001900846006840F0010008600846006861
:1059B00000F00100019000BF00BF00BF0020019077
:1059C0000846006840F0020008600846006800F0E1
:1059D0000200019000BF00BF00BF002001900846F8
:1059E000006840F0080008600846006800F0080001
:1059F000019000BF00BF00224CF20D014348FDF7AB
:105A0000DBFB012232214148FDF7D6FB0122302188
:105A10003F48FDF7D1FB012211463E48FDF7CCFB84
:105A200001224FF4C0513C48FDF7C6FB002242F270
:105A300092013948FDF7C0FB0122D1033748FDF739
:105A4000BBFB00224FF404713248FDF7B5FB4CF26A
:105A50003F0002900120039000200490059002A9CD
:105A60002A48FDF79DFA42F20300029000200390BD
:105A7000049002A92648FDF793FA302002900120F5
:105A8000039000200490059002A92148FDF788FAB0
:105A900040F2112002900120039000200490059014
:105AA00002A91C48FDF77CFA43F6920002900120FF
:105AB000039000200490059002A91748FDF770FAA2
:105AC00044F20C00029000200390049002A91248B6
:105AD000FDF766FA4FF40040029001200390002089
:105AE0000490059002A90D48FDF75AFA0120029092
:105AF0004FF4881003900020049002A90648FDF797
:105B00004FFA07B000BD00003038024000100240DC
:105B10000008024000040240000C02400000024065
:105B200010B50B480B4908600B4848600021094834
:105B30008160C1604FF48041016100214161816158
:105B4000C1610162FDF744FB08B1FCF7F5FC10BD33
:105B5000005400400C030020A086010010B50B4843
:105B60000B4908600B484860002109488160C1600A
:105B70004FF480410161002141618161C161016295
:105B8000FDF726FB08B1FCF7D7FC10BD005800401C
:105B900060030020A086010010B50B480B49086087
:105BA0000B484860002109488160C1604FF4804182
:105BB0000161002141618161C1610162FDF708FB62
:105BC00008B1FCF7B9FC10BD005C0040B403002034
:105BD000A086010010B50E480E4908604FF482708F
:105BE000486000210B488160C160016141614FF450
:105BF000007181611821C1610021016241628162ED
:105C00000A21C162FEF706F908B1FCF795FC10BD48
:105C1000003001400804002010B50E480E4908600D
:105C20004FF48270486000210B488160C1600161BF
:105C300041614FF4802181610021C16101624162B3
:105C400081620A21C162FEF7E5F808B1FCF774FC35
:105C500010BD0000003C00406004002010B50A4860
:105C60000A4908602F20486000210848816040F6FA
:105C70001F21C160002101618161FEF749FB08B16C
:105C8000FCF75AFC10BD0000004401402006002033
:105C900000B58FB0242106A8FAF71DFE002004905D
:105CA00005900090019002900390224822490860DC
:105CB000002048600021204881604FF6FF71C160DC
:105CC0000021016141618161FEF718FE08B1FCF716
:105CD00033FC03200690002007900120089000204C
:105CE00009900A900B9001200C9000200D900E90CE
:105CF00006A91148FEF7C7FC08B1FCF71DFC0020FF
:105D00000490059004A90C48FEF7A8FA08B1FCF726
:105D100013FC0020009001200190002002900390CD
:105D2000082269460448FEF77AFD08B1FCF704FC36
:105D30000FB000BD00000140B804002000B58DB0D8
:105D4000002009900A900B900C90079008901C215D
:105D50006846FAF7C0FD4FF080401F4908600920EF
:105D6000486000211C4881604FF2FF21C160002182
:105D700001618161FEF7CCFA08B1FCF7DDFB4FF45D
:105D80008050099009A91448FEF7F7FB08B1FCF709
:105D9000D3FB1148FEF7BDFF08B1FCF7CDFB002097
:105DA0000790089007A90C48FEF758FA08B1FCF7CD
:105DB000C3FB602000900020019002900490042218
:105DC00069460548FEF723FF08B1FCF7B5FB02481A
:105DD000FEF7CAFE0DB000BD0005002000B58DB075
:105DE000002009900A900B900C90079008901C21BD
:105DF0006846FAF770FD1F481F4908600020486098
:105E000000211D4881608621C160002101618161FE
:105E1000FEF77EFA08B1FCF78FFB4FF48050099033
:105E200009A91548FEF7A9FB08B1FCF785FB124844
:105E3000FEF76FFF08B1FCF77FFB0020079008908A
:105E400007A90D48FEF70AFA08B1FCF775FB6020B8
:105E500000900020019002900490042269460648B8
:105E6000FEF7D5FE08B1FCF767FB0348FEF77CFEA2
:105E70000DB000BD00040040480500201CB5002006
:105E8000009001900E480F490860172048600021DB
:105E90000C48816040F61F21C16000218161FEF73E
:105EA00037FA08B1FCF748FB0020009001906946E2
:105EB0000448FEF7D3F908B1FCF73EFB1CBD000017
:105EC00000100040900500201CB5002000900190BB
:105ED0000E480F4908601720486000210C48816077
:105EE00040F61F21C16000218161FEF711FA08B15F
:105EF000FCF722FB00200090019069460448FEF761
:105F0000ADF908B1FCF718FB1CBD000000140040FF
:105F1000D805002010B50B480B4908604FF4E1305C
:105F20004860002108488160C16001610C21416125
:105F300000218161C161FFF747F908B1FCF7FCFA64
:105F400010BD0000004C00406806002010B50B4852
:105F50000B4908604FF4E130486000210848816037
:105F6000C16001610C21416100218161C161FFF7C4
:105F70002BF908B1FCF7E0FA10BD00000010014059
:105F8000B006002010B50D480D4908604FF496602A
:105F900048604FF480510A4881600021C1604FF48D
:105FA000C06101610C21416100218161C161FFF784
:105FB0000BF908B1FCF7C0FA10BD00000044004026
:105FC000F806002010B50B480B4908604FF4E1308B
:105FD0004860002108488160C16001610C21416175
:105FE00000218161C161FFF7EFF808B1FCF7A4FA65
:105FF00010BD0000004800404007002010B50B48CD
:106000000B4908604FF4E130486000210848816086
:10601000C16001610C21416100218161C161FFF713
:10602000D3F808B1FCF788FA10BD00000014014055
:106030008807002000BFFEE730B502464FF6FF702C
:1060400012B10446A14200D130BD11E012F8014B5B
:10605000604000230AE000F0010424B140104AF23D
:106060000104604000E040105C1CE3B2082BF2DB4E
:106070000C00A1F10105A9B2E8D100BFE4E700BF1F
:10608000FEE7000030B501287BD1CB1E152B77D25F
:10609000DFE803F00B10151A1F7676762432767639
:1060A0007676404E5C61666C71004FF47A63BC4C4E
:1060B000238065E04FF4FA53B94C238060E042F648
:1060C000E063B74C23805BE04FF47A53B44C2380F9
:1060D00056E044F62063B24C238051E05AB1B14BF4
:1060E00093ED000AF7EE000A30EE200A83ED000A75
:1060F0000123AD4C237043E05AB1AA4B93ED000A43
:10610000F7EE000A30EE600A83ED000A0123A64C88
:10611000237035E05AB1A54B93ED000AF7EE000A63
:1061200030EE200A83ED000A01239F4C237027E004
:106130005AB19E4B93ED000AF7EE000A30EE600A6A
:1061400083ED000A0123984C237019E04FF47A6321
:10615000934C638014E04FF4FA53914C63800FE04A
:1061600042F6E0638E4C63800AE00AE04FF47A5313
:106170008B4C638004E044F62063894C638000BF4D
:1061800000BF022819D10B2907D149F21873884C96
:10619000246863629823874C236002290DD132B1B1
:1061A000854B1B7843F02003834C237005E0824B22
:1061B0001B7803F0DF03804C237003280FD10429E0
:1061C0000DD132B17C4B1B7843F080037A4C2370A5
:1061D00005E0794B1B7803F07F03774C237004288C
:1061E00077D1A1F11003062B27D2DFE803F00327B4
:1061F0004B739AC1714B1B8B714C24881B1B6F4CCA
:106200002383704B1B88248B1B1B1BB26C4C23807D
:106210002346B3F90030002B04DB23461B88604C77
:1062200063810AE0664CB4F9004063424FF6FF74A4
:10623000E41A641C5A4D6C8100BFA3E05F4B1B8ABB
:10624000614C24881B1B5D4C2382604B1B88248A75
:106250001B1B1BB25C4C23802346B3F90030002B80
:1062600004DB23461B884E4C63820AE0564CB4F98B
:10627000004063424FF6FF74E41A641C484D6C8280
:1062800000BF7FE04D4B5B894F4C64881B1B4B4C20
:1062900063814E4B9B88248A2344484C64891B1B92
:1062A0001BB2494C63802346B3F90230002B04DB58
:1062B00023465B883A4CA3820AE0434CB4F902407F
:1062C00063424FF6FF74E41A641C354DAC8200BF84
:1062D00058E058E0394B9B893B4CA4881B1B374C3A
:1062E000A3813A4B1B89248A2344344CA4891B1B69
:1062F0001BB2354CA3802346B3F90430002B04DBDA
:1063000023469B88264CE3820AE02F4CB4F90440D4
:1063100063424FF6FF74E41A641C214DEC8200BF07
:1063200030E0264BDB89284CE4881B1B234CE3819F
:10633000264B9B89248A2344204CE4891B1B1BB2D7
:10634000214CE3802346B3F90630002B04DB2346BF
:10635000DB88134C23830AE01B4CB4F906406342EC
:106360004FF6FF74E41A641C0D4D2C8300BF09E046
:10637000052304E000240A4D25F813405B1C0D2B77
:10638000F8DB00BF00BF052803D1022901D1104B63
:106390001A60062803D10123014CA4F86C3030BDEB
:1063A000E6000020140000206000002018000020FB
:1063B000B804002050000020080B0020140B00201F
:1063C0002C0000205C320020340000206C320020C1
:1063D0005400002030B504280DD132B10124064DFF
:1063E0002C600024054D2C6005E00024024D2C603B
:1063F0000124024D2C6030BDFC0100200002002071
:106400007047704770470000F0B505AC70CC06F0DF
:106410000F074FEA261C0CEB8C0C07EB4C07DFF840
:1064200098C08CF8007000F00F074FEA201C0CEBAE
:106430008C0C07EB4C07DFF884C08CF8007001F07F
:106440000F074FEA211C0CEB8C0C07EB4C07DFF815
:1064500070C08CF8007002F00F074FEA221C0CEBA2
:106460008C0C07EB4C07DFF85CC08CF8007003F075
:106470000F074FEA231C0CEB8C0C07EB4C07DFF8E3
:1064800048C08CF8007004F00F074FEA241C0CEB96
:106490008C0C07EB4C07DFF834C08CF8007005F06B
:1064A0000F074FEA251C0CEB8C0C07EB4C07DFF8B1
:1064B00020C08CF80070F0BDF8010020F20100202F
:1064C000F3010020F4010020F5010020F601002076
:1064D000F701002010B504461B48048001201B4929
:1064E00008703CB91A480078401EC2B263210020EF
:1064F000FBF724FF012C07D115480078401EC2B2DB
:1065000063210120FBF71AFF022C07D11048007805
:10651000401EC2B263210220FBF710FF032C07D1FB
:106520000B480078401EC2B263210320FBF706FF30
:10653000042C07D106480078401EC2B26321042013
:10654000FBF7FCFE10BD0000F0010020140200204B
:10655000F90100207047000070B506460D4614464C
:10656000012E0BD1012D03D104F57A600949088071
:106570000E2D03D104F57A6006494880052E07D117
:10658000012D05D1FF21A1EB4401C8B200F051FB60
:1065900070BD0000E60000207CB505460C4616469E
:1065A000012D6BD1A249304601F09AFFA14880ED40
:1065B000000A092C07D190ED000ABCEEC00A10EECB
:1065C000100A9D4908800A2C25D19A4890ED000AAE
:1065D0009A4880ED000A90ED000AB5EEC00AF1EE8F
:1065E00010FA08DB90ED000ABCEEC00A10EE100AAB
:1065F0009149C8800FE0914991ED000AB1EE400A3F
:10660000BDEEC00A10EE100A4FF6FF71091A491CC0
:10661000894AD18000BF0F2C08D1864890ED000A2E
:10662000BCEEC00A10EE100A83494880102C25D118
:10663000804890ED000A824880ED000A90ED000A43
:10664000B5EEC00AF1EE10FA08DB90ED000ABCEEE0
:10665000C00A10EE100A784908810FE0784991EDE0
:10666000000AB1EE400ABDEEC00A10EE100A4FF665
:10667000FF71091A491C704A118100BF042D69D1AC
:10668000072C08D16A49304601F02AFFBDEEC00A46
:106690006C4880ED000A082C0CD16549304601F0A9
:1066A0001FFFF2EE040A20EE200ABDEEC00A664883
:1066B00080ED000A092C0CD15D49304601F010FF35
:1066C000F2EE040A20EE200ABDEEC00A5E4880ED1C
:1066D000010A0A2C0CD15649304601F001FFF2EEB6
:1066E000040A20EE200ABDEEC00A574880ED020AD7
:1066F0000B2C0CD14E49304601F0F2FEF2EE040AAA
:1067000020EE200ABDEEC00A4F4880ED030A0C2C93
:106710000BD14749304601F0E3FEBDEEC00A4B48BD
:1067200080ED000A0088444988800D2C12D1404930
:10673000304601F0D5FE464880ED000A90ED000A93
:10674000DFED440A20EE200ABCEEC00A10EE100A6B
:1067500039494883062D6AD1092C18D13E48011FBA
:106760000B1F1A1FCDE900103CA13046F9F778FF46
:1067700000200AE038490C3931F820108AB200F1C3
:1067800028012D4B23F81120401C0428F2DB0A2C91
:1067900018D13148011F0B1F1A1FCDE900102FA17E
:1067A0003046F9F75DFF00200AE02B490C3931F83B
:1067B00020108AB200F12C011F4B23F81120401C3D
:1067C0000428F2DB0B2C18D12348011F0B1F1A1FC2
:1067D000CDE9001021A13046F9F742FF00200AE080
:1067E0001D490C3931F820108AB200F13001124BEA
:1067F00023F81120401C0428F2DB0C2C0AD10C4990
:10680000304601F06DFEBCEEC00A10EE100A0A49D7
:10681000A1F868000D2C0AD10549304601F060FE50
:10682000BCEEC00A10EE100A0349A1F86A007CBD54
:10683000EC01002004020020E600002014000020EB
:10684000180000205C3200206C320020080200207A
:106850000C0200200000C8428832002025642E254A
:10686000642E25642E25640070477047704770477A
:106870002DE9FE4F04460D466678A77894F8078008
:106880002079E17840EA0129A079617940EA012A7A
:10689000207A0106607A41EA0041A07A41EA0020AC
:1068A000E17A40EA010B0D2E2AD008DC012E0DD032
:1068B000032E0CD00B2E27D00C2E73D11CE00F2EE4
:1068C0002AD0B12E43D0F72EF7D12BE000BF454B95
:1068D0005B79DFF810C19CF804C043EA0C22414BFD
:1068E000DB78DFF800C19CF802C043EA0C213D4B85
:1068F0005878FFF7BAFF72E00120FFF7B7FF6EE0AC
:106900000020FFF7B3FF6AE0A81F82B23549891C57
:106910000120FFF777FD62E0002211461046FFF7E5
:1069200071FD5CE02F48017AC0792E4A9279DFF838
:10693000B4C0CDE9002002919CF805309CF80420F9
:106940009CF803109CF80200FFF75EFD47E0012F62
:1069500003D14846FFF7BEFD3FE0A8F110000C2828
:1069600039D2DFE800F0060C1319203838333838F4
:10697000262D627A51464846FFF784FB2CE004F14D
:10698000080251464846FFF707FE25E05A465146A1
:106990004846FFF736FD1FE05A4651464846FFF786
:1069A000DBFD19E01AE05A4651464846FFF728FD3C
:1069B00012E0637A227A51464846FFF70BFD0BE05E
:1069C000227A51464846FFF7C5FD05E05146484644
:1069D000FFF74AFF00E000BF00BF00E000BF00BFBC
:1069E000BDE8FE8F1C3200207CB504460E461546DD
:1069F0003346012202212046009500F065F828B1B7
:106A0000606D40F02000606503207CBD1648006882
:106A10001821B0FBF1F01549B0FBF1F04FF47A7199
:106A2000484301906068B0F5827F0DD13346002263
:106A300080212046009500F047F898B1606D40F045
:106A4000200060650320E0E700BF019800B908E07E
:106A50000198401E019020688068C0F3C010002893
:106A6000F3D100BF0020D0E7A400002040420F0077
:106A700070B50024002520E06006040E01222021CC
:106A80001048FCF799FB052003F0DDF940210D4883
:106A9000FCF780FB10B144F0010401E024F0010494
:106AA000052003F0D0F9002220210648FCF784FBE2
:106AB0000A2003F0C8F9681CC5B2082DDCDB2046AB
:106AC00070BD0000000002402DE9F84F04460D465D
:106AD00090461E46DDF82890FCF774FBA0EB0900F9
:106AE000371AFCF76FFB82462C480068C0F3CB30A6
:106AF0007843009045E0701C002842D0FCF762FB10
:106B0000A0EB0A00B84200D2A7BB2068406820F082
:106B1000E000216848606068B0F5827F0DD1A06810
:106B2000B0F5004F03D0A068B0F5806F05D12068A4
:106B3000006820F0400021680860A06AB0F5005F9E
:106B40000DD100BF2068006820F400502168086063
:106B50002068006840F400502168086000BF0120F0
:106B600084F8510000BF002084F8500000BF0320CB
:106B7000BDE8F88FFFE7009800B900270098401E95
:106B80000090206880682840A84201D1012000E0E0
:106B900000204045AFD10020EAE70000A40000201B
:106BA00070B50446002524E0052003F04CF904F0FC
:106BB000800028B1012280210F48FCF7FDFA04E093
:106BC000002280210C48FCF7F7FA012220210A4814
:106BD000FCF7F2FA0A2003F036F96006040E0022F0
:106BE00020210548FCF7E8FA052003F02CF9681C81
:106BF000C5B2082DD8DB70BD000002407047000010
:106C00000549086000BF0449091F096801F04001F7
:106C10000029F8D0704700000414014010B5044664
:106C200003E02078FFF7ECFF641C20780028F8D1FF
:106C300010BD10B50446EE20FFF7E2FF6020FFF71D
:106C4000DFFFE0B2FFF7DCFFFF20FFF7D9FFFC20FA
:106C5000FFF7D6FFFF20FFF7D3FFFF20FFF7D0FF9E
:106C600010BD70B504460D461646EE20FFF7C8FF6E
:106C7000B120FFF7C5FF1020FFF7C2FF200AFFF782
:106C8000BFFFE0B2FFF7BCFF280AFFF7B9FFE8B289
:106C9000FFF7B6FFF0B2FFF7B3FFFF20FFF7B0FF3B
:106CA000FC20FFF7ADFFFF20FFF7AAFFFF20FFF753
:106CB000A7FF70BD10B5012210210748FCF77CFA30
:106CC000012220210448FCF777FA012211460348EB
:106CD000FCF772FA10BD00000008024000040240F8
:106CE00070B505460E461446EE20FFF789FFB12029
:106CF000FFF786FF1020FFF783FF280AFFF780FFCA
:106D0000E8B2FFF77DFF300AFFF77AFFF0B2FFF736
:106D100077FF200EFFF774FFC4F30740FFF770FF03
:106D2000C4F30720FFF76CFFE0B2FFF769FFFF2015
:106D3000FFF766FFFC20FFF763FFFF20FFF760FF10
:106D4000FF20FFF75DFF70BD2DE9FF412DED020B28
:106D500004460D46174698460026EE20FFF750FFE2
:106D6000B120FFF74DFF0720FFF74AFF200AFFF78A
:106D700047FFE0B2FFF744FF280AFFF741FFE8B200
:106D8000FFF73EFF0220FFF73BFF07F00F01B8F1CE
:106D9000000F01D0802200E000221143C8B2FFF7AB
:106DA0002FFF002607E0C6F103011DF80100FFF7E1
:106DB00027FF701CC6B2042EF5DBFF20FFF720FF73
:106DC000FC20FFF71DFFFF20FFF71AFFFF20FFF752
:106DD00017FF06B0BDE8F0812DE9F04105460E46EB
:106DE00014461F46DDF81880EE20FFF709FFB1209A
:106DF000FFF706FF0720FFF703FF280AFFF700FF52
:106E0000E8B2FFF7FDFE300AFFF7FAFEF0B2FFF737
:106E1000F7FE0FB1012100E00021C8B2FFF7F0FE3C
:106E200008F00F0141F08000FFF7EAFE200EFFF7A7
:106E3000E7FEC4F30740FFF7E3FEC4F30720FFF7C4
:106E4000DFFEE0B2FFF7DCFEFF20FFF7D9FEFC20FB
:106E5000FFF7D6FEFF20FFF7D3FEFF20FFF7D0FE9F
:106E6000BDE8F08170B504460D461646EE20FFF7EA
:106E7000C7FEB120FFF7C4FE1020FFF7C1FE200AB5
:106E8000FFF7BEFEE0B2FFF7BBFE280AFFF7B8FE31
:106E9000E8B2FFF7B5FE3046FFF7C0FEFF20FFF770
:106EA000AFFEFC20FFF7ACFEFF20FFF7A9FEFF209E
:106EB000FFF7A6FE70BD10B5FCF744FB10BD000047
:106EC00000B593B0302107A8F9F705FD142102A8F9
:106ED000F9F701FD00BF002001902348006840F051
:106EE0008050214908600846006800F080500190F9
:106EF00000BF00BF00BF002001901C48006840F4A4
:106F000080401A4908600846006800F480400190FB
:106F100000BF00BF012007900004089002200D90E0
:106F200041050E9108210F915A21109102211191D2
:106F30000421129107A8FCF71FFD08B1FBF7FCFA2A
:106F40000F20029002200390002004904FF4805004
:106F5000059000200690022102A8FCF7CDFB08B1A5
:106F6000FBF7EAFA13B000BD403802400070004061
:106F70000348006840F47000014908607047000051
:106F800088ED00E010B50348FDF738FD0248FDF735
:106F900035FD10BDB80400202006002010B50248C1
:106FA000FDF72CFD10BD00009005002010B5024833
:106FB000FDF724FD10BD0000D805002010B50268C3
:106FC0002D4B98420ED0B0F1804F0BD02B4B9842F6
:106FD00008D02B4B984205D02A4B984202D02A4B1E
:106FE000984203D122F070024B681A43224B984218
:106FF00020D0B0F1804F1DD0204B98421AD0204BAA
:10700000984217D01F4B984214D01F4B984211D072
:107010001E4B98420ED01E4B98420BD01D4B9842EF
:1070200008D01D4B984205D01C4B984202D01C4BF7
:10703000984203D122F44072CB681A4322F08003B5
:107040004C6943EA040202608B68C3620B68836286
:10705000094B984202D00C4B984201D10B69036353
:1070600001234361036903F001031BB1036923F0AA
:107070000103036110BD0000000001400004004056
:1070800000080040000C00400004014000400140A6
:10709000004401400048014000180040001C00402E
:1070A0000020004030B501F01F05012404FA05F36B
:1070B000046A9C430462046A01F01F0502FA05F5A4
:1070C0002C43046230BD30B50C46816821F47F4109
:1070D00042EA032525432943816030BD0A46816881
:1070E00021F0700142F007031943816070470000EE
:1070F00030B5026A056A25F00105056243688469B6
:1071000024F0700424F003040D682C4322F00202E2
:107110008D682A43104DA84200D103E00F4DA842CC
:1071200006D100BF22F00802CD682A4322F00402F3
:10713000094DA84202D0094DA84207D123F480731B
:1071400023F400734D692B438D692B4343608461A5
:107150004D684563026230BD0000014000040140FB
:1071600030B5026A056A25F0100505624368846936
:1071700024F4E04424F440740D6844EA052422F029
:1071800020028D6842EA0512124DA84200D103E0A8
:10719000114DA84207D100BF22F08002CD6842EA1B
:1071A000051222F040020B4DA84202D00A4DA8421F
:1071B00009D123F4806323F400634D6943EA850316
:1071C0008D6943EA8503436084614D68856302628B
:1071D00030BD0000000001400004014030B5026AEB
:1071E000056A25F4807505624368C46924F070045B
:1071F00024F003040D682C4322F400728D6842EAE7
:107200000522124DA84200D103E0114DA84207D13A
:1072100000BF22F40062CD6842EA052222F48062B7
:107220000A4DA84202D00A4DA84209D123F4805346
:1072300023F400534D6943EA05138D6943EA0513AE
:107240004360C4614D68C563026230BD0000014007
:107250000004014030B5036A056A25F480550562D3
:107260004468C26922F4E04222F440720D6842EAA6
:10727000052223F400538D6843EA0533084DA842E4
:1072800002D0084DA84204D124F480444D6944EA58
:1072900085144460C2614D680564036230BD00001E
:1072A000000001400004014030B50B461446026A5C
:1072B000056A25F001050562816921F0F00141EAC6
:1072C000041122F00A021A438161026230BD0000FB
:1072D00070B50C461546026A066A26F0010606627B
:1072E0008169184EB04214D0B0F1804F11D0164EC3
:1072F000B0420ED0154EB0420BD0154EB04208D061
:10730000144EB04205D0144EB04202D0134EB042DB
:1073100001D1012600E000261EB121F0030129431E
:1073200001E041F0010121F0F001F02606EA031628
:10733000314322F00A0204F00A06324381610262FC
:1073400070BD000000000140000400400008004043
:10735000000C0040000401400040014000180040C3
:1073600030B50B461446026A056A25F01005056221
:10737000816921F4704141EA043122F0A00242EA1D
:1073800003128161026230BD70B50C461546026A77
:10739000066A26F010060662816921F4407141EA0E
:1073A000052121F470414FF4704606EA033631435B
:1073B00022F0A002A02606EA04163243816102628E
:1073C00070BD70B50C461546026A066A26F48076D2
:1073D0000662C16921F00301294321F0F001F02682
:1073E00006EA0316314322F420624FF4206606EACF
:1073F00004263243C161026270BD70B50C46154669
:10740000026A066A26F480560662C16921F4407158
:1074100041EA052121F470414FF4704606EA033633
:10742000314322F420424FF4204606EA0436324328
:10743000C161026270BD000010B50248FDF750FD49
:1074400010BD00006806002070B50546AC6B00203A
:10745000E085E0842046FDF741FD70BD70B506462D
:107460000025B46B20684069C0F3C01594F8410052
:10747000212805D125B10020E084204600F08FF8B6
:1074800020684069C0F3801594F84200222805D195
:1074900025B10020E085204600F03BF8606C40F00C
:1074A000100060642046FDF719FD70BD70B50546FB
:1074B000AC6B2868006800F48070F8B90020E084A4
:1074C00000BF00BF2168143151E8001F21F0800087
:1074D0002168143141E80002002AF3D100BF00BF47
:1074E00000BF21680C3151E8001F41F040002168C5
:1074F0000C3141E80002002AF3D102E02046FEF7F9
:107500005DF970BD70B50446A56B2846FEF766F9B7
:1075100070BD00BF00BF02680C3252E8002F22F499
:10752000907102680C3242E80013002BF3D100BFC7
:1075300000BF00BF0268143252E8002F22F00101A0
:107540000268143242E80013002BF3D100BF016B34
:1075500001290ED100BF00BF02680C3252E8002F93
:1075600022F0100102680C3242E80013002BF3D124
:1075700000BF202180F8421000210163704710B540
:1075800004462068C06820F040002168C8602020C0
:1075900084F841002046FEF711F9002010BD00BF1D
:1075A00000BF02680C3252E8002F22F0C0010268CE
:1075B0000C3242E80013002BF3D100BF202180F8E9
:1075C00041107047F8B5044694F84200222875D15E
:1075D000A068B0F5805F0CD1206950B90025A66A7B
:1075E00020684068C0F308003080A06A801CA06258
:1075F00015E0A56A0026A068B0F5805F03D0A068FA
:1076000028B9206918B920684068287004E020680B
:10761000406800F07F002870A06A401CA062E08DE6
:10762000401E80B2E085002846D12068C06820F066
:1076300020002168C8602068C06820F4807021683C
:10764000C8602068406920F001002168486120205E
:1076500084F8420000206063206B012826D10020BE
:10766000206300BF00BF21680C3151E8001F21F0EA
:10767000100021680C3141E80002002AF3D100BF5C
:107680002068006800F0100010280AD100BF002018
:10769000009020680068009020684068009000BF5B
:1076A00000BFA18D2046FDF718FC02E02046FDF743
:1076B000B5FF0020F8BD01E00020FBE70220F9E75C
:1076C0002DE9F84F04462068006920F44050E16835
:1076D0000843216808612169A0680843616908437B
:1076E000E169084300902068C06849F20C61884352
:1076F000009908432168C8602068406920F4407000
:10770000A16908432168486176492068884203D00E
:1077100075492068884203D1FCF7C6F8814602E02B
:10772000FCF7B2F88146E069B0F5004F6CD1022059
:107730006168A0FB015003461920A9FB00700146B7
:107740002A463846F8F7C8FD6421B0FBF1F04FEA4D
:10775000001A02206168A0FB01510B461920A9FB09
:1077600000712A463846F8F7B7FD83460220616863
:10777000A0FB015003461920A9FB00712A46384698
:10778000F8F7AAFD6421B0FBF1F000EBC00101EBBA
:107790000010ABEB8000322101EBC0006421B0FB94
:1077A000F1F000F0F8000AEB400A02206168A0FB4B
:1077B000015003461920A9FB007001462A463846AD
:1077C000F8F78AFD834602206168A0FB015003465A
:1077D0001920A9FB00712A463846F8F77DFD64217F
:1077E000B0FBF1F000EBC00101EB0010ABEB80004F
:1077F000322101EBC0006421B0FBF1F000F0070082
:107800005044216888606AE004206168A0FB015050
:1078100003461920A9FB007001462A463846F8F7AE
:107820005BFD824604206168A0FB015003461920DD
:10783000A9FB007001462A463846F8F74DFD642141
:10784000B0FBF1F000EBC00101EB0010AAEB8000EF
:10785000322101EB00106421B0FBF1F000F0F00ADE
:1078600004206168A0FB017003461920A9FB0051A8
:107870003A462846F8F730FD6421B0FBF1F00AEBF8
:10788000001A04206168A0FB01510B461920A9FBD6
:1078900000712A463846F8F71FFD834604206168C8
:1078A000A0FB015003461920A9FB007001462A469F
:1078B0003846F8F711FD6421B0FBF1F000EBC00190
:1078C00001EB0010ABEB8000322101EB00106421D2
:1078D000B0FBF1F000F00F00504421688860BDE873
:1078E000F88F0000001001400014014010B503465D
:1078F00099629A85DA8500205864222083F8420034
:10790000186928B11868C06840F480701C68E0608D
:107910001868406940F001001C6860611868C06820
:1079200040F020001C68E060002010BD014691F886
:107930004100212828D18868B0F5805F0BD1086903
:1079400048B90A6A1088C0F308000B685860086AD2
:10795000801C086205E00B6A581C086218780B68E6
:107960005860C88C401E80B2C88458B90868C06886
:1079700020F080000B68D8600868C06840F04000C4
:107980000B68D860002070470220FCE72DE9F8431F
:1079900004460D4617469846089E31E0701C70B3A9
:1079A000FBF710FCA0EB0800B04200D816B903208A
:1079B000BDE8F8832068C06800F00400F8B1802DAD
:1079C0001ED0402D1CD020680068C0F3C000B0B1AC
:1079D00000BF002000902068006800902068406888
:1079E000009000BF00BF2046FFF793FD08206064B1
:1079F00000BF002084F8400000BF0120D8E7FFE767
:107A0000206800682840A84201D1012000E0002041
:107A1000B842C3D00020CBE710B50248FDF760FAAA
:107A200010BD0000B006002010B50248FDF758FA5E
:107A300010BD0000F806002010B50248FDF750FA0E
:107A400010BD00004007002010B50348FDF748FABC
:107A500004F058FD10BD00008807002010B52DED82
:107A60000C8B82B0FD48008800283BD1FC48007890
:107A700000F0200038B3FB480068401CF94908605A
:107A800008460068052805DA012262210020FAF77D
:107A900055FC04E0002262211046FAF74FFCF14841
:107AA00000680A2807DD0020EE490860EE480078EB
:107AB000401EED490870EC48007801280ADA0320DE
:107AC000E949087006E002F085FC032262210020EB
:107AD000FAF734FCE4480078401EC2B2632100206B
:107AE000FAF72CFCDD480088012873D1DC480078C7
:107AF00000F0200038B3DB480068401CD94908601A
:107B000008460068052805DA012262211046FAF7C6
:107B100015FC04E0002262210120FAF70FFCD14895
:107B200000680A2807DD0020CE490860CE480078AA
:107B3000401ECD490870CC48007801280ADA03209D
:107B4000C949087006E002F045FC022262210120CA
:107B5000FAF7F4FBC4480078401EC2B2632101204A
:107B6000FAF7ECFB00200090C048028800230921AE
:107B70000120FFF731F900200090BC484288002323
:107B80000F210120FFF728F9B9484088B0F57A7F26
:107B900009DD00200090B64842880023182101200A
:107BA000FFF71AF907E0002003460246182100906B
:107BB0000120FFF711F9AE488088B0F57A7F0ADD21
:107BC00000200090AA488288002319210120FFF795
:107BD00003F908E03FE00020034602461921009027
:107BE0000120FFF7F9F800231A46A24890ED000A99
:107BF0000A210120FFF7A8F800231A469E4890EDBD
:107C0000000A10210120FFF79FF898480088B0F57E
:107C10007A6F08DD95480088A0F57A620121084650
:107C2000FFF75EF804E0002201210846FFF758F84C
:107C30008E484088B0F57A6F08DD8C484088A0F502
:107C40007A620E210120FFF74BF804E000220E219A
:107C50000120FFF745F88148008802287DD180483F
:107C6000007800F0200038B37E480068401C7D4951
:107C7000086008460068052805DA01226221022012
:107C8000FAF75CFB04E0002262210220FAF756FBBF
:107C9000744800680A2807DD0020724908607248AD
:107CA0000078401E704908706F48007801280ADA91
:107CB00003206D49087006E002F08CFB022262216D
:107CC0001046FAF73BFB68480078401EC2B26321B9
:107CD0000220FAF733FB6648008BB0F5FA7F1ADD15
:107CE0006349088B05F050FD41EC1A0B9FED630BC7
:107CF00053EC102B05F040FB41EC190B05F04EFA4C
:107D000008EE100A00230322B0EE480A11460220B2
:107D1000FFF71AF807E000231A469FED5A0A0321DD
:107D20000220FFF711F85248008A00EE100AB8EE60
:107D3000400AF2EE040A80EE201AB0EE418A0123D6
:107D40001A46B0EE480A06210220FEF7FDFF484819
:107D500040894749098A401A00E00EE100EE100A06
:107D6000B8EEC00AF2EE040A80EE201AB0EE418AA4
:107D700001231A46B0EE480A07210220FEF7E4FF6D
:107D80003B4880893A49098A401A00EE100AB8EE49
:107D9000C00AF2EE040A80EE201AB0EE418A0123F6
:107DA0001A46B0EE480A08210220FEF7CDFF3048FF
:107DB000C0892F49098A401A00EE100AB8EEC00A9D
:107DC000F2EE040A80EE201AB0EE418A01231A4630
:107DD000B0EE480A09210220FEF7B6FF2A480068E3
:107DE000F8B12348C18A808A01EB004000EE100AF6
:107DF000B8EEC00ADFED250A70EE600A1B488088E5
:107E000000EE100AB8EE400A80EE801AB0EE418A09
:107E100001230222B0EE480A04211046FEF794FF27
:107E200007E0012302229FED170A04211046FEF706
:107E30008BFF1748006880B10C49488B05F0A4FC03
:107E400041EC1D0B9FED130B53EC102B05F094FA36
:107E500041EC1C0B53EC1C2B20E056E0F001002001
:107E6000DA00002010020020F9010020E6000020C6
:107E7000140B002014000020180000200000000057
:107E800000408F4000000000000200208096184B48
:107E9000FC01002000000000000059409FEDFE0B97
:107EA00051EC100B05F068FA41EC1A0BFC48C18A42
:107EB000808A01EB004000EE100AB8EEC00A5FEDC8
:107EC0000D0A70EE600AF748808800EE100AB8EEDE
:107ED000400A80EE801A11EE104A204605F0C2FEDC
:107EE00041EC1B0B53EC1A2B05F09EFC41EC190BDB
:107EF00005F054F908EE100A01230222B0EE480AF8
:107F000005211046FEF720FF07E0012302221FEDA6
:107F1000230A05211046FEF717FFE348007800F01A
:107F2000200028B1012202210846FEF79AFE04E053
:107F3000002202210846FEF794FEDC48007800F09B
:107F4000800028B101220C210220FAF7F7F904E0A1
:107F500000220C210220FAF7F1F9D448007800F051
:107F6000400028B101220D210220FAF7E7F904E0D0
:107F700000220D210220FAF7E1F9CD4800880328FC
:107F80004BD1CA48007800F0200038B3C9480068D7
:107F9000401CC849086008460068052805DA012227
:107FA00062210320FAF7CAF904E0002262210320CB
:107FB000FAF7C4F9BF4800680A2807DD0020BD4968
:107FC0000860BD480078401EBB490870BA48007878
:107FD00001280ADA0320B849087006E002F0FAF92D
:107FE000022262210320FAF7A9F9B3480078401E63
:107FF000C2B263210320FAF7A1F9AB48007800F080
:10800000800028B1012204210320FEF72AFE04E0AB
:10801000002204210320FEF724FEA548008804283E
:108020007ED1A248007800F0200038B3A148006853
:10803000401CA049086008460068052805DA0122AE
:1080400062210420FAF77AF904E000226221042078
:10805000FAF774F9974800680A2807DD0020954967
:10806000086095480078401E93490870924800784F
:1080700001280ADA03209049087006E002F0AAF904
:10808000022262210420FAF759F98B480078401E39
:10809000C2B263210420FAF751F98148008BB0F590
:1080A000FA7F09DD002000907D48028B0023022129
:1080B0000420FEF791FE07E000200346024602215D
:1080C00000900420FEF788FE7548008A00EE100A32
:1080D000B8EE400AF2EE040A80EE201AB0EE418AB1
:1080E00001231A46B0EE480A03210420FEF72CFEB5
:1080F0006B4840896A49098A401A00EE100AB8EEB6
:10810000C00AF2EE040A80EE201AB0EE418A012382
:108110001A46B0EE480A04210846FEF715FE00E0B4
:1081200043E05F4880895E49098A401A00EE100AE0
:10813000B8EEC00AF2EE040A80EE201AB0EE418AD0
:1081400001231A46B0EE480A05210420FEF7FCFD83
:108150005348C0895249098A401A00EE100AB8EE05
:10816000C00AF2EE040A80EE201AB0EE418A012322
:108170001A46B0EE480A06210420FEF7E5FD00206D
:1081800000904848828800230C210420FEF724FE3A
:108190004448408B642190FBF1F4002003462246C2
:1081A0000D2100900420FEF717FE414800880528A5
:1081B0003BD13E48007800F0200038B33D480068CD
:1081C000401C3C49086008460068052805DA012281
:1081D00062210520FAF7B2F804E0002262210520AE
:1081E000FAF7ACF8334800680A2807DD0020314967
:1081F000086031480078401E2F4908702E480078EA
:1082000001280ADA03202C49087006E002F0E2F89F
:10821000022262210520FAF791F827480078401ED3
:10822000C2B263210520FAF789F8214800880628A0
:108230007DD12248007868B31A48B0F85600194931
:10824000B1F85410CDE900101648B0F85230B0F82B
:1082500050201BA11D48F8F7C3F81248B0F85E0083
:108260001049B1F85C10CDE900100E48B0F85A3052
:10827000B0F8582012A11648F8F7B2F80948B0F83B
:1082800066000849B1F86410CDE900100548B0F85F
:1082900062301FE04BE000000000000000004E4094
:1082A000140B0020E6000020080B0020DA0000205C
:1082B000F001002010020020F9010020140200202B
:1082C00025642E25642E25642E256400BC310020F3
:1082D000DC310020B0F86020AFF21C011648F8F73E
:1082E0007FF8164A09210620FEF7BCFD144A0A2130
:1082F0000620FEF7B7FD104A0B210620FEF7B2FD5F
:10830000002000900F48B0F8682000230C210620C0
:10831000FEF762FD002000900A48B0F86A200023B2
:108320000D210620FEF758FD00200749087002B015
:10833000BDEC0C8B10BD0000FC310020BC310020D6
:10834000DC310020E60000201402002000BFFEE720
:108350000246024B23F8121070470000E60000208E
:1083600070B50A46B2F57F4F19D1A0F11001CC17B4
:1083700001EB5474E410174D2C5D0B46DD1703EB35
:108380005575ED10A3EBC5060125B5402C43E5B2AC
:10839000CC1701EB5474E4100E4E355518E0BAB901
:1083A000A0F11001CC1701EB5474E410094D2C5DC1
:1083B0000B46DD1703EB5575ED10A3EBC506012544
:1083C000B540AC43CD1701EB5575ED10014E74551A
:1083D00070BD0000080B002002480068C0F30220B6
:1083E000704700000CED00E010B5002804DB0A0720
:1083F000130E054A135406E00A07140E034A00F050
:108400000F031B1FD45410BD00E400E018ED00E082
:1084100030B540F2FF742DED048BF0EE608A18EE5B
:10842000901A85B0B0EE408A9FED2B9B05468DEDEE
:10843000008B34EA115147D053EC192B51EC180B37
:1084400005F0F2F840D02A4651EC180B05F0B7FCC5
:1084500041EC180B18EE900A8DED008B34EA1050A9
:108460001CD053EC192B51EC180B05F0DDF82BD177
:108470000220F9F784F800F05FF810EE901A18EE79
:10848000900A8DED020B8DED008B61F31E000390C1
:108490009DED020B05B0BDEC048B30BD0220F9F759
:1084A0006EF800F039F810EE901A18EE900A8DED83
:1084B000020B8DED008B61F31E0003909DED020B0E
:1084C00005B0BDEC048B30BD05B0B0EE480AF0EE4F
:1084D000680ABDEC048B30BD000000000000000005
:1084E00000B583B09FED0A0B0A4601468DED000BE7
:1084F0006846F8F705FB9DED000B51EC100B04F0FE
:108500004DFE03B000EE100A00BD000000000000A8
:1085100000000000000000009FED050B10B553ECBB
:10852000102B51EC100B05F07FF941EC100B10BD36
:1085300000000000000000709FED050B10B553EC2B
:10854000102B51EC100B05F06FF941EC100B10BD26
:10855000000000000000001030B504462DED048B33
:1085600081B06A4691ED008B51EC180B01F0ECFEE6
:1085700000989FED239B7E300090002821DC53EC77
:10858000192B51EC180B05F04FF81AD0002140F6CA
:1085900008004FF00000054651EC180B04F0FEFDFA
:1085A00008EE100A40F6080005EA00014FF000004E
:1085B000B5EEC08AF1EE10FA04BF0220F8F7DFFF33
:1085C00017E00098FF280EDB0220F8F7D8FF53ECE5
:1085D000192B51EC180B05F025FA8CBF9FED0A8A78
:1085E0009FED0A8A05E051EC180B04F0D7FD08EE68
:1085F000100A84ED008A01B0BDEC048B30BD000090
:108600000000000000000000000080FF0000807FEC
:1086100010B5044690ED000B0846FFF7F9FE84ED17
:10862000000B10BD30380A2801D20120704700200D
:10863000704700BF7047000010B52DED048B3D481A
:1086400000683D49098808443A490860084640687E
:10865000394949880844374948600846806836499E
:1086600089880844334988600846C0683249C98807
:1086700008443049C86031480068401C2F490860F0
:1086800008460068312852DD2A49086805F07CF860
:1086900041EC190B9FED2A0B53EC102B04F06CFEF0
:1086A00041EC180B05F02CF82749088000202149DF
:1086B0000860486805F068F841EC190B9FED200B45
:1086C00053EC102B04F058FE41EC180B05F018F891
:1086D0001D494880002017494860886805F054F813
:1086E00041EC190B9FED160B53EC102B04F044FEDC
:1086F00041EC180B05F004F81349888000200D495F
:108700008860C86805F040F841EC190B9FED0C0B30
:1087100053EC102B04F030FE41EC180B04F0F0FF8A
:108720000949C88000200349C86004490860BDECBD
:10873000048B10BDFC0200206400002074000020A7
:1087400000000000000049406C00002010B5042229
:1087500002490348FAF7ECF810BD0000640000205D
:108760005402002003200EE0C11E4C4A32F81120B2
:108770004B4B23F811204B4931F81020C11E474BB9
:1087800023F81120401C0D28EEDB454800884349A2
:10879000098888421CD00120434908703F4800885E
:1087A000B0F5704F0BDD3D480088A0F5803000EE3D
:1087B000100AB8EEC00A3D4880ED000A08E03748CC
:1087C000008800EE100AB8EE400A384880ED000A32
:1087D000334840883149498888421CD001203249B9
:1087E00008702E484088B0F5704F0BDD2B4840884C
:1087F000A0F5803000EE100AB8EEC00A2C4880EDDB
:10880000000A08E02548408800EE100AB8EE400A49
:10881000274880ED000A02203CE0214931F8101081
:108820001E4A32F81020914233D001211E4A1170A5
:10883000062817DA194931F81010B1F5704F08DD24
:10884000164931F810100AB2811E1A4B23F8112074
:108850001FE0124931F810100AB2811E154B23F89F
:10886000112016E00D4931F81010B1F5704F08DDF8
:108870000A4931F810100AB2811F0F4B23F811205A
:1088800007E0064931F810100AB2811F0A4B23F89D
:108890001120401C0A28C0DB704700003002002075
:1088A0001C020020E60000206000002014000020D0
:1088B000180000202C0000203400002010B52DED01
:1088C000028BB0EE408A00249FED0D0A28EE000ACC
:1088D000B0EE408A9FED0B0A28EE000ADFED0A0A8F
:1088E00080EE201ABCEEC10A10EE100A84B20748CE
:1088F0000460204600F00CF8BDEC028B10BD0000B7
:108900000000C8420000804500404E45D4000020D1
:1089100070B505464FF6FF7000EA8504C4F30D04F8
:10892000012202212148FAF747FC012211461F4883
:10893000FAF742FC0A2001F086FA002202211B48C5
:10894000FAF73AFC0A2001F07EFA002626E001221E
:1089500011461648FAF730FC04F40040B0F5004F19
:1089600005D1012251021248FAF726FC05E0002247
:108970004FF400710E48FAF71FFC0A2001F063FA69
:10898000002201210948FAF717FC0A2001F05BFADE
:108990004FF6FF7000EA4404701CC6B2102ED6DBFE
:1089A000012202210148FAF707FC70BD00100240C5
:1089B0000004024010B52DED028BB0EE408A002479
:1089C0009FED0C0A28EE000AB0EE408A9FED0A0ADD
:1089D00028EE000ADFED090A80EE201ABCEEC10A7B
:1089E00010EE100A84B2204600F00AF8BDEC028BAB
:1089F00010BD00000000C8420000804500404E4508
:108A000070B505464FF6FF7000EA8504C4F30D0407
:108A1000012210212148FAF7CFFB012208211F482B
:108A2000FAF7CAFB0A2001F00EFA002210211B48B7
:108A3000FAF7C2FB0A2001F006FA002625E001221F
:108A400008211648FAF7B8FB04F40040B0F5004FCF
:108A500005D1012204211148FAF7AEFB04E00022FF
:108A600004210E48FAF7A8FB0A2001F0ECF90022D5
:108A700008210A48FAF7A0FB0A2001F0E4F94FF6B2
:108A8000FF7000EA4404701CC6B2102ED7DB01222E
:108A900010210248FAF790FB70BD00000010024060
:108AA00070B50546002600243D2000F0C1FF284691
:108AB00000F0D8FF0122D1030B48FAF77DFB0FE04D
:108AC0000520FAF759FA00F023F90446102C00D0DB
:108AD00007E03046711CCEB2C82801DDFA2070BD17
:108AE000EEE700BF2046FAE70000024070B50446FA
:108AF000062000F09DFF204600F0B4FF00F008FCC7
:108B000005460122D1030248FAF756FB284670BDFC
:108B10000000024010B5192000F08AFF022001F089
:108B200099F900F0F5FB044600F0F2FB04EB00209D
:108B300084B20122D1030248FAF73EFB204610BD61
:108B40000000024010B5262000F072FF00F0E0FBAC
:108B500004460122D1030248FAF72EFB204610BD3D
:108B60000000024070B50446282000F061FF002597
:108B700005E000F0CDFB04F8010B681CC5B2082D20
:108B8000F7DB0122D1030248FAF716FB70BD0000A3
:108B90000000024010B5012000F04AFF00F0B8FBD1
:108BA00004460122D1030248FAF706FB204610BD15
:108BB0000000024070B500250024272000F038FF97
:108BC0000122D1030B48FAF7F7FA0FE00A20FAF76F
:108BD000D3F900F09DF80446102C00D007E0284699
:108BE000691CCDB2C82801DDFA2070BDEEE700BFD8
:108BF0002046FAE70000024010B5052000F018FFFB
:108C00000122D1030148FAF7D7FA10BD0000024053
:108C100070B50446232000F00BFF002505E014F892
:108C2000010B00F01FFF681CC5B2042DF7DB012209
:108C3000D1030248FAF7C0FA70BD000000000240FC
:108C400070B50446222000F0F3FE002505E014F87C
:108C5000010B00F007FF681CC5B2042DF7DB0122F1
:108C6000D1030248FAF7A8FA70BD000000000240E4
:108C700070B50446242000F0DBFE002505E014F862
:108C8000010B00F0EFFE681CC5B2042DF7DB0122DA
:108C9000D1030248FAF790FA70BD000000000240CC
:108CA00070B505460026412000F0C2FE284600F0BF
:108CB000D9FE0122D1030C48FAF77EFA0FE0142006
:108CC000FAF75AF900F024F80446102C00D007E017
:108CD0003046711CCEB2C82801DDFA2070BDEEE727
:108CE00000BF2046FAE700000000024010B504462D
:108CF00004B910BD214602A0F7F766FB00BFF8E7F4
:108D00004572726F723A20253032580D0A00000009
:108D100010B52C2000F08CFE00F0FAFA0446012277
:108D2000D1030248FAF748FA204610BD000002407D
:108D30002DE9F04107460C4615460CB9BDE8F08117
:108D40003C2000F075FE384600F08CFEE0B200F0EA
:108D500089FE201200F086FE012001F07BF800263B
:108D600005E000F0D5FA28706D1C701C86B2A64292
:108D7000F7DB0122D1030248FAF71EFA00BFDDE754
:108D80000000024070B505463B2000F051FE284629
:108D900000F068FE00F0BCFA044600F0B9FA04EBFB
:108DA000002084B20122D1030248FAF705FA2046D6
:108DB00070BD00000000024070B50446302000F095
:108DC00037FE204600F04EFE022001F043F800F08E
:108DD0009FFA05460122D1030248FAF7EDF9284629
:108DE00070BD00000000024000B587B000BF00BFAA
:108DF000002001903048006840F001002E490860D2
:108E00000846006800F00100019000BF00BF00BFED
:108E100000BF00BF002001900846006840F0080035
:108E200008600846006800F00800019000BF00BF1D
:108E300000BF00BF00BF002001900846006840F05E
:108E4000080008600846006800F00800019000BFB4
:108E500000BF00BF4FF40040029001200590039036
:108E600002A91648FAF79CF800224FF40041134873
:108E7000FAF7A2F90120029000200390012004904B
:108E80000220059002A90E48FAF78AF80220029003
:108E90000120039004900220059002A90848FAF7E7
:108EA0007FF8012202210648FAF786F91420FAF722
:108EB00063F807B000BD00003038024000000240F7
:108EC000000C024070B5FFF78FFF27482749C1F813
:108ED00058022748C1F85C022648C1F86002022007
:108EE00088706520FFF702FE04469A2C04D01F48C4
:108EF000D0F8581220468847FFF77EFE6420FAF724
:108F00003BF8FFF757FE05461848D0F85812284698
:108F1000884700F0EFFC00BFFFF714FE13494870CC
:108F20000A465078D2F85C12884713480068401C03
:108F30001149086008460068322802DD40200B49CC
:108F400048700A4840780128E6D0FFF723FE074919
:108F500008700846017809A0F7F736FA4FF47A70DE
:108F6000FAF70AF870BD0000ED8C0008941C002090
:108F70005992000831930008D0010020434833394A
:108F800035564552203A202532780D0A000000005F
:108F900010B5002015E000F128014A4A12F811101E
:108FA000494A115400F12C01464A12F81110474A5F
:108FB000115400F13001434A12F81110444A11547F
:108FC000401C0428E7DB3F48B0F8680041490880AE
:108FD0003C48B0F86A004049088002203F4981F8C7
:108FE000680105213D4880F8691137490968C0F8D2
:108FF0009C1136490968C0F8A01135490968C0F8C4
:10900000A411354801883548A0F87211022180F872
:109010006A113349C0F874114FF48061C0F87811B7
:109020003049C0F880114FF48061C0F8841100F518
:10903000B47000F02FFD022028490870002048700D
:10904000084621490968416320490968816320492C
:109050000968C1631F480088204948810220887040
:109060002148C8604FF480611C4801611F4981613B
:109070004FF48061C161482201461D48F7F7F9FBB2
:109080000321002000F0DAFA12480188002000F0E5
:109090000BFB40F6B830F9F76FFF002000F0B6F890
:1090A000044613481838D0F8581220468847002044
:1090B00000F098FC04460E481838D0F858122046A4
:1090C000884710BDE6000020D4010020D801002010
:1090D000DC010020E0010020E2010020F82E002049
:1090E000F8260020F82A0020F81E0020F822002090
:1090F000AC1C002010B5FFF70DFD044604F0010084
:1091000010B12248FFF72EFD04F0040020B1FFF754
:1091100019FD1E49C91E487004F0080020B1012045
:109120001A49C91E887010BD04F0100010B100204B
:1091300000F0E0FA04F0200010B1012000F0DAFAAB
:1091400004F0400010B1022000F0D4FA04F08000D6
:1091500010B1032000F0CEFA04F4807010B10420A6
:1091600000F0C8FA04F4007010B1052000F0C2FA53
:1091700004F4806010B1062000F0BCFA04F4006032
:1091800010B1072000F0B6FA00BFCCE7971C002012
:1091900010B50446582000F04BFC204600F062FC5D
:1091A00010BD10B50446562000F042FCE0B200F0BD
:1091B00059FCC4F3072000F055FCC4F3074000F04D
:1091C00051FC200E00F04EFC10BD10B50446572097
:1091D00000F02EFCE0B200F045FCC4F3072000F0E4
:1091E00041FCC4F3074000F03DFC200E00F03AFCC7
:1091F00010BD10B5C820FFF7CBFF43F69820FFF74E
:10920000D0FF43F69820FFF7E0FF10BD70B505468C
:1092100000260024352000F00BFC284600F022FC3C
:109220000122D1030B48F9F7C7FF0FE00520F9F73A
:10923000A3FEFFF76DFD0446102C00D007E030467A
:10924000711CCEB2C82801DDFA2070BDEEE700BF68
:109250002046FAE70000024010B50446042C12D064
:1092600004DC012C07D0022C19D108E0082C0ED008
:10927000102C14D10FE00FA0F7F7A6F813E011A0FF
:10928000F7F7A2F80FE013A0F7F79EF80BE015A090
:10929000F7F79AF807E017A0F7F796F803E019A098
:1092A000F7F792F800BF00BF4FF47A70F9F764FE49
:1092B00010BD000050485920444953434F4E4E0DB5
:1092C0000A0000005048592031304D5F464C4C0D8B
:1092D0000A0000005048592031304D5F48414C464B
:1092E0000D0A0000504859203130304D5F464C4C3B
:1092F0000D0A0000504859203130304D5F48414C34
:10930000460D0A00504859204155544F0D0A00009F
:1093100010B5FF2000F003F80446204610BD70B5DC
:109320000446204603F02AF80546284670BD000092
:1093300070B500240FE18A48407801282FD1884871
:10934000807838B186488078012803D084488078B6
:10935000022824D104EBC4018148183010F83100F0
:1093600002281BD104EBC4027D49183101EBC20174
:109370004878FFF795FB0020FFF792FC05467848F8
:10938000D0F8581228468847012104EBC4027448DB
:10939000183000F83210022071498870D9E0704806
:1093A00040780128FAD004EBC4016D48183010F859
:1093B00031000128F2D16A48807802280BD1FFF7EA
:1093C0001BFC6420F9F7D8FDFFF7F4FB6420F9F7E4
:1093D000D3FD00F08FFA04EBC4016148183000EBB4
:1093E000C100807830B1012830D0022865D0032830
:1093F0007ED189E004EBC4025948183000EBC2006A
:10940000C11C204600F0E0F80221204600F016F9C9
:1094100004EBC4025248183000EBC2000189204618
:1094200000F0F4F804EBC4024D48183000EBC20021
:109430004189204600F038F92046FFF7E7FE05464F
:109440004748D0F85812284688477AE0FFF7D1FEFF
:1094500004EBC4024248183000EBC200C11C204695
:1094600000F0B2F80321204600F0E8F804EBC40253
:109470003B48183000EBC2000189204600F0C6F8D6
:1094800004EBC4023648183000EBC2004189204684
:1094900000F00AF92046FFF7B9FE05463048D0F83B
:1094A000581228468847204600F076FA05462C4890
:1094B000D0F858122846884743E00321204600F0A0
:1094C000BDF804EBC4022648183000EBC200418905
:1094D000204600F0E9F840F6B830F9F74DFD204697
:1094E000FFF794FE05461E48D0F85812284600E0C3
:1094F00018E08847204600F075FA05461848D0F86D
:109500005812284688471CE00121204600F096F8B2
:109510002046FFF77BFE05461148D0F85812284632
:1095200088470EE00321204600F088F804EBC402CF
:109530000B48183000EBC2004189204600F0B4F817
:1095400000BF00BF022104EBC4020548183000F838
:109550003210601CC4B2072C7FF7EDAE70BD000066
:10956000941C00202DE9F04107460D461446392091
:1095700000F05EFA384600F075FAE0B200F072FAD8
:10958000201200F06FFA002605E015F8010B00F03C
:1095900069FA701C86B2A642F7DB0122D1030248A9
:1095A000F9F70AFEBDE8F0810000024070B50546FB
:1095B0000C46592000F03CFA284600F053FA2046A9
:1095C00000F050FA70BD000070B505460C46312021
:1095D00000F02EFA284600F045FA14F8010B00F0CE
:1095E00041FA14F8010B00F03DFA14F8010B00F0F9
:1095F00039FA14F8010B00F035FA0122D1030248C0
:10960000F9F7DAFD70BD00000000024070B50546B4
:109610000C46322000F00CFA284600F023FAE0B2A3
:1096200000F020FA201200F01DFA0122D1030248B6
:10963000F9F7C2FD70BD00000000024070B505469C
:109640000C46342000F0F4F9284600F00BFA2046CE
:1096500000F008FA0122D1030148F9F7ADFD70BD11
:109660000000024070B506460C461546522000F038
:10967000DFF9304600F0F6F9204600F0F3F928460D
:1096800000F0F0F970BD70B506460C461546532043
:1096900000F0CEF9304600F0E5F9204600F0E2F99E
:1096A000284600F0DFF970BD70B505460C46332042
:1096B00000F0BEF9284600F0D5F9E0B200F0D2F98A
:1096C000201200F0CFF90122D1030248F9F774FD0E
:1096D00070BD00000000024070B505460C465120E8
:1096E00000F0A6F9284600F0BDF9204600F0BAF9CE
:1096F00070BD00002DE9F041044600262046FFF72A
:109700005BFB054605F0040000286DD08CBB2046AD
:10971000FFF738FB04EBC402754901EBC201C861D5
:1097200004EBC401724800EBC100808B86B204EBED
:10973000C4016F4800EBC100314682692046FFF743
:10974000F7FA002104EBC402694800EBC20080690B
:10975000815501F0E7FE04EBC401654800EBC10050
:10976000007D40F0040104EBC402614800EBC2003C
:109770000175052C38D12046FFF704FB04EBC40229
:109780005B4901EBC201C86104EBC401584800EB1E
:10979000C100808B86B204EBC401554800EBC100C8
:1097A000314682692046FFF7C3FA002104EBC40268
:1097B0004F4800EBC2008069815504EBC4024C495C
:1097C00001EBC2018869314602F046FE04EBC40198
:1097D000474800EBC100007D40F0040104EBC402E7
:1097E000434800EBC200017505F0080078B104EBB6
:1097F000C4013F4800EBC1008078012807D1012156
:109800002046FFF7D3FE3C212046FFF765FF05F019
:109810001000C8B304EBC402354901EBC20148781B
:10982000FFF7F4FC074632481838D0F8581238468B
:10983000884704EBC4012E4800EBC1008078012862
:1098400002D0022821D10FE004EBC402284901EB29
:10985000C201487800F0A0F8074625481838D0F82B
:1098600058123846884711E004EBC402204901EB46
:10987000C201487800F0B6F807461D481838D0F8FD
:1098800058123846884701E004E000BF00BFC820F6
:10989000F9F772FB05F0400040B304EBC401144833
:1098A00000EBC1008078012820D1C820F9F764FBC3
:1098B00004EBC4020E4901EBC2014878FFF7A6FC95
:1098C00007460B481838D0F858123846884704EB3A
:1098D000C402074901EBC201487800F05DF8074671
:1098E00003481838D0F8581238468847BDE8F08148
:1098F000AC1C002010B5042200210846FFF7B2FE80
:10990000022204210020FFF7BEFE042206210120CE
:10991000FFF7A8FE02220A210120FFF7B4FE04226D
:109920000C210220FFF79EFE022210211046FFF7B5
:10993000AAFE042212210320FFF794FE0222162120
:109940000320FFF7A0FE042218211046FFF78AFE2D
:1099500002221C210420FFF796FE04221E2105206E
:10996000FFF780FE022222210520FFF78CFE042251
:1099700024210620FFF776FE022228210620FFF789
:1099800082FE04222A210720FFF76CFE02222E21EC
:109990000720FFF778FE10BD70B5054600260024AD
:1099A000372000F045F8284600F05CF80122D1038A
:1099B0000B48F9F701FC0FE00520F9F7DDFAFFF796
:1099C000A7F90446102C00D007E03046711CCEB237
:1099D000C82801DDFA2070BDEEE700BF2046FAE797
:1099E0000000024070B5054600260024362000F035
:1099F0001FF8284600F036F80122D1030B48F9F78A
:109A0000DBFB0FE00520F9F7B7FAFFF781F9044611
:109A1000102C00D007E03046711CCEB2C82801DD02
:109A2000FA2070BDEEE700BF2046FAE700000240D2
:109A300010B504460122D1030948F9F7BDFB002205
:109A40004FF400410648F9F7B7FB022000F002FA94
:109A50002046FFF764FC022000F0FCF910BD000076
:109A60000000024010B504462046FFF758FC10BD28
:109A700010B501210548F9F78DFB08B9FFF73AFB4E
:109A80000349D1F86002804710BD0000000C02407D
:109A9000941C002038B504460CB9002038BD04F1F0
:109AA0003400FFF7CDF804F13800FFF7B1F804F106
:109AB0003C00FFF7DDF858A0F6F786FC3720005D84
:109AC00000903620035D3520025D94F834105FA0CD
:109AD000F6F77AFC94F83B00009094F83A3094F84A
:109AE00039203820015D60A0F6F76EFC94F83F0045
:109AF000009094F83E3094F83D203C20015D61A038
:109B0000F6F762FCFFF756F8617801EBC102644991
:109B100001EBC20048222146F6F7ABFEA07830B137
:109B200001281FD0022844D0032872D162E0607857
:109B3000E11CFFF749FD60780221FFF77FFD2189D5
:109B40006078FFF763FD61896078FFF7ADFD6078AD
:109B5000FFF75CFB054652481838D0F858122846E3
:109B6000884756E0FFF745FB6078E11CFFF72CFDC6
:109B700060780321FFF762FD21896078FFF746FDD9
:109B800061896078FFF790FD6078FFF73FFB05463D
:109B900043481838D0F85812284688476078FFF7AD
:109BA000FBFE05463E481838D0F85812284688472C
:109BB0002FE060780321FFF741FD61896078FFF7AE
:109BC00073FD40F6B830F9F7D7F96078FFF71EFB60
:109BD000054633481838D0F8581228468847607828
:109BE000FFF700FF05462E481838D0F858122846CF
:109BF00088470EE060780121FFF720FD6078FFF7CD
:109C000005FB054626481838D0F8581228468847DC
:109C100000BF00BF012041E7BEB2CCAC4950D0C567
:109C2000CFA22E2E2E2E2E2E2E2E2E2E2E2E2E2E3F
:109C30002E2E2E2E2E2E2E2E2E2E2E2E2E2E2E2E44
:109C40002E2E2E2E2E2E2E0D0A00000049503A25C3
:109C50003032642E253032642E253032642E253089
:109C600032640D0A00000000475749503A2530324F
:109C7000642E253032642E253032642E2530326435
:109C80000D0A00004D61736B3A253032642E253089
:109C900032642E253032642E253032640D0A0000E5
:109CA000AC1C00205748007800015649497840EA2A
:109CB00011105549086008460068B0F5006F04DBD4
:109CC00008460068A0F5805008604E4880784D49ED
:109CD000497801F00F0140EA01204B4948600846ED
:109CE0004068B0F5006F04DB08464068A0F580507E
:109CF00048604448C07800034249097940EA0110AD
:109D00004049497940EA11103F4988600846806817
:109D1000B0F5002F04DB08468068A0F5801088604D
:109D2000384840790007000B3649897940EA01201C
:109D30003449C97908433449086108460069B0F5D7
:109D4000002F04DB08460069A0F5801008612D484B
:109D5000407A2C49097A40EA01202B49C86008461C
:109D6000C068B0F5004F04DB0846C068A0F580303D
:109D7000C8602448C07A2349897A40EA01202249F0
:109D8000486108464069B0F5004F04DB0846406969
:109D9000A0F5803048611B48C07A1A49097B40EA27
:109DA00001201949886108468069B0F5004F04DB3D
:109DB00008468069A0F5803088611248C07B11494F
:109DC000897B40EA01201049C8610846C069B0F5A6
:109DD000004F04DB0846C069A0F58030C86109481F
:109DE000407C0849097C40EA01200749086208468E
:109DF000006AB0F5004F04DB0846006AA0F5803029
:109E000008627047680A0020900A002010B50122FD
:109E100002210948F9F7D0F9002201210648F9F793
:109E2000CBF9012210210448F9F7C6F900220821D4
:109E30000148F9F7C1F910BD0010024001B50098C2
:109E4000F9F79AF808BD00E000BF0100A0F1010099
:109E5000FAD1704711B527E0009CB4F5617F02D9B3
:109E60004FF4617400E0009C23464FF0E024A069A9
:109E70003E2404FB1301002908DB00BF4FF0E0245F
:109E8000A26982420DDA8A42F8DA0AE04FF23024FF
:109E9000214400BF4FF0E024A2698242FADD8A42E9
:109EA000F8DC009CE41A0094009C002CD4D118BD6E
:109EB00010B501213948F9F76DF9C401022137487D
:109EC000F9F768F904EB80144FF400513348F9F7BF
:109ED00061F904EB401032490870084600783149B6
:109EE00008703148007800F0800028B1012210216C
:109EF0002E48F9F761F904E0002210212B48F9F708
:109F00005BF92948007800F0200028B10122D10334
:109F10002748F9F751F905E000224FF400412448A1
:109F2000F9F74AF92048007800F0040068B149F2D6
:109F3000187020490968486298201F4908601A482B
:109F4000007800F0FB00184908701748007800F00E
:109F5000020070B1052004E00021184A22F8101018
:109F6000401C0928F8DB1048007800F0FD000E497D
:109F700008700D48007800F0010070B1092004E07D
:109F800000210E4A22F81010401C0D28F8DB06486C
:109F9000007800F0FE000449087010BD000802407F
:109FA000D8000020DA000020080B00200004024046
:109FB00000100240B804002050000020E6000020FD
:109FC00000B587B000BF002001901048006840F045
:109FD00002000E4908600846006800F00200019087
:109FE00000BF00BF0022C0210948F9F7E5F8C020F2
:109FF000029011200390002004900320059002A9F4
:10A000000348F8F7CDFF07B000BD0000303802402C
:10A010000004024010B5142200213E4800F088F8E8
:10A020003C4840783B49097840EA012000EE100A9C
:10A03000B8EEC00A384880ED000A90ED000ADFED66
:10A04000370AB4EEE00AF1EE10FA0CDD90ED000AEA
:10A05000F7EE000A30EE600ADFED310A30EE600AFA
:10A0600080ED000A04E02C4890ED000A80ED000A23
:10A070002848C0782749897840EA012000EE100A74
:10A08000B8EEC00A274880ED000A90ED000ADFED27
:10A09000230AB4EEE00AF1EE10FA0CDD90ED000AAE
:10A0A000F7EE000A30EE600ADFED1D0A30EE600ABE
:10A0B00080ED000A04E01B4890ED000A80ED000AE4
:10A0C00000200FE0811C4900491C124A525C811C8F
:10A0D000104B13F8111042EA012109B2124A22F87A
:10A0E0001010401C0428EDDB00200FE0811D49000A
:10A0F000491C084A525C811D064B13F8111042EAB4
:10A10000012109B2094A22F81010401C0428EDDB95
:10A1100010BD0000F40A0020140000200000704769
:10A1200000FF7F47180000202C0000203400002092
:10A130002DE9F04107460D46164600F053FDA020DC
:10A1400000F026FD00F078FD00B12CE0281200F0B0
:10A150001FFD00F071FD00B125E0E8B200F018FD30
:10A1600000F06AFD00B11EE000F03CFDA12000F00F
:10A170000FFD00F061FD00B115E000240CE000F0DF
:10A18000E5FC3855701EA04202D000F0ABFC01E0A7
:10A1900000F0C8FC601C84B2B442F0DB00F03AFD71
:10A1A0000120BDE8F08100F035FD0020F9E7000056
:10A1B00010B5294890ED000ABDEEC00A10EE100A55
:10A1C000000A26490870244890ED000ABDEEC00A36
:10A1D00010EE100A4870224890ED000ABDEEC00A49
:10A1E00010EE100A000A88701D4890ED000ABDEEBE
:10A1F000C00A10EE100AC870002010E0194931F8AA
:10A200001010C1F30722811C144B03F811201549CB
:10A2100011F81020811C4900491C5A54401C042884
:10A22000ECDB002010E0104931F81010C1F30722D8
:10A23000811D0A4B03F811200B4911F81020811DD4
:10A240004900491C5A54401C0428ECDB142200210C
:10A25000024800F00BF810BD14000020E00A0020B6
:10A26000180000202C000020340000202DE9F047C9
:10A270000746884691464646002533E015B106F06C
:10A280001F0020BB00F0C6FC00240AE000F0AAFC7E
:10A29000A02000F07DFC00F0CFFC00B904E0601CC1
:10A2A00084B2B4F57A7FF1DB00BFB4F57A7F00D1D8
:10A2B00036E0301200F06CFC00F0BEFC00B12FE084
:10A2C000F0B200F065FC00F0B7FC00B128E0785D6A
:10A2D00000F05EFC00F0B0FC00B121E0701C86B222
:10A2E000681C85B24D45C9DB00F094FC00240AE0EF
:10A2F00000F078FCA02000F04BFC00F09DFC00B9C1
:10A3000004E0601C84B2B4F57A7FF1DB00BFB4F5E1
:10A310007A7F00D104E000F07DFC0120BDE8F087E9
:10A3200000F078FC0020F9E713B50C464FF6FF73F8
:10A33000012269460248FBF79BF900981CBD00000A
:10A34000B00600200000000010B582B01446CDE930
:10A3500000010023009A2360194B21F0004098422D
:10A360002ADA024328D0B0F5801FA8BF226810DA8D
:10A370009FED150B53EC102B9DED000B51EC100BCA
:10A3800003F052FACDE900016FF0350221F00040F0
:10A3900022600F4B6FF31E5103EB205010442060DE
:10A3A00041F0FF5040F0005001909DED000B00BFC8
:10A3B00002B051EC100B10BD9DED000BF8E7000052
:10A3C0000000F07F0000000000000000000050438B
:10A3D00002FCFFFF3F48007898BB01203D49087010
:10A3E0003D48008840F6B831884203DD01203B49F2
:10A3F00008706EE03848008840F6BE21884203DDD0
:10A4000002203649087064E03348008840F6C411E1
:10A41000884203DD0320314908705AE02E48008845
:10A4200040F6CA01884203DD04202C49087050E040
:10A4300029480088B0F5FA6F4BDD052027490870E0
:10A4400047E0FFE724480088B0F5396F03DD0120BD
:10A45000224908703DE02048008840F69621884255
:10A4600009DD1D48008840F67C31884203DA02206D
:10A470001A4908702DE01848008840F69C1188425F
:10A4800009DD1548008840F68221884203DA03205E
:10A49000124908701DE01048008840F6A201884269
:10A4A00009DD0D48008840F68811884203DA04204F
:10A4B0000A4908700DE008480088B0F5FA6F08DD19
:10A4C0000548008840F68E01884202DA05200349DB
:10A4D00008707047FA010020140B0020F9010020D9
:10A4E00010B5002280210D48F8F766FE6420F8F7C9
:10A4F00043FD012280210948F8F75EFE0122084948
:10A500000848FBF775F8012207490848FBF770F87F
:10A510006FF0010006490968086110BD000C024097
:10A52000A901002068060020A8010020F8060020EC
:10A530002006002010B56FF001000D490968086180
:10A540000B48F9F7FBFF0B4800680B490860002037
:10A55000084908600848008881B2084801F07CFF7B
:10A5600005480068052802DD01200549086010BD86
:10A5700020060020B4010020C4010020941800200F
:10A58000C801002010B50122D1021548F8F714FEC9
:10A590000A2001F003FF134A1221102000F05EFA96
:10A5A0004FF4C870FFF74AFC0F480178062000F00E
:10A5B0007BFAC820FFF742FC0C480178072000F026
:10A5C00073FAC820FFF73AFC09480178092000F027
:10A5D0006BFAC820FFF732FCFFF764FB10BD0000E8
:10A5E000000C0240680A0020C4000020C5000020C2
:10A5F000C600002000B52DED108B8BB0FE48006822
:10A6000007280CD2DFE800F0040C156B737DFE0008
:10A610000221082000F048FA0120F749086013E2FF
:10A62000F64A0321084600F019FA0220F2490860B0
:10A630000AE2F248C01EC0780104F048C01E00794A
:10A6400041EA0020ED49C91EC9780843EC49086376
:10A650000846006BB0F5000F04DB0846006BA0F164
:10A6600080700863E649086B03F077F841EC180B3B
:10A670009FEDE40B53EC102B02F07EFEE04AC2E9A2
:10A680000E011146486803F068F841EC1A0BDC48EB
:10A6900090ED0E1BB0EE410AF0EE610A53EC102B68
:10A6A00051EC1A0B03F0C0F841EC180BD4490868C0
:10A6B00003F053F841EC1A0B9FEDD40B53EC102B25
:10A6C00003F0B2F841EC190B53EC182B02F098FD93
:10A6D000CB4AC2E912010320C7490860B4E1012155
:10A6E000082000F0E1F90420C3490860ACE1C34A46
:10A6F000D21E0321002000F0B1F90520BE490860F8
:10A70000A2E1BE48C01E00780004BC49C91E4978B9
:10A7100040EA0120B949C91E89780843B84948620E
:10A720000846406AB0F5000F04DB0846406AA0F115
:10A7300080704862B249486A03F00FF841EC180B88
:10A740009FEDB00B53EC102B02F016FEAC4AC2E9A1
:10A750000A011146C86903F000F841EC1D0BA84836
:10A7600090ED0A1BB0EE410AF0EE610A53EC102B9B
:10A7700051EC1D0B03F058F841EC1B0BA049486944
:10A7800002F0EBFF41EC1C0B53EC1B2B02F038FDED
:10A7900041EC190B9A4890ED0A2BB0EE420AF0EE0C
:10A7A000620A90ED0E2BB0EE421AF0EE621A53ECF4
:10A7B000102B51EC110B03F037F841EC1A0B53EC52
:10A7C000192B03F031F841EC180B8D49C86802F0E1
:10A7D000C4FF41EC1B0B8A4890ED0E1BB0EE410A02
:10A7E000F0EE610A53EC102B51EC1B0B03F01CF83C
:10A7F00041EC190B8249086A02F0AFFFCDE9000174
:10A800007F4800E06EE090ED0A1BB0EE410AF0EEEA
:10A81000610A53EC102B9DED001B51EC110B03F062
:10A8200003F8CDE902017649886902F096FF41EC10
:10A830001F0B9DED020B53EC102B02F0E1FC41ECE1
:10A840001E0B6F4890ED0A1BB0EE410AF0EE610A54
:10A8500053EC102B51EC1E0B02F0E6FFCDE9040186
:10A860006749086902F079FF41EC1D0B9DED040B6F
:10A8700053EC102B02F0C4FC41EC1C0B604890ED33
:10A880000A1BB0EE410AF0EE610A53EC102B51ECBA
:10A890001C0B02F0C9FF41EC1B0B5949886802F000
:10A8A0005CFF53EC1B2BCDE906019DED060B51EC33
:10A8B000100B02F0A5FC41EC1A0B53EC192B02F023
:10A8C0009FFC53EC182BCDE908019DED080B51ECD2
:10A8D000100B02F095FC4A4AC2E9100106204649D5
:10A8E0000860B1E04B49B1F9000002F036FF41ECDD
:10A8F000190B434890ED101BB0EE410AF0EE610ACF
:10A900009FED451B53EC112B51EC100B02F034FD65
:10A9100041EC1A0B53EC192B02F072FC41EC180BB2
:10A920009FED3F0B53EC102B03F07CF832D83448EA
:10A9300090ED101BB0EE410AF0EE610A9FED381B5E
:10A9400053EC112B51EC100B02F06EFE22D031496A
:10A95000B1F9000002F001FF41EC190B284890ED1D
:10A96000101BB0EE410AF0EE610A9FED2B1B53EC79
:10A97000112B51EC100B02F0FFFC41EC1A0B53ECC5
:10A98000192B02F03DFC41EC180B02F0B9FE2649F0
:10A99000088255E01A4890ED101BB0EE410AF0EE27
:10A9A000610A51EC100B02F0EDFB41EC190B9FED2D
:10A9B0001A0B53EC102B02F0DFFC41EC180B02F0E9
:10A9C0006FFE00B213490880B1F9000002F0C5FE25
:10A9D00041EC190B0A4890ED101BB0EE410AF0EE65
:10A9E000610A9FED0D1B53EC112B51EC100B02F083
:10A9F000C3FC41EC1A0B19E0D0000020CA00002073
:10AA0000900A00200000000000000F41000000003C
:10AA10000000E03F3400002000000000000059402A
:10AA20000000000000000000140B002053EC192B64
:10AA300002F0E6FB41EC180B02F062FE05490882C9
:10AA400000200549086000BF00BF0BB0BDEC108BB3
:10AA500000BD0000140B0020D00000202DE9F041C3
:10AA600005460E46174600224FF400610D48F8F7E0
:10AA7000A3FB0A2001F092FC45F0800001F0D4FE17
:10AA8000002403E000F060FE3855641CB442F9DB9A
:10AA90000122D1020348F8F78FFB0A2001F07EFC67
:10AAA000BDE8F081000C024070B505460C4600225E
:10AAB0004FF400610A48F8F77FFB0A2001F06EFCB2
:10AAC000284601F0B1FE204601F0AEFE0122D1027F
:10AAD0000348F8F771FB0A2001F060FC70BD00002C
:10AAE000000C024010B54FF400000949086000F066
:10AAF00011F840200649086000F00CF84FF480007F
:10AB00000349086000F006F880200149086010BD84
:10AB100018040240002001E0411CC8B22828FBDBD9
:10AB20007047000010B5802007490860FFF7F2FF6A
:10AB3000402005490860FFF7EDFF4FF4800002490F
:10AB40000860FFF7E7FF10BD1804024070B500244D
:10AB5000002516E06006040E40200C490860FFF74F
:10AB6000D9FF0A480838006800F0800008B1601C6E
:10AB7000C4B24FF4800005490860FFF7CBFF681CA2
:10AB8000C5B2082DE6DB204670BD00001804024067
:10AB900070B5044600251FE004F0800018B1802045
:10ABA0000F49086003E04FF400000D490860FFF70B
:10ABB000B1FF40200A490860FFF7ACFF4FF4800066
:10ABC00007490860072D01D1802008606006040E47
:10ABD000FFF7A0FF681CC5B2082DDDDB70BD0000CB
:10ABE0001804024010B58020094908604020086020
:10ABF000FFF790FF4FF4000005490860FFF78AFF58
:10AC00004FF4800002490860FFF784FF10BD000088
:10AC10001804024010B54FF40000064908604020B7
:10AC20000860FFF777FF802002490860FFF772FF96
:10AC300010BD00001804024010B580200B490860C8
:10AC400040200860FFF766FF08480838006800F0F9
:10AC5000800008B1012400E000244FF48000034983
:10AC60000860FFF757FF204610BD0000180402409F
:10AC70002DED0A8BF8F772FCFCF722F9FAF75AFE71
:10AC8000FAF70CFEFAF7AEFDFBF744F9FBF75EF9B5
:10AC9000FBF778F9FBF7A2F8FBF794F9FAF740FF16
:10ACA000FAF75CFFFAF778FFFAF794FFFAF7B4FFC8
:10ACB000FAF7EEFFFBF7A2F9FBF7E0F8FBF704F970
:10ACC000FAF7CCFFFBF73AF86420FFF7B7F801F08A
:10ACD0004FFD6420FFF7B2F8FFF754FCFFF796F83A
:10ACE000FDF734FDFC49FD4800F02EFCFFF7F8FBB2
:10ACF000FB480068C06840F02000F9490968C86056
:10AD0000F848F9F7C7FB3C21F748F9F721FD49F26C
:10AD10001870F54909684862F448F9F7FAFF042108
:10AD2000F248FAF72BF8F248F9F7B4FB0421F0489F
:10AD3000FAF724F847F23050ED4909688863432058
:10AD4000EA4909688863FFF73BF9FFF763F941F2C5
:10AD50007070E849488310226421E748FFF7E8F95A
:10AD6000002007E0E4490A5C00F12801E14B23F8E8
:10AD70001120401C0C28F5DBDF48407BDE49097BB5
:10AD800040EA0120DB49A1F86800DB48C07BDA49D2
:10AD9000897B40EA0120D749A1F86A0008221421E2
:10ADA000D648FFF7C5F9D5484078D449097840EA34
:10ADB000012000B2D2490880D048C078CF498978B4
:10ADC00040EA012000B2CF490880CC484079CB4905
:10ADD000097940EA012000B2CB490880C748C07910
:10ADE000C649897940EA012000B2C84908801AE2C0
:10ADF000C048B0F86C00012827D1002007E000F11E
:10AE00002801BC4A12F81110BB4A1154401C0C28EE
:10AE1000F5DBB848B0F868000012B7490873B548C8
:10AE200090F868004873B348B0F86A00001288735D
:10AE3000B04890F86A00C87310226421AE48FFF74A
:10AE400015FA0220AB49A1F86C00B148006801284E
:10AE500006D1FEF737F8FEF79BF80220AC490860F0
:10AE6000AB48006802280CD1FEF702FEA148B0F8FA
:10AE70006C00022805D100209E49A1F86C0001F069
:10AE80009FF94021A34800F0DBFBA3490860084676
:10AE90000068002809DD9F484078072805D008464B
:10AEA000008881B29B48FBF7E3FC9C48006830B106
:10AEB000FCF7D4FDFFF79EFB00209849086001F0E5
:10AEC0005FFBFDF74FFCFEF7F3FFFDF7B5FB89488D
:10AED000008800EE100AB8EE400A9148D0ED000A52
:10AEE00030EE200ADFED8F0A80EE201A8E4890EDBA
:10AEF000000AB4EE401AF1EE10FA3BD07D4800880B
:10AF000000EE100AB8EE400A8548D0ED000A30EE97
:10AF1000200ADFED840A80EE201A834880ED001AB3
:10AF200090ED000AF3EE090AB4EEE00AF1EE10FA31
:10AF300003DDB3EE090A80ED000A7248B0F90000A3
:10AF400000EE100AB8EEC00A6D48B0F9000000EE3D
:10AF5000900AF8EEE00A744890ED001A00EE810ABB
:10AF6000DFED720A80EE201AB0EE418AB0EE480A98
:10AF7000FDF7A4FC5F48408800EE100AB8EE400AD6
:10AF80006B48D0ED000A30EE200ADFED660A80EE55
:10AF9000201A684890ED000AB4EE401AF1EE10FA5B
:10AFA0003BD05448408800EE100AB8EE400A604892
:10AFB000D0ED000A30EE200ADFED5A0A80EE201AAA
:10AFC0005C4880ED001A90ED000AF3EE090AB4EE39
:10AFD000E00AF1EE10FA03DDB3EE090A80ED000A93
:10AFE0004A48B0F9000000EE100AB8EEC00A464820
:10AFF000B0F9000000EE900AF8EEE00A4D4890ED3E
:10B00000001A00EE810ADFED490A80EE201AB0EE48
:10B01000418AB0EE480AFDF7CDFC47480068474931
:10B02000086031480068406A434908600846006883
:10B0300042490968401A4249884205DA4148006895
:10B04000401C404908600DE03B4800683B490968E6
:10B05000401A4CF25031884204DD3A480068401EE4
:10B060003849086037480068C0EB00403249096839
:10B07000084435490860084600684FF6FF7101EA48
:10B0800010403249888230480088C8823049B1F97E
:10B09000000002F062FB41EC190B2E48008800EE24
:10B0A000100AB8EE400ADFED2C0A20EE200A9FEDD0
:10B0B0002B1AC0EE010A9FED2A0A80EE801A11EECB
:10B0C000104A204602F0CEFD9FED260B53EC102BCC
:10B0D00002F0AAFB4AE00000D8050020B0060020DC
:10B0E0008807002090050020B804002048050020B3
:10B0F00000050020E60000203C0000202400002085
:10B100001C0000201E000020200000202200002043
:10B11000540000201C3200204C0000208000002041
:10B120001400002000007A440C00002000401C465F
:10B130001800002010000020040000200000002063
:10B14000B03CFFFF5000002008000020140B00203E
:10B150002C0000206C00002000404E45000080457F
:10B160009EEFA73D295C8FC2F528F03F9FED2E0B87
:10B1700053EC102B02F08CFC53EC192B02F040F82E
:10B1800002F0BEFA2A4908832A49498840F6E44277
:10B1900001FB02F0C11700EB1151C1F30F31244A3A
:10B1A00011802448808800EE100AB8EE400A5FED56
:10B1B000160A60EE200A1FED171A80EE810A5FED75
:10B1C000180A80EE201ABCEEC10A10EE100A1146D1
:10B1D00048801848C08800EE100AB8EE400A5FEDBB
:10B1E000220A60EE200A1FED231A80EE810A5FED2D
:10B1F000240A80EE201ABCEEC10A10EE100A8880E4
:10B200000D48006838B14FF480410C48F7F7CAFF89
:10B210000020094908600A48007820B1FEF7C8FFFD
:10B22000002007490870E3E500000000004051409D
:10B23000140B00206C000020880000200010024049
:10B24000600000202DE9F04104460D460CB1022DAE
:10B2500001DABDE8F08126786778012E01D0002E52
:10B2600048D1052F3AD008DC012F0DD0022F11D084
:10B27000032F15D0042F37D118E0062F1CD00F2F25
:10B2800020D0102F30D123E0A81E81B2A01C00F0E6
:10B2900085FA2EE0A81E81B2A01C00F0EFFB28E08A
:10B2A000A81E81B2A01C00F051FD22E0A81E81B2B0
:10B2B000A01C00F06BFE1CE0A81E81B2A01C01F0D7
:10B2C00065FE16E0A81E81B2A01C01F0E9FA10E0AC
:10B2D000A81E81B2A01C01F05DFC0AE0A81E81B28C
:10B2E000A01C01F079FD04E06078012100F06EF807
:10B2F00000BF00BF00BFACE72DE9F04104460D469A
:10B300000CB1022D01DABDE8F081A679E779012EB2
:10B3100001D0002E58D1052F48D008DC012F0DD0C8
:10B32000022F13D0032F19D0042F47D11EE0062F70
:10B3300024D00F2F2AD0102F40D12FE0A5F10800E4
:10B3400081B204F1080000F0DBFA3CE0A5F108004E
:10B3500081B204F1080000F03FFC34E0A5F10800E0
:10B3600081B204F1080000F077FD2CE0A5F108009F
:10B3700081B204F1080000F08BFE24E0A5F1080082
:10B3800081B204F1080001F061FE1CE0A5F10800A3
:10B3900081B204F1080001F039FB14E0A5F10800C6
:10B3A00081B204F1080001F07DFC0CE0A5F1080079
:10B3B00081B204F1080001F075FD04E0E07901219B
:10B3C00000F040F800BF00BF00BF9CE7F0B5ADF251
:10B3D000044D05460E460024002701222146641C28
:10B3E00001A8425445F080022146641C4254214683
:10B3F000641C46542146FAF71FFE07462146641C8A
:10B4000001A847543A122146641C42540B48008A52
:10B41000A04201DB204601E00848008A0749488233
:10B420004A8AC86801A9F5F7DFF90448428AC16869
:10B43000034800F0FBF80DF2044DF0BD500A002067
:10B44000B006002070B5ADF5806D05460E460024AF
:10B4500000222146641C0DF8012001222146641CB3
:10B460000DF8012000222146641C0DF80120214620
:10B47000641C0DF801202146641C0DF801200322F4
:10B480002146641C0DF8012001222146641C0DF8A0
:10B49000012045F080022146601CC4B20DF8012055
:10B4A0002046611CCCB20DF80060FF2C01DC214667
:10B4B00000E0FF210948816201468A6A486A6946BC
:10B4C000F5F792F90548008D82B20448416A0020E0
:10B4D000FEF748F80DF5806D70BD0000941C00204B
:10B4E0002DE9F04100240E480568C488022C01DAD9
:10B4F000BDE8F081A01E295C601E285C41EA00279F
:10B50000A01E81B22846FAF797FD0646B74200D042
:10B51000EEE7034AD1881068FFF794FE00BFE7E723
:10B52000500A002070B500240648056B808E84B256
:10B53000022C00DA70BD21462846FFF7DDFE00BF71
:10B54000F8E70000941C002070B505460C46114930
:10B550002868884212D1104810490860002088806D
:10B56000C88008720E48C8604FF4806008820020CE
:10B57000488201220B492846FAF73AF80A488442E1
:10B5800006D16FF00100216808612046F8F782FFBC
:10B5900070BD000000100140940C0020500A0020F3
:10B5A0009410002090000020D805002010B5184805
:10B5B000808840F2FF3188420EDB002014498880E9
:10B5C00008460068002101604FF6FF730A2211A1AE
:10B5D0001348FAF74DF814E0124801780C488288B5
:10B5E0008088401C0A4B98801846006881540E4899
:10B5F000F8F7A4FF00200C49096848620A48F8F7E8
:10B6000049FF012207490648F9F7F2FF10BD000083
:10B61000500A0020CAFDBEDDD2E7B3F600000000EC
:10B62000B006002090000020D805002070B5044628
:10B630000D461646324629462046FAF779F870BD7F
:10B64000F8B504460D460026002000902FE068461D
:10B6500000F038F81948008820B99DF80000EE285D
:10B6600000D024E015480088A84208DA9DF80010B0
:10B67000124802880088401C104B1880A1549DF885
:10B6800000000F49096840EA01200D49086008469A
:10B6900000686FF44031884208D1084806880020CD
:10B6A00007490860054908803046F8BD00BF00F032
:10B6B0003BF80028CBDC0020F7E70000E801002081
:10B6C000E401002001460B4840880A4A1288904253
:10B6D0000FD008484288001D805C0870054A5288D7
:10B6E000501CC21700EB5262D211A0EBC212014BE8
:10B6F0005A8070473831002001460A4B1B88581C7D
:10B70000C31700EB5363DB11A0EBC3139AB20548D8
:10B710004088904205D003480388001DC154001F93
:10B720000280704738310020064800888030054A82
:10B730005288811AC81701EB5060C011A1EBC010EC
:10B7400080B270473831002070B500240122110307
:10B750001148F7F731FD00251AE000224FF480511F
:10B760000D48F7F729FD042000F018FE6006040ECE
:10B770004FF480410848F7F70DFD044301221103FF
:10B780000548F7F719FD042000F008FE681CC5B253
:10B79000082DE2DB204670BD000C02402DE9F04F81
:10B7A000ADF2144D054600240020CDF804044FF4FA
:10B7B000806101A8F5F78FF86878297840EA0129B7
:10B7C000E878A97840EA0126012E01DA502E70DCD3
:10B7D000B9F15F0F6EDC06EB090060287EDCF01D1E
:10B7E000C11700EB5171C1F3C701CDF8101401224C
:10B7F0002046611CCCB201A90A542046611CCCB27F
:10B8000001A90A542046621CD4B201AADDF8101422
:10B8100011540027BB462FE0002001A9085582469D
:10B820001BE009EB070188B20DF20C41F6F79CFE14
:10B8300001A8005D9DF80C1401FA0AF1084301A962
:10B840000855781C87B2B74203DB0120CDF8040409
:10B8500006E00AF1010000F0FF0ABAF1080FE0DB90
:10B8600000BF601CC4B2DDF80404012800D107E069
:10B870000BF1010000F0FF0BDDF810048345CBDB7A
:10B8800000BF214601A8FAF7D7FB80462046611C7D
:10B89000CCB201A901F800804FEA28222046611CA1
:10B8A000CCB201A90A541448008AA04203DB204606
:10B8B00003E017E012E01048008A0F4948824A8AE4
:10B8C000C86801A9F4F790FF0B48428AC1680B4889
:10B8D000FFF7ACFE0DF2144DBDE8F08F0220CDF85D
:10B8E000080402E00320CDF808040120DDF8081464
:10B8F000FFF76CFD00BFEDE7500A0020B006002006
:10B900002DE9F04FADF20C4D054600240020CDF896
:10B9100000044FF480616846F4F7DDFF6878297809
:10B9200040EA0129E878A97840EA0126012E01DAE7
:10B93000502E71DCB9F15F0F6FDC06EB0900602857
:10B94000FADCF01DC11700EB5171C1F3C7080022EA
:10B950002046611CCCB20DF8002001222046611C5B
:10B96000CCB20DF8002000222046611CCCB20DF8AC
:10B9700000202046611CCCB20DF800202046611C3E
:10B98000CCB20DF8002008F10300C2B22046611CC1
:10B99000CCB20DF8002001222146601CC4B20DF883
:10B9A00001202046611CCCB20DF800202046611C0D
:10B9B000CCB20DF8008000274FF0000A32E00020E2
:10B9C0000DF8040083461CE009EB070188B20DF571
:10B9D0008161F6F7C9FD1DF804009DF8081401FA0D
:10B9E0000BF10843C0B20DF80400781C87B2B742CF
:10B9F00003DB0120CDF8000406E00BF1010000F0AC
:10BA0000FF0BBBF1080FDFDB00BF601CC4B2DDF829
:10BA10000004012802D107E024E01FE00AF1010040
:10BA200000F0FF0AC245CADB00BFFF2C01DC214643
:10BA300000E0FF211048816201468A6A486A69462F
:10BA4000F4F7D2FE0C48008D82B20B48416A002008
:10BA5000FDF788FD0DF20C4DBDE8F08F0220CDF80A
:10BA6000040402E00320CDF804040120DDF80414EE
:10BA7000FFF7E8FC00BFEDE7941C00202DE9F04F34
:10BA8000ADF2144D054600240020CDF8040468787A
:10BA9000297840EA0129E878A97840EA0126012EB0
:10BAA00001DA602E71DCB9F15F0F6FDC06EB090083
:10BAB00060287FDCF01DC11700EB5171C1F3C70195
:10BAC000CDF8101401222046611CCCB201A90A5401
:10BAD00002222046611CCCB201A90A542046621CF5
:10BAE000D4B201AADDF8101411540027BB462FE090
:10BAF000002001A9085582461BE009EB070188B226
:10BB00000DF20C41F6F74CFD01A8005D9DF80C14F8
:10BB100001FA0AF1084301A90855781C87B2B74217
:10BB200003DB0120CDF8040406E00AF1010000F077
:10BB3000FF0ABAF1080FE0DB00BF601CC4B2DDF8F9
:10BB40000404012800D107E00BF1010000F0FF0B15
:10BB5000DDF810048345CBDB00BF214601A8FAF7CE
:10BB60006BFA80462046611CCCB201A901F8008026
:10BB70004FEA28222046611CCCB201A90A5414487D
:10BB8000008AA04203DB204603E017E012E01048E1
:10BB9000008A0F4948824A8AC86801A9F4F724FE3E
:10BBA0000B48428AC1680B48FFF740FD0DF2144D67
:10BBB000BDE8F08F0220CDF8080402E00320CDF8A4
:10BBC00008040220DDF80814FFF700FC00BFEDE7D1
:10BBD000500A0020B00600202DE9F04FADF20C4DC8
:10BBE000054600240020CDF800046878297840EA52
:10BBF0000129E878A97840EA0126012E01DA602EB1
:10BC000072DCB9F15F0F70DC06EB09006028FADC2A
:10BC1000F01DC11700EB5171C1F3C7080022204687
:10BC2000611CCCB20DF8002001222046611CCCB270
:10BC30000DF8002000222046611CCCB20DF8002037
:10BC40002046611CCCB20DF800202046611CCCB20D
:10BC50000DF8002008F10300C2B22046611CCCB2EE
:10BC60000DF8002001222146601CC4B20DF801200D
:10BC700002222046611CCCB20DF800202046611C37
:10BC8000CCB20DF8008000274FF0000A32E000200F
:10BC90000DF8040083461CE009EB070188B20DF59E
:10BCA0008161F6F77DFC1DF804009DF8081401FA87
:10BCB0000BF10843C0B20DF80400781C87B2B742FC
:10BCC00003DB0120CDF8000406E00BF1010000F0D9
:10BCD000FF0BBBF1080FDFDB00BF601CC4B2DDF857
:10BCE0000004012802D107E024E01FE00AF101006E
:10BCF00000F0FF0AC245CADB00BFFF2C01DC214671
:10BD000000E0FF211048816201468A6A486A69465C
:10BD1000F4F76AFD0C48008D82B20B48416A00209E
:10BD2000FDF720FC0DF20C4DBDE8F08F0220CDF8A0
:10BD3000040402E00320CDF804040220DDF804141A
:10BD4000FFF780FB00BFEDE7941C00202DE9F04FCA
:10BD5000ADF2044D064600241EB90DF2044DBDE8B7
:10BD6000F08F7078317840EA0127F078B17840EAB6
:10BD70000125012D63DB602D61DC5F2F5CDC781910
:10BD8000002859DB7819602856DC01222046611C06
:10BD9000CCB201A90A5403222046611CCCB201A9ED
:10BDA0000A546806020E2046611CCCB201A90A544E
:10BDB0004FF0000816E007EB080188B2F6F7C0FB69
:10BDC00081464FEA29222046611CCCB201A90A54BF
:10BDD0002046611CCCB201A901F8009008F10100D5
:10BDE0001FFA80F8A845E6DB214601A8FAF724F9F6
:10BDF00082462046611CCCB201A901F800A04FEA9E
:10BE00002A222046611CCCB201A90A541048008A9B
:10BE1000A04201DB204601E00D48008A0C4948821F
:10BE20004A8AC86801A9F4F7DFFC0948428AC16858
:10BE30000848FFF7FBFB90E74FF0020B01E04FF0E3
:10BE4000030B59460320FFF7C1FA00BF85E7000046
:10BE5000500A0020B00600202DE9F04FADF2044D4D
:10BE600006468A4600241EB90DF2044DBDE8F08F47
:10BE70007078317840EA0127F078B17840EA0125FE
:10BE8000012D79DB602D77DC5F2F72DC78190028BB
:10BE90006FDB781960286CDC00222046611CCCB274
:10BEA00001A90A5401222046611CCCB201A90A54FE
:10BEB00000222046611CCCB201A90A542146601C14
:10BEC000C4B201A842542046611CCCB201A90A5454
:10BED000022000EB4500401CC2B22046611CCCB2DF
:10BEE00001A90A5401222046611CCCB201A90A54BE
:10BEF00003222046611CCCB201A90A546806020E36
:10BF00002046611CCCB201A90A544FF0000816E08B
:10BF100007EB080188B2F6F713FB81464FEA2922A6
:10BF20002046611CCCB201A90A542146601CC4B24F
:10BF300001A800F8019008F101001FFA80F8A84557
:10BF4000E6DBFF2C01DC214600E0FF210E48816288
:10BF500001468A6A486A01A9F4F746FC0A48008D3E
:10BF600082B20948416A0020FDF7FCFA7CE703E051
:10BF7000FFE74FF0020B01E04FF0030B594603209F
:10BF8000FFF760FA00BF6FE7941C00202DE9F04F27
:10BF9000ADF2044D054600241DB90DF2044DBDE877
:10BFA000F08F6878297840EA0127E878A97840EA94
:10BFB0000126012E60DB602E5EDC5F2F59DCB81994
:10BFC000602856DC01222046611CCCB201A90A542B
:10BFD00004222046611CCCB201A90A547006020E4C
:10BFE0002046611CCCB201A90A544FF0000816E0AB
:10BFF00007EB080188B2F6F7ADFA81464FEA29222D
:10C000002046611CCCB201A90A542146601CC4B26E
:10C0100001A800F8019008F101001FFA80F8B0456E
:10C02000E6DB214601A8FAF707F882462046611CA4
:10C03000CCB201A901F800A04FEA2A222046611CD7
:10C04000CCB201A90A541048008AA04201DB204664
:10C0500001E00D48008A0C4948824A8AC86801A953
:10C06000F4F7C2FB0848428AC1680848FFF7DEFAC5
:10C0700093E74FF0020B01E04FF0030B5946042009
:10C08000FFF7A4F900BF88E7500A0020B00600209F
:10C090002DE9F04FADF2044D06468A4600241EB944
:10C0A0000DF2044DBDE8F08F7078317840EA012739
:10C0B000F078B17840EA0125012D76DB602D74DC43
:10C0C0005F2F6FDC781960286CDC00222046611C31
:10C0D000CCB201A90A5401222046611CCCB201A9AC
:10C0E0000A5400222046611CCCB201A90A54204601
:10C0F000611CCCB201A90A542046611CCCB201A932
:10C100000A54022000EB4500401CC2B22146601CCC
:10C11000C4B201A8425401222046611CCCB201A93C
:10C120000A5404222046611CCCB201A90A546806B4
:10C13000020E2046611CCCB201A90A544FF000083F
:10C1400016E007EB080188B2F6F704FA81464FEAD9
:10C1500029222046611CCCB201A90A542046611C48
:10C16000CCB201A901F8009008F101001FFA80F893
:10C17000A845E6DBFF2C01DC214600E0FF210F484B
:10C18000816201468A6A486A01A9F4F72DFB0B48CF
:10C19000008D82B20948416A0020FDF7E3F97FE78C
:10C1A00003E0FFE74FF0020B01E04FF0030B5946AD
:10C1B0000420FFF747F900BF72E70000941C00203D
:10C1C00010B5002015E000F12801634A12F81110A3
:10C1D000624A115400F12C015F4A12F81110604AB2
:10C1E000115400F130015C4A12F811105D4A1154EB
:10C1F000401C0428E7DB5848B0F868005A4908801A
:10C200005548B0F86A005949088059494878FCF700
:10C2100047FC0020FCF744FD04465648D0F858126D
:10C220002046884701205249087091F86901FCF7BF
:10C2300037FC0020FCF734FD04464E48D0F8581275
:10C240002046884701204A4981F86801022049496F
:10C2500088704FF4FA70F6F78FFEFCF7CDFC4FF4C0
:10C26000FA70F6F789FEFCF7A5FC04464148D0F8C1
:10C27000581220468847FDF73DFB00BFFCF762FCE3
:10C280003C4948700A465078D2F85C1288473A48D0
:10C290000068401C3849086008460068322802DD02
:10C2A000402034494870334840780128E6D04FF4A4
:10C2B0007A70F6F761FE02202D4981F868010521A8
:10C2C0002B4880F8691125490968C0F89C11244958
:10C2D0000968C0F8A01123490968C0F8A4112348CF
:10C2E00001882348A0F8721100F5B470FDF7D2FB65
:10C2F00002201F4908700020487008461749096845
:10C30000416317490968816316490968C163164882
:10C3100000881749488103210020FDF78FF9124852
:10C3200001880020FDF7C0F940F6B830F6F724FE8A
:10C330000020FCF76BFF04460E48D0F85812204648
:10C3400088470020FDF74EFB04460A48D0F85812F3
:10C350002046884710BD0000E6000020D4010020E0
:10C36000D8010020DC010020E0010020E2010020D3
:10C37000F82E0020941C0020D001002001B582B0CE
:10C380004FF47A70012301AA02A900900248F7F73E
:10C3900025FE9DF804000EBD6004002010B5044683
:10C3A0002046FDF757FD10BD17480068401C164990
:10C3B000086008460068092805DD01201349086067
:10C3C00000201149086012480068401C10490860AC
:10C3D00008460068632805DD01200E49086000203A
:10C3E0000B4908600C480068401C0B49086008466F
:10C3F0000068B0F57A7F05DB01200849086000205D
:10C4000005490860704700007C000020780000208B
:10C4100084000020800000208C0000208800002084
:10C4200010B5094800780949087001220848F9F751
:10C430007FF9012205490520FDF794F80122024900
:10C440000448F9F7D5F810BDA80100209414002085
:10C4500068060020F806002070B504460D4600224C
:10C4600010210448F6F7A8FE2A4621460248F9F7AB
:10C470005FF970BD000C0240F806002010B51848A6
:10C48000006840F2FF3188420DDB0020144908604B
:10C490001448002101604FF6FF730A2212A11548CB
:10C4A000F9F7E6F816E0144801780D4802680068CC
:10C4B000401C0B4B18600B4881541048F8F73EF8AD
:10C4C00000200E49096848620C48F7F7E3FF002096
:10C4D0000B490860012208490648F9F789F810BDA0
:10C4E000B401002094180020CAFDBEDDD2E7B3F6E7
:10C4F0000000000068060020A9010020200600209E
:10C50000C801002010B50B4800680068C0F3401057
:10C5100030B109480068C4B22046FFF7EDF800BF0B
:10C5200004480068C06840F0200002490968C860FB
:10C5300010BD0000880700200414014070B50446B7
:10C54000F5F728FF8020FAF72BFB2046FAF728FBA7
:10C55000FAF78EFA0546FAF7ADFB284670BD70B5BE
:10C5600005460C46F5F716FF0020FAF719FB28469A
:10C57000FAF716FB2046FAF713FBFAF79BFB70BDA0
:10C5800010B52DED048BF6F727F80446207868499E
:10C59000086008460068000208606078096808437F
:10C5A000634908600846006800020860A0780968CE
:10C5B00008435F49086008460068B0F5000F0FDBCC
:10C5C00008460068A0F1807000EE100AB8EEC00ABC
:10C5D000DFED580A80EE201A574880ED001A0BE074
:10C5E000534890ED000AB8EEC00ADFED520A80EE23
:10C5F000201A514880ED001A4F48D0ED000A9FEDF7
:10C600004F0A9FED4F1A01EE200AF2EE080A80EE63
:10C61000201A4C4880ED001AE0784B490860084623
:10C6200000680002086020790968084346490860EC
:10C6300008460068B0F5004F2BDD0968434A881AA8
:10C6400001F08BF841EC190B9FED410B53EC102BD3
:10C6500000F092FE41EC180B00F0A0FD3E4908608E
:10C660000846D0ED000A9FED3D1A9FED3D0A00EE11
:10C67000810AF7EE000A30EE200ABCEEC00A10EE86
:10C68000100A81B2374A384800780F3022F810106B
:10C6900025E02D490968A1F59A7001F05EF841EC9A
:10C6A000190B9FED2B0B53EC102B00F065FE41ECAA
:10C6B000180B00F073FD28490860084690ED000A49
:10C6C000DFED260A20EE200ABCEEC00A10EE100AAA
:10C6D00081B2244A244800780F3022F810102348F1
:10C6E0002149097830F9110000EE100AB8EEC00AAD
:10C6F0001448D0ED000AB2EE041A00EE810ABCEE36
:10C70000C00A10EE100A81B2164A17480078001DC0
:10C7100022F8101014480078401C1349087008468D
:10C720000078032801DD01200870BDEC048B10BDEA
:10C73000B00000200000004BC000002000A00C460C
:10C7400000401C46B8000020B40000203401010065
:10C750000000000000007040BC0000200000C84243
:10C7600000FF7F47140B0020A800002034000020A9
:10C7700000B587B0142102A8F4F7ADF800BF00207F
:10C7800001902648006840F00100244908600846EE
:10C79000006800F00100019000BF00BF402002903F
:10C7A00000200390049002A91D48F6F7F9FBA02091
:10C7B00002900120039000200490059002A91848DF
:10C7C000F6F7EEFBFAF776FA0120F6F7D5FB012033
:10C7D000144908700A20F6F7CFFB81210020FFF7EB
:10C7E000BEFE02200F4908700A20F6F7C5FB812122
:10C7F0000020FFF7B4FE03200A4908700A20F6F76C
:10C80000BBFB81210020FFF7AAFE0120054908702B
:10C810000A20F6F7B1FB07B000BD00003038024037
:10C8200000000240A800002070B504460122110358
:10C830001A48F6F7C1FC00252CE000224FF4805185
:10C840001648F6F7B9FC0420FFF7A8FD04F08000B5
:10C8500028B1012251031148F6F7AEFC05E0002291
:10C860004FF400510D48F6F7A7FC6006040E0420B3
:10C87000FFF794FD012211030848F6F79DFC042000
:10C88000FFF78CFD4FF480410448F6F783FC044326
:10C89000681CC5B2082DD0DB204670BD000C0240DC
:10C8A0002DE9F04FADF2144D044600250020CDF8DF
:10C8B00004046078217840EA012AE078A17840EA0F
:10C8C00001262079CDF80C04012E77DB502E75DC83
:10C8D000DDF80C04C000B042F7DBBAF15F0F6EDC8C
:10C8E0000AEB060060287EDC0027A94636E009F145
:10C8F0000500205CCDF808044FF0000B21E001207A
:10C9000000FA0BF0DDF80814084020B14FF47F4026
:10C91000CDF8100402E00020CDF810040AEB070166
:10C9200088B2DDF81014FBF71BFD781C87B2B74204
:10C9300003DB0120CDF8040406E00BF1010000F058
:10C94000FF0BBBF1080FDADB00BFDDF804040128A0
:10C9500000D107E009F1010000F0FF09DDF80C0447
:10C960008145C4DB00BF01222846691CCDB20DF809
:10C9700000200F222846691CCDB20DF800200DEBD7
:10C98000050021680160281DC5B229466846F9F7EF
:10C9900053FB804608F0FF022846691CCDB20DF813
:10C9A00000204FEA28222846691CCDB20DF800204D
:10C9B0001448008AA84203DB284603E017E012E08F
:10C9C0001048008A0F4948824A8AC8686946F3F7C6
:10C9D0000BFF0C48428AC1680B48FEF727FE0DF298
:10C9E000144DBDE8F08F0220CDF8000402E00320D2
:10C9F000CDF800040F20DDF80014FEF7E7FC00BFBF
:10CA0000EDE70000500A0020B00600202DE9F34FAA
:10CA1000ADF2144D054600240020CDF804046878DA
:10CA2000297840EA0129E878A97840EA012628799E
:10CA3000CDF80C04012E7DDB502E7BDCDDF80C04E0
:10CA4000C000B042F7DBB9F15F0F74DC09EB060000
:10CA50006028FADC0027A04636E008F10500285CD3
:10CA6000CDF808044FF0000A21E0012000FA0AF096
:10CA7000DDF80814084020B14FF47F40CDF81004D1
:10CA800002E00020CDF8100409EB070188B2DDF8C0
:10CA90001014FBF765FC781C87B2B74203DB01205A
:10CAA000CDF8040406E00AF1010000F0FF0ABAF133
:10CAB000080FDADB00BFDDF80404012800D107E02D
:10CAC00008F1010000F0FF08DDF80C048045C4DB2C
:10CAD00000BF00222046611CCCB201A90A540122E9
:10CAE0002046611CCCB201A90A5400222046611CD8
:10CAF000CCB201A90A542046611CCCB201A90A5447
:10CB00002046611CCCB201A90A54DDF81804801C2F
:10CB1000C2B22046611CCCB201A90A5401222046AF
:10CB2000611CCCB201A90A540F222046611CCCB270
:10CB300001A901E023E01FE00A5401A8204429686C
:10CB40000160201DC4B2FF2C01DC214600E0FF2162
:10CB50000F48816201468A6A486A01A9F3F744FED8
:10CB60000B48008D82B20A48416A0020FCF7FAFCAB
:10CB70000DF21C4DBDE8F08F4FF0020B01E04FF0BD
:10CB8000030B59460F20FEF75DFC00BFF0E70000E5
:10CB9000941C00202DE9F04FADF2044D0446002610
:10CBA0001CB90DF2044DBDE8F08F6078217840EAA1
:10CBB0000128E078A17840EA012794F804A0012F29
:10CBC00062DB602F60DCBAEB470F5DD1B8F15F0F1D
:10CBD00057DC08EB0700602853DC002514E0062032
:10CBE00000EB4500205C052101EB4501615C40EA5A
:10CBF0000120CDF8000408EB050188B2DDF800142F
:10CC0000FBF7A6FB681C85B2BD42E8DB012230467B
:10CC1000711CCEB20DF8002010223046711CCEB22D
:10CC20000DF800200DEB060021680160301DC6B232
:10CC300031466846F9F700FA814609F0FF023046AE
:10CC4000711CCEB20DF800204FEA29223046711C2B
:10CC5000CEB20DF800201148008AB04201DB304608
:10CC600001E00E48008A0D4948824A8AC868694630
:10CC7000F3F7BAFD0948428AC1680948FEF7D6FCB5
:10CC80008FE74FF0020B01E04FF0030B0BF0FF01B9
:10CC90001020FEF79BFB00BF83E70000500A002036
:10CCA000B00600202DE9F04FADF2044D054689464F
:10CCB00000241DB90DF2044DBDE8F08F6878297885
:10CCC00040EA0128E878A97840EA012795F804A00D
:10CCD000012F75DB602F73DCBAEB470F70D1B8F111
:10CCE0005F0F6ADC08EB0700602866DC002614E0B2
:10CCF000062000EB4600285C052101EB4601695C3B
:10CD000040EA0120CDF8000408EB060188B2DDF806
:10CD10000014FBF71DFB701C86B2BE42E8DB00224C
:10CD20002046611CCCB20DF8002001222046611C77
:10CD3000CCB20DF8002000222046611CCCB20DF8C8
:10CD400000202046611CCCB20DF800202046611C5A
:10CD5000CCB20DF8002009F10200C2B22046611CDD
:10CD6000CCB20DF8002001222046611CCCB20DF897
:10CD7000002010222046611CCCB20DF800200DEBE3
:10CD8000040029680160201DC4B2FF2C01DC21468B
:10CD900000E0FF210F48816201468A6A486A6946BD
:10CDA000F3F722FD0B48008D82B20A48416A002049
:10CDB000FCF7D8FB7EE703E0FFE74FF0020B01E052
:10CDC0004FF0030B0BF0FF011020FEF73BFB00BF01
:10CDD00070E70000941C00202DE9F047ADF5806D50
:10CDE00005468A4600246878297840EA0129E878CF
:10CDF000A97840EA012717B1B7F57F4F45D1B9F1BE
:10CE00005F0F3FDC39464846FBF7AAFA012220466D
:10CE1000611CCCB20DF8002005222046611CCCB26A
:10CE20000DF800200DEB040029680160201DC4B23C
:10CE300021466846F9F700F90646F2B22046611C21
:10CE4000CCB20DF8002032122046611CCCB20DF895
:10CE500000201248008AA04201DB204601E00F4872
:10CE6000008A0E4948824A8AC8686946F3F7BCFCC2
:10CE70000A48428AC1680A48FEF7D8FB0DF5806D62
:10CE8000BDE8F0874FF0020801E04FF0030841468B
:10CE90000520FEF79BFA00BFF0E70000500A0020D3
:10CEA000B00600202DE9F043ADF2044D054688465A
:10CEB00000246878297840EA0129E878A97840EACE
:10CEC000012616B1B6F57F4F57D1B9F15F0F52DC8D
:10CED00031464846FBF744FA00222046611CCCB29A
:10CEE00001A90A5401222046611CCCB201A90A54AE
:10CEF00000222046611CCCB201A90A542046611CC4
:10CF0000CCB201A90A542046611CCCB201A90A5432
:10CF100008F10200C2B22046611CCCB201A90A5439
:10CF200001222046611CCCB201A90A5405222046E8
:10CF3000611CCCB201A90A5401A8204429680160EF
:10CF4000201DC4B2FF2C01DC214600E0FF210E4869
:10CF5000816201468A6A486A01A9F3F745FC0A48DA
:10CF6000008D82B20848416A0020FCF7FBFA0DF2FE
:10CF7000044DBDE8F083022700E003273946052071
:10CF8000FEF760FA00BFF2E7941C00202DE9F0479D
:10CF9000ADF5806D05468A4600241DB90DF5806DFE
:10CFA000BDE8F0876878297840EA0127E878A97811
:10CFB00040EA01285F2F3CDC41463846FBF7C8F9C0
:10CFC00001222046611CCCB20DF80020062220462A
:10CFD000611CCCB20DF800200DEB04002968016043
:10CFE000201DC4B221466846F9F726F80646F2B27B
:10CFF0002046611CCCB20DF8002032122046611C84
:10D00000CCB20DF800200F48008AA04201DB204678
:10D0100001E00C48008A0B4948824A8AC868694680
:10D02000F3F7E2FB0748428AC1680748FEF7FEFAB9
:10D03000B4E74FF0020949460620FEF7C7F900BFE2
:10D04000ACE70000500A0020B00600202DE9F043B4
:10D05000ADF2044D05460F4600241DB90DF2044DF6
:10D06000BDE8F0836878297840EA0126E878A97855
:10D0700040EA01285F2E4EDC41463046FBF768F956
:10D0800000222046611CCCB201A90A54012220468C
:10D09000611CCCB201A90A5400222146601CC4B212
:10D0A00001A842542046611CCCB201A90A54204672
:10D0B000611CCCB201A90A54B81CC2B22046611C42
:10D0C000CCB201A90A5401222046611CCCB201A9AC
:10D0D0000A5406222046611CCCB201A90A5401A8B8
:10D0E000204429680160201DC4B2FF2C01DC2146C8
:10D0F00000E0FF210C48816201468A6A486A01A962
:10D10000F3F772FB0848008D82B20748416A00209D
:10D11000FCF728FAA2E74FF0020949460620FEF77D
:10D1200091F900BF9AE70000941C002010B5002977
:10D130000AD00878002807D005487844F4F760F949
:10D14000002801D0002010BD0248784410BD000026
:10D15000320E00002A0E000010B500290AD008780F
:10D16000002807D005487844F4F74AF9002801D090
:10D17000002010BD0248784410BD0000220E0000BF
:10D180001A0E000081F00041704780F000407047A7
:10D1900021F00041704720F00040704721F000422C
:10D1A000A2F16052B2F5801F01F0004328BFD2F116
:10D1B0007F6C0BD95FEA001C43EAC20242EB50705D
:10D1C00018BF704728BF20F001007047B2F5801FDC
:10D1D000BCBF184670474FEA410C1CF5001F02D235
:10D1E000084600F0B5BD70B500F0C8FB000000892E
:10D1F000FFF7F6BF4FF00040A0F580007047000039
:10D2000010B591EA030F48BF83F0004300F1488452
:10D21000841A71EB030C05D2121943EB0C03001BAB
:10D2200061EB0C01DFF824E14FEA1154A4EB135C2D
:10D230001EEA430F18BF9EEA445F73D023EA0E0331
:10D24000DCF1200E21EA045143F4801332D322FA98
:10D250000CFE10EB0E0023FA0CFE41EB0E01CCF19C
:10D26000200E03FA0EFE10EB0E0051F10001B1F595
:10D27000801FCCF1200E32D201EB045112FA0EF2D3
:10D28000BDE8104058BF7047401C38BF5FEA4202FB
:10D2900018BF7047002814BF20F0010041F10001C1
:10D2A0004FEA410313F5001F38BF7047A1F1C04199
:10D2B00000F0B2BB012A43EB0302ACF1200CDCF11D
:10D2C0001F0E32BF4FF0000E23FA0CF310EB0300D9
:10D2D00041EB0451B4EB115FD0D0A1EB045101F547
:10D2E000801149085FEA300001EB04510ED350F180
:10D2F000000038BF12FA0EFE08D1BDE81040C9E7A1
:10D30000401C38BF5FEA4202CAD1C3E7BDE8104003
:10D310004FEA410313F5001F38BF7047A1F1C04128
:10D3200000F07ABB9EEA445F08D011EA5E0FBDE8C8
:10D33000104004BF01F0004100207047BDE81040DC
:10D3400070B500F01BFB00BF64FBBE3E0000E0FFB9
:10D3500002494FF0000000F000BD00BF0000F87F60
:10D36000491058BFC1F140415B1058BFC3F1404361
:10D370008B42EFF3008070472DE9C04130B4DFF8F5
:10D38000A0C23CEA111418BF3CEA131400F0EC8070
:10D3900081EA03051CEA111444EAD57418BF1CEA9B
:10D3A000131500F0C780A4EB05044FF0004545EAD3
:10D3B000C12145EAC32341EA505143EA525304F1E3
:10D3C0007F74994204F500344FEAC0204FEAC2222C
:10D3D00008BF904200F09C804FEA13650FF24016A0
:10D3E000765D4FEA134506FB05F7C7F1807706FB2C
:10D3F00007F74FEAD737A7FB03687642C8F58038AE
:10D40000A7FB06CE38BFA8F1010807FB08E64FF0DE
:10D41000000EA6FB028CE6FB03CEDCF1000CCEF185
:10D42000004E38BFAEF1010EA6FB0C584FF00007BE
:10D430004FF00005E6FB0E87A1FB08C6A0FB07CE58
:10D4400016EB0E0645F10005E1FB076515F1E04E10
:10D450007EBFA4F580345FEA46066D4116F1800771
:10D4600045F100054FEA17274FEA066647EA0567C8
:10D47000A6F1DE46B6F1805F4FEA15251FD9384682
:10D4800024F0010C05EBC471BCF1FE6F01EB0C1133
:10D4900002D8F0BCBDE8008124425CBF01F5801ECB
:10D4A0009EEAC47F02D4F0BCBDE80081244238D497
:10D4B000F0BCA1F1C041BDE8004100F0ADBA4FEAB7
:10D4C000D22242EA43524FEAD323A7FB02864FEA15
:10D4D000D02040EA415007FB03661EEA0E0F4FEAD8
:10D4E000D12105FB026658BFA6EB0056B6EB0056ED
:10D4F0004FEA520E4EEAC37E18EB0E0E56EB530E59
:10D50000BDD518EB02085E417F1C55F10005B6E75A
:10D510004FF480154FF000074FF000064FF0000861
:10D52000ADE7F0BC4FF0000001F1C04101F0004157
:10D53000BDE8008111EA0C1F0CEA131500D00CE0C5
:10D5400013EA0C1F00F025804FF00000F0BC81EAC8
:10D55000030101F00041BDE80081F0BCBDE80041DD
:10D5600081EA030100F058BAF0BCBDE8004170B593
:10D5700000F004FA097EFC3E00F007B881EA0301DE
:10D580004FF0000001F00041704781EA030100F014
:10D5900043BAF0BCBDE800414FF00000214970479C
:10D5A000FFFDFBF9F7F5F4F2F0EEEDEBE9E8E6E468
:10D5B000E3E1E0DEDDDBDAD8D7D5D4D3D1D0CFCDEF
:10D5C000CCCBCAC8C7C6C5C4C2C1C0BFBEBDBCBB28
:10D5D000BAB9B8B7B6B5B4B3B2B1B0AFAEADACAB23
:10D5E000AAA9A8A8A7A6A5A4A3A3A2A1A09F9F9EFD
:10D5F0009D9C9C9B9A9999989797969595949393AF
:10D60000929191908F8F8E8E8D8C8C8B8B8A898945
:10D6100088888787868585848483838282818180C8
:10D620000000FF070000F87F51EA030C17D41CF537
:10D63000801F58BFBCF5801F00F10680994218BFBB
:10D64000704708BF9042704707D711F5801F58BF39
:10D6500013F5801F19D499427047894270471CF511
:10D66000801F08D5BCF5801FF7D58B4218BF7047C7
:10D6700008BF824270474FF4001C1CEB410F38BFBB
:10D680001CEB430F01D28B42704770B500F076F966
:10D69000922449004FF000514FF08053FFF760BED5
:10D6A0004FEA41034FEA5353A3F58063D3F11E03BE
:10D6B000C8BFD3F1210C0CDD4FF0004242EAC12279
:10D6C00042EA505232FA03FC8CEAE17CACEBE170A6
:10D6D0007047102BC4BF0020704703F5787CBCF165
:10D6E000FF3F04D06FF0004282EA2100704770B51E
:10D6F00000F044F94992248000207047F2E70000CE
:10D700004FEA1153A3F58063D3F11E03A8BFD3F1F1
:10D71000200C08DB4FF0004242EAC12252EA50528C
:10D7200032FA03F0704709420BD4102BC4BF00201B
:10D73000704703F5787CBCF1FF3F05D04FF0FF3018
:10D7400070474FF00000704770B500F017F900BF48
:10D750004992248000207047F0E710F0004248BF53
:10D760004042B0FA80F310FA03F10AD0C3F11D036E
:10D7700003F580634FEA415002EB035202EBD121E3
:10D7800070474FF000007047B0FA80F310FA03F1D1
:10D790000AD0C3F11D0303F580634FEA41504FEAFD
:10D7A000035202EBD12170474FF000007047000098
:10D7B00051EA030C17D41CF5801F58BFBCF5801F1D
:10D7C00000F10680994218BF704708BF9042704729
:10D7D00007D711F5801F58BF13F5801F19D4994240
:10D7E0007047894270471CF5801F08D5BCF5801F23
:10D7F000F7D58B4218BF704708BF824270474FF47D
:10D80000001C1CEB410F38BF1CEB430F01D28B42B5
:10D81000704770B500F0B2F8922449004FF0005103
:10D820004FF08053FFF79CBDDFF848C170B51CEA8C
:10D83000111E1EBF1CEA13159EEA0C0F95EA0C0F71
:10D8400000F06F8081EA030423EA4C134EEAD47E91
:10D8500021EA4C1141F4801143F48013AE44A1FB42
:10D86000024CA0FB0365AEF17F7E361955EB0C052B
:10D87000A1FB034C4CF10003A0FB021C16EB0C06B1
:10D88000654153F10003094218BF46F0010613F445
:10D89000007F0BD14FEA03314FEA0530340341EAF0
:10D8A000155140EA16506FF003020AE04FEAC32117
:10D8B0004FEAC520F40241EA555140EA56506FF054
:10D8C000020202EB2E4201EB025585EACE710AD02C
:10D8D0005FEA440C18BF24F0004450F1000041F10D
:10D8E000000120EAD47040F2FE7C624500D270BD97
:10D8F000A84214BF4FF080444FF04044002E08BFB0
:10D900000024BEF1806FA8BFA1F1C041BDE8704006
:10D9100080F282804FF0000001F1C04101F000412F
:10D9200070479EEA0C0F0CEA131518BF95EA0C0F0E
:10D9300006D04FF0000081EA030E0EF0004170BDEA
:10D9400000F01CF88900013E00F007B800F009B8AB
:10D950004FEA430C5FEA5C5C08D081EA030100F007
:10D960005BB84FEA410C5FEA5C5CF6D14FF0000017
:10D97000014970470000FF070000F87F0EF1020E1A
:10D980002EF0030E5EF8046B364205D4012A43EBF9
:10D99000030515F5001F12D8012841EB010C1CF5F9
:10D9A000001F0CD80ED14FEAD17C15F5001F0CEBEF
:10D9B0004C0C0CF1020C08BF4CEBD37C04E04FF094
:10D9C000080C01E04FEAD37C0CEB4C0526FA05F677
:10D9D00006F00706B6F1040C06D20EEB860CBDE885
:10D9E00070404CF0010C6047DFE80CF0090B0202BC
:10D9F0004FF000414FF00000A1F5002170BD194625
:10DA00001046012851EB010418BFD4F5001484BF5F
:10DA1000002001F0004170BD0808A0F500114FEA98
:10DA20003101704753EA010C17D41CF5801F58BF11
:10DA3000BCF5801F00F106808B4218BF704708BFFD
:10DA40008242704707D713F5801F58BF11F5801F1A
:10DA500019D48B4270479B4270471CF5801F08D534
:10DA6000BCF5801FF7D5994218BF704708BF904298
:10DA700070474FF4001C1CEB430F38BF1CEB410FE9
:10DA800001D2994270470FB40CBC03BCFFF7C1BE72
:10DA900010B591EA030F48BF83F000433FF5B8ABE0
:10DAA000841A71EB030C07D212198CF0004C43EB73
:10DAB0000C03001B61EB0C01DFF8A4E14FEA1154E9
:10DAC000A4EB135C1EEA430F18BF9EEA445F00F00C
:10DAD000B08023EA6E03524221EA0451C3EB6E0385
:10DAE00038BF5B1EDCF1200E25D322FA0CFE10EBB2
:10DAF0000E0043FA0CFE41EB0E01CCF1200E03FAAE
:10DB00000EFE10EB0E0051F10001CCF1200E29D4D5
:10DB100012FA0EF201EB0451BDE8104058BF7047F5
:10DB2000401C1CBFB2F1004F704700280CBF491CBD
:10DB300020F00100704712EB020E43EB030218BF06
:10DB40004FF0010E4EEA4202ACF1200CDCF11E0E49
:10DB500054D943FA0CFE10EB0E0051F1FF31CCF119
:10DB60001E0ED5D50EF1010E12FA0EFE404141EB0C
:10DB7000010101EB445C5FEA5C5C10D910EBDE70E4
:10DB800001EB045138BFBEF1004FBDE8104018BF93
:10DB9000704700280CBF491C20F00100704730D2AC
:10DBA0004FEAD42C11F5001124F400641BD0B1FA13
:10DBB00081F20B3AA41AA41ED2F12003914030FA4C
:10DBC00003F31943904001EBCC71002C01EB04519D
:10DBD000BDE81040A8BF704701F1C0414FF0000000
:10DBE00001F000417047B0FA80F310FA03F100D160
:10DBF00010BDE41A173C4805C90AE4E701EB0451DB
:10DC000010BD491001EB0451BDE810404FEA30004F
:10DC100002E04FF0000170474A0008BF0042F8D010
:10DC2000B2F5001F28BF704701F000414FF000001F
:10DC300070479EEA445F07D011EA5E0FBDE81040CE
:10DC400004BF002100207047BDE8104070B5FFF709
:10DC500095FE00BF40DFF63E83F00041104670475E
:10DC60000000E0FF43004FEAD30C4FEA3C0C434076
:10DC70001FBF40070CF1605113F0FE4F70471CF0BE
:10DC8000006F03D100200CF0004170470CF00043FE
:10DC900043EA507010B540EACC0000F00EF800BF27
:10DCA000000000924FEA0001FFF7B6BE4FF00041BE
:10DCB0004FF00000A1F5002170470EF1020E2EF08A
:10DCC000030E5EF8044B244204D44FEA4102B2F141
:10DCD0007F4F11D84FEA4003B3F17F4F0CD80ED1DC
:10DCE0004FEAD07CB2F17F4F0CEB4C0C0CF1020CE4
:10DCF00008BF4CEBD17C04E04FF0080C01E04FEA88
:10DD0000D17C0CEB4C0324FA03F404F00704B4F1C7
:10DD1000040C06D20EEB840CBDE810404CF0010C54
:10DD20006047DFE80CF0070802024FF00040A0F562
:10DD3000800010BD0846420018BFD2F1807288BF33
:10DD400000F0004010BD4FF04070E1EE100A704747
:10DD5000FF2141EAD050C00570470CF00F03092B9A
:10DD600008BF082000F05F800A2B0BD0082B18BFDB
:10DD7000704708BF1CF0400F0AD04FF000004FF072
:10DD8000000170471CF0400F18BF4FF00040704773
:10DD90001CF0100F08D020F0704300F07F4242EAE0
:10DDA000D3014FEA4370704700F0604021F07F429A
:10DDB00042EA000201F07F4040EA727070474FF083
:10DDC000FF0C4CF4E06C1CEA11531CBF9CEA030CE2
:10DDD0009445C2BFDA4201EB02517047002B0DD0CF
:10DDE000BCF1000F0FD0002A01F00041A4BF41F0A8
:10DDF000E04141F07F614FF00000704701F00041C9
:10DE00004FF00000704750EA01334FF09B0C18BFF1
:10DE10004CF0806C7FF49CAA7047F3F797B9F3F746
:10DE2000B5BBF3F73FBD1CF4801F11D01CF4E02FED
:10DE300003D06FEACC31490070474FF04050EFF308
:10DE4000008222F0704242EA000282F300887047AA
:10DE50004FF0000070470006101600061016000074
:10DE6000000000000000010203040607080900008A
:10DE7000000001020304303132333435363738398B
:10DE80004142434445464030580030313233343506
:10DE90003637383961626364656640307800040063
:10DEA0000008000000000000000200010000100057
:10DEB00002400000000000A000000000054000003B
:10DEC000000000C8000000000C4000000000409C62
:10DED00000000000194000000020BCBE000000004F
:10DEE00034400000BFC91B8E00000004B540000094
:10DEF000504BCFD06607E2CF010000006C4100001C
:10DF00003E8251AADFEEA73401000000D942000092
:10DF1000DCB5A0E23A301F97FFFFFFFFB4450000D9
:10DF2000FD25A0C8E9A3C14FFFFFFFFFFF3F000091
:10DF30000000008000000000FF3F000000000080A3
:10DF40000000000098E00008000000201C02000013
:10DF5000C4010008F0E000081C020020D4360000D4
:10DF600020020008000000000000F07F1C000000FC
:10DF700043000000F8FFFFFF0C0000000E0000004F
:10DF80000F0000002E000000100100004300000000
:10DF9000F8FFFFFF004040404040404040404141CA
:10DFA000414141404040404040404040404040406E
:10DFB0004040404040050202020202020202020208
:10DFC0000202020202202020202020202020200205
:10DFD0000202020202029090909090901010101095
:10DFE0001010101010101010101010101010101031
:10DFF00002020202020288888888888808080808C5
:10E000000808080808080808080808080808080890
:10E0100002020202400000000000000000000000B8
:10E0200000000000000000000000000000000000F0
:10E0300000000000000000000000000000000000E0
:10E0400000000000000000000000000000000000D0
:10E0500000000000000000000000000000000000C0
:10E0600000000000000000000000000000000000B0
:10E0700000000000000000000000000000000000A0
:10E080000000000000000000000000000000000090
:10E09000000000000000000001241726F3FFDE2628
:10E0A000CA0210191DC0A872C204156EFFFFFF45F9
:10E0B0000FFA13E2024B98321042014B24F408018C
:10E0C00017041374F40CF2AA02BFC804270B16211C
:10E0D0001DC0A872C204156EFFFFFF0515FA0FE2FE
:10E0E0001322053201290441526483704229180029
:040000050800018965
:00000001FF
